:100000000C94C3060C9412070C9412070C9412075C
:100010000C9412070C9412070C9412070C941207FC
:100020000C9412070C94E2160C9412070C9412070D
:100030000C94B5340C9412070C9412070C9412070C
:100040000C9412070C9412070C9457150C94120779
:100050000C94270C0C9412070C94F10B0C941207BF
:100060000C94F71B0C9412070C9459300C94120743
:100070000C94BD780C9412070C94B9730C9412076D
:100080000C9412070C9412070C941207221C271CC4
:100090002C1C351C4C1C631C731C831CA01C3E1E9A
:1000A000631C001D111D401D5E1D7B1DD51D301ED6
:1000B0000E20A0205D21DD214622F62201255E25AD
:1000C000CB2515266026AD26FE265827B7275128B2
:1000D000EC28E6298130A830EB305B317331B43144
:1000E0006732273327332733273327332733273301
:1000F0002733273327332733DE32E032E532FD3230
:10010000FF320A0D426174743A0020256420436571
:100110006C6C732000204C6F77207761726E696E73
:1001200067206C6576656C3A2025642E2564000A8C
:100130000D466F756E6420424C2D4374726C3A20EC
:10014000002564000A0D0A0D2121204D4953534911
:100150004E4720424C2D4354524C3A2025642021D6
:1001600021000A0D3D3D3D3D3D3D3D3D3D3D3D3D7B
:100170003D3D3D3D3D3D3D3D3D3D3D3D3D3D3D3DAF
:100180003D3D3D3D3D3D3D000A0D43616C69627260
:100190006174696E67207072657373757265207320
:1001A000656E736F722E2E004F4B0A0D000A0D46BE
:1001B0006C696768742D74696D65202575206D699B
:1001C0006E2020546F74616C3A2575206D696E0045
:1001D0000A0D436F6E74726F6C3A2000486561645B
:1001E000696E67486F6C64004E6F726D616C202899
:1001F0004143432D4D6F646529000A0D3D3D3D3D52
:100200003D3D3D3D3D3D3D3D3D3D3D3D3D3D3D3D1E
:100210003D3D3D3D3D3D3D3D3D3D3D3D3D3D3D0A41
:100220000D00416E676C654E69636B2020202020B5
:100230002020416E676C65526F6C6C20202020205E
:1002400020204163634E69636B2020202020202002
:100250002020416363526F6C6C20202020202020DE
:1002600020205961774779726F202020202020209C
:1002700020204865696768742056616C7565202088
:1002800020204163635A202020202020202020208D
:1002900020204761732020202020202020202020A3
:1002A0002020436F6D706173732056616C756520FB
:1002B0002020566F6C74616765205B302E31565D6F
:1002C00020205265636569766572204C6576656CA1
:1002D00020204779726F20436F6D70617373202007
:1002E00020204D6F746F722031202020202020208C
:1002F00020204D6F746F722032202020202020207B
:1003000020204D6F746F7220332020202020202069
:1003100020204D6F746F7220342020202020202058
:1003200020203136202020202020202020202020A6
:100330002020313720202020202020202020202095
:100340002020313820202020202020202020202084
:100350002020313920202020202020202020202073
:100360002020536572766F2020202020202020201E
:100370002020486F7665726761732020202020203E
:10038000202043757272656E74205B302E31415DA2
:1003900020204361706163697479205B6D41685D01
:1003A0002020323420202020202020202020202027
:1003B0002020323520202020202020202020202016
:1003C0002020323620202020202020202020202005
:1003D00020203237202020202020202020202020F4
:1003E00020204932432D4572726F72202020202038
:1003F0002020424C204C696D697420202020202050
:1004000020204750535F4E69636B2020202020201E
:1004100020204750535F526F6C6C202020202020FA
:10042000202021212120494E434F4D504154494223
:100430004C4520212121002E000A0D20444143205B
:100440006F7220493243204552524F522120436857
:1004500065636B204932432C2033567265662C202D
:1004600044414320616E6420424C2D4374726C0001
:100470005B25695D005B25695D002B204D696B7212
:100480006F4B6F70746572202B0048573A56256485
:100490002E25642053573A25642E25642563005386
:1004A000657474696E673A2564202573004861722B
:1004B0006477617265204572726F7220313A2564EB
:1004C000202121004D697373696E6720424C2D43D2
:1004D00074726C3A25642121004D6978657220455B
:1004E00072726F722100493243204552524F52219D
:1004F0002121004865696768743A20202535690024
:10050000536574706F696E743A2535690050726571
:1005100073737572653A253569004F666673657445
:100520003A20202535690048656967687420636F43
:100530006E74726F6C0044495341424C454400480C
:10054000656967687420636F6E74726F6C004449EC
:100550005341424C4544006163742E2062656172D0
:10056000696E67004E69636B3A20202020202025A9
:10057000356900526F6C6C3A2020202020202535F0
:100580006900436F6D706173733A202020253569CF
:10059000004B313A25346920204B323A253469200A
:1005A000004B333A25346920204B343A25346920F6
:1005B000004B353A25346920204B363A25346920E2
:1005C000004B373A25346920204B383A25346920CE
:1005D000004E693A2534692020526F3A253469204B
:1005E0000047733A253469202047693A2534692049
:1005F0000050313A253469202050323A25346920A0
:100600000050333A253469202050343A253469208B
:10061000004779726F202D2053656E736F72004E04
:1006200069636B25346920282533692E25692900E3
:10063000526F6C6C25346920282533692E25692971
:100640000047696572253469202825336929004EE1
:1006500069636B2025346920282533692E25782984
:1006600000526F6C6C2025346920282533692E25B3
:10067000782900596177202025346920282533699D
:1006800029004E69636B20253469202825336929A8
:10069000282533692900526F6C6C20253469202885
:1006A00025336929282533692900596177202025B8
:1006B00034692028253369292825336929004143D5
:1006C00043202D2053656E736F72004E69636B205B
:1006D00025346920282533692900526F6C6C202548
:1006E0003469202825336929005A20202020253408
:1006F0006920282533692900566F6C746167653A53
:100700002020202533692E253169560043757272E9
:10071000656E743A2020202533692E253169410009
:10072000506F7765723A20202020202534695700C9
:100730004469736368617267653A202535696D4164
:10074000680052656365697665720052432D5253A5
:1007500053493A202020202534690052432D5175F9
:10076000616C6974793A202534690052432D4368DD
:10077000616E6E656C733A25346900436F6D70610C
:1007800073730048656164696E673A202025356996
:100790000056616C75653A2020202025356900538C
:1007A000746172743A2020202025356900506F74DE
:1007B00069313A202025336900506F7469323A203C
:1007C0002025336900506F7469333A20202533693E
:1007D00000506F7469343A202025336900506F74DB
:1007E00069353A202025336900506F7469363A2004
:1007F0002025336900506F7469373A20202533690A
:1008000000506F7469383A202025336900536572AF
:10081000766F202000536574706F696E74202025F8
:10082000336900506F736974696F6E3A20253369BC
:100830000052616E67653A2533692D25336900459D
:10084000787465726E436F6E74726F6C2020004E08
:10085000693A2534692020526F3A253469200047CF
:10086000733A253469202047693A253469200048C5
:10087000693A253469202043663A253469200042CC
:100880004C2D4374726C204572726F727320002578
:10089000336420253364202533642025336420000D
:1008A00025336420253364202533642025336420D8
:1008B00000253364202533642025336420253364E8
:1008C0002000424C2054656D7065726174757265CC
:1008D00000253369202533692025336920253369B4
:1008E00020002533692025336920253369202533ED
:1008F00069200025336920253369202533692025A7
:1009000033692000424C2D4374726C20666F756E03
:1009100064200020256320202025632020202563DB
:10092000202020256320002025632020202563200F
:1009300020202563202020256320002025632020FF
:10094000202D2020202D2020202D2000313000318E
:100950003100313200466C696768742D54696D65E9
:10096000202000546F74616C3A2535756D696E00F6
:100970004163743A20202535756D696E00287265D3
:1009800073657429000A0D47656E65726174696E3E
:10099000672064656661756C7420506172616D6575
:1009A00074657220536574202564000A0D557369BF
:1009B0006E6720506172616D657465722053657455
:1009C000202564000A0D47656E65726174696E6763
:1009D0002064656661756C74204D69786572205479
:1009E00061626C65000A0D4D697865722D436F6E0A
:1009F0006669673A202725732720282575204D6FC3
:100A0000746F727329000A0D3D3D3D3D3D3D3D3DF6
:100A10003D3D3D3D3D3D3D3D3D3D3D3D3D3D3D3D06
:100A20003D3D3D3D3D3D000A0D414343206E6F7409
:100A30002063616C69627261746564210D0A000053
:100A4000008F001E01AD013B02CA025803E6037489
:100A50000402058F051B06A7063307BE074808D208
:100A6000085B09E3096B0AF20A780BFD0B810C04A1
:100A70000D860D070E870E060F840F00107B10F5F4
:100A8000106E11E5115B12CF124213B313231492AF
:100A900014FE146A15D3153B16A11605176717C85F
:100AA0001727188318DE1837198E19E319361A8795
:100AB0001AD61A231B6E1BB61BFD1B411C831CC3BD
:100AC0001C001D3C1D751DAB1DE01D121E421E6F3E
:100AD0001E9A1EC31EE91E0D1F2E1F4D1F691F8467
:100AE0001F9B1FB01FC31FD31FE11FEC1FF51FFB70
:100AF0001FFF1F002003010000116D00020101040F
:100B00006E01030202986E02000303F56E2532693E
:100B10002E25316956002533642563202530336442
:100B20006D00537461747573004552524F523A20F0
:100B300025326400253469202532693A253032692E
:100B4000002534696D25630025336920253369202C
:100B50002533692025336900253369202533692031
:100B6000253369202533690054656D7065726174A1
:100B700075726573202020200025634320202020EB
:100B800020002532692E2531695620202533692E13
:100B9000253169410025346957202536696D416842
:100BA000002532756D2F73205361743A256420003F
:100BB00020203344004E6F4678004447505300488D
:100BC0006F6D653A2533646D202533642563004ECF
:100BD0006F204E6176694374726C21000A0D77773D
:100BE000772E4D696B726F4B6F707465722E6465F2
:100BF0002028632920486953797374656D732047F1
:100C00006D6248000A0D74686520757365206F6613
:100C1000207468697320736F6674776172652069E8
:100C200073206F6E6C79207065726D697474656481
:100C3000200A0D6F6E206F726967696E616C204DBE
:100C4000696B726F4B6F707465722D486172647757
:100C5000617265004143542044534C004A657469F5
:100C600020736174656C6C6974005370656B747289
:100C7000756D20736174656C6C697420284C6F7796
:100C8000207265736F6C7574696F6E29005370659F
:100C90006B7472756D20736174656C6C6974202857
:100CA0003230343829005370656B7472756D20735F
:100CB0006174656C6C6974004D756C7469736967F7
:100CC0006E616C2050504D000A0D52656365697667
:100CD00065723A2000756E6B6E6F776E2E205573BD
:100CE000696E672050504D2E2E2E006E6F7420734B
:100CF0007570706F727465642062792068617264C7
:100D00007761726521000A0D3D3D3D3D3D3D3D3D14
:100D10003D3D3D3D3D3D3D3D3D3D3D3D3D3D3D3D03
:100D20003D3D3D3D3D3D3D3D3D3D3D000A0D466C5B
:100D300069676874436F6E74726F6C0A0D486172F4
:100D400064776172653A25642E25640A0D536F66D7
:100D500074776172653A5625642E256425632000F8
:100D60000A0D3D3D3D3D3D3D3D3D3D3D3D3D3D3D16
:100D70003D3D3D3D3D3D3D3D3D3D3D3D3D3D3D3DA3
:100D80003D3D3D3D3D0011241FBECFEFD0E4DEBF11
:100D9000CDBF11E0A0E0B1E0E0EEF6EF00E00BBF68
:100DA00002C007900D92A43FB107D9F718E0A4EF55
:100DB000B1E001C01D92A13AB107E1F77AEAE2E0A1
:100DC000F0E081E280935700D4907E010894E11C0A
:100DD000F11C20EF37EF41E050E087016FE0DA01CE
:100DE000C9012F5F3F4F4F4F5F4FABBFFC01879152
:100DF000F80181938F01615067FFF1CFF7016EE039
:100E0000819178277095615067FFFACF88897817AC
:100E100029F0F7E9DF1611F40000FECF0E94D30796
:100E20000C946F7B0C94000080910906E82FFF273B
:100E3000EE0FFF1FE05DF84F808191818D5E9F4F27
:100E400014F010920301808191818A5B9F4FCCF452
:100E5000809103018823A9F481E0809303018091AC
:100E600064048F5F80936404853038F088EE93E0EB
:100E7000909324028093230204C066E970E00E94EC
:100E80001F388091640499279093DE058093DD05D7
:100E900008951F93CF93DF93182F882389F082E062
:100EA00091E09F938F938BE392E19F938F93E091D7
:100EB0003004F091310409950F900F900F900F902E
:100EC00080912C06823308F044C084EF91E00E94A8
:100ED0006216EC01112329F0CE010E946B168823C3
:100EE000D9F3C2E0D0E026E530E080911D01909179
:100EF0001E018217930730F02196255D3F4FC730C2
:100F0000D10598F380912C069927C89F9001C99F1D
:100F1000300DD89F300D1124209300011123D9F0FA
:100F200068EC70E08C2F0E941F38DF93CF938AE02B
:100F300091E09F938F938BE392E19F938F93E09146
:100F40003004F091310409958DB79EB706968DBF98
:100F500002C080930001112311F1809100016AE029
:100F60000E94C27A892F99279F938F9380910001C5
:100F70000E94C27A99279F938F9385E191E09F9376
:100F80008F938BE392E19F938F93E0913004F091E4
:100F9000310409952DB73EB7285F3F4F2DBFDF9134
:100FA000CF911F910895CFEFD0E4DEBFCDBF88244D
:100FB000992414B815B807EE13E00253104017FF38
:100FC000FCCF85E18093020181E887B93E9A8FEFDB
:100FD00088B98BE184B981E085B98EE38AB987E469
:100FE0008BB9469A84B7877F84BF809160008861FF
:100FF000809360001092600084EC99E0909324024A
:101000008093230210921B0310921A03109235074B
:101010001092340710921D0310921C0310921F03AC
:1010200010921E0384EC94E0A0E0B0E08093950160
:1010300090939601A0939701B093980128980E94ED
:10104000CB160E949C160E9443120E9499340E9463
:10105000B01A0E9410300E94CE650E94E46F0E9478
:10106000F077809102018C3010F4299A01C0299800
:1010700078940E942A2F80916C02826080936C0287
:1010800010926E020E94D24384EF91E00E94621699
:101090008C0180916C0280FD05C0C8010E946B1616
:1010A0008823B9F38FE291E09F938F93BBE3AB2E3C
:1010B000B2E1BB2EBF92AF92E0913004F0913104C7
:1010C000099580EA9FE00E9462168C01C0E0D0E0A2
:1010D0000F900F900F900F90A2EDEA2EA6E0FA2E3F
:1010E000F6E8CF2EF6E0DF2E0E94D24380916C020C
:1010F00080FD05C0C8010E946B168823B9F3F60174
:1011000080811816ACF40BC00E94D24380916C020F
:1011100080FD05C0C8010E946B168823B9F3C80181
:101120000E946B16882321F4F7018081882364F7DD
:10113000F701808187FF18C02196DF93CF93219715
:1011400081E491E09F938F93BF92AF92E09130043E
:10115000F091310409958091F4018F5F8093F4013F
:101160008DB79EB706968DBF2196E4E0F0E0CE0ED7
:10117000DF1E88E090E0E80EF91ECC30D10508F4BF
:10118000B3CFC0E0D0E00FEC16E0E6E8EE2EE6E0EC
:10119000FE2EF801838187FD1CC0F701808118169F
:1011A000C4F42196DF93CF93219784E491E09F9339
:1011B0008F938BE392E19F938F93E0913004F091B2
:1011C0003104099582E0809321028DB79EB706967F
:1011D0008DBFF801838180788383219684E090E03D
:1011E000E80EF91E085F1F4FCC30D10590F282E661
:1011F00091E09F938F93CBE3D2E1DF93CF93E09184
:101200003004F09131040995909107068091F40122
:101210000F900F900F900F90981728F480914A0428
:10122000806180934A0488E891E09F938F93DF93D5
:10123000CF93E0913004F0913104099588EE93E06A
:101240000E9462168C010E94B61A0F900F900F90A8
:101250000F90C8010E946B168823D9F388EA91E0A9
:101260009F938F93DF93CF93E0913004F0913104FB
:10127000099580E00E94E138809102010F900F9063
:101280000F900F908A3011F0843110F0289801C02F
:10129000289A80ED97E0909324028093230285E5BD
:1012A000809366048EE090E00E94A22D9927182F6B
:1012B00000278FE090E00E94A22D080F111D1093CF
:1012C000FA010093F9018AE090E00E94A22D99278B
:1012D000182F00278BE090E00E94A22D080F111D0F
:1012E0001093F8010093F7010F5F1F4F39F08091C1
:1012F000F9019091FA018F5F9F4F41F41092FA012A
:101300001092F9011092F8011092F7018091F70103
:101310009091F8019F938F938091F9019091FA0138
:101320009F938F938DEA91E09F938F93DF93CF9359
:10133000E0913004F091310409958DB79EB708967D
:101340008DBF80ED91E09F938F93DF93CF93E091DA
:101350003004F09131040995809115060F900F909B
:101360000F900F90E0913004F091310482FF07C09C
:101370008CED91E09F938F93DF93CF9308C088EE1D
:1013800091E09F938F938BE392E19F938F930995C5
:101390000F900F900F900F900E94851F88E893E1A7
:1013A000909392018093910181E0809365040E9463
:1013B000490780912F060E9456778AEF91E09F930C
:1013C0008F93DF93CF93E0913004F091310409952E
:1013D00080ED97E00E9462168C018AEF90E00E94F7
:1013E0006216EC0183E08093B5050F900F900F908B
:1013F0000F90CE010E946B16882339F084E690E0AE
:101400000E946216EC010E94AC788091270288232A
:1014100009F4DFC180910F01882309F4DAC1109229
:10142000270280916404882319F00E94140702C0E7
:101430000E9477460E94D243209102012A3011F087
:10144000243110F0289801C0289A809120039091AF
:101450004A04882339F0809120038150809320032F
:10146000977F0AC080916F00806280936F00109216
:10147000310710923007986090934A04809191014F
:1014800090919201019790939201809391018091A4
:10149000910190919201892B29F080916D0288230E
:1014A00009F43EC08091910190919201892B01F540
:1014B0000E94363085E090E09093920180939101F4
:1014C0008091EF059091F00501969093F00580933F
:1014D000EF058091E80280688093E80280914A04D9
:1014E000816080934A048091B60582608093B6053E
:1014F00080910801909109018F5F9F4F19F58091AC
:1015000017038823F9F080E197E2909324028093F7
:10151000230280E890E0909309018093080112C0B3
:101520002A3011F0243110F0289801C0289A8091B7
:10153000230290912402892B29F48091E8028F776D
:101540008093E80280912702882309F042C10E941B
:1015500087120E94650EC8010E946B16882309F449
:1015600034C10C5E1F4F80916D0290914A04882314
:1015700039F0926090934A048091B60582600CC065
:101580009D7F90934A0480919101909192010797D9
:1015900028F08091B6058D7F8093B60580919101EA
:1015A00090919201079728F080914A048E7F809352
:1015B0004A0480910501882321F081508093050120
:1015C00025C0809370041092F8021092F7021092D6
:1015D000F6021092F5021092F4021092F30280913A
:1015E0000801909109018F5F9F4F81F48091200342
:1015F000882361F488E99AE390932402809323027C
:1016000080E09CE090930901809308018091EA01B9
:10161000893C70F081508093EA018091E8028F7BD1
:101620008093E80280914A048B7F80934A0435C0FE
:1016300080910E08882309F18091E80280648093EC
:10164000E80280914A04846080934A0480910801F2
:10165000909109018F5F9F4F81F480911703882338
:1016600061F088E99AE3909324028093230280E05A
:1016700098EA909309018093080110920204109255
:101680000104109200041092FF038FEF9FEF9093DC
:101690003C0880933B081092EA0180910001282FBA
:1016A000332780911D0190911E0182179307CCF47E
:1016B0008091E80280628093E80280910801909115
:1016C00009018F5F9F4FC1F480E797E19093240257
:1016D0008093230280E093E09093090180930801B6
:1016E0000BC08091230290912402892B29F48091D0
:1016F000E8028F7D8093E8020E94CC6984E08093A9
:10170000220280911703882329F45AEA852E55E096
:10171000952E12C08091FB018F5F8093FB01813376
:1017200059F41092FB018091F5019091F601019618
:101730009093F6018093F5010894811C911CF2E7C7
:101740008F16FBE09F0609F040C088249924209161
:10175000F9013091FA012F5F3F4F3093FA01209346
:10176000F9018091F7019091F80101969093F801A9
:101770008093F701832F9927682F8EE090E00E94D5
:10178000AA2D8091F9019091FA019070682F8FE055
:1017900090E00E94AA2D8091F7019091F801892F85
:1017A0009927682F8AE090E00E94AA2D8091F70186
:1017B0009091F8019070682F8BE090E00E94AA2D24
:1017C00084E190E00E9462168C010E941C6A0E94D3
:1017D000FB6F80912202882309F00BCE0E94EF65F7
:1017E00008CE1F920F920FB60F9211248F939F93E2
:1017F000EF93FF93809107018823E1F48091150214
:101800009091160201969093160280931502FC01A6
:10181000EB5EFA4FE081ED3019F0803A910539F432
:10182000109216021092150281E080930701E09356
:10183000C60004C01092160210921502FF91EF919B
:101840009F918F910F900FBE0F901F9018951F9230
:101850000F920FB60F9211242F933F934F935F93E4
:101860006F937F938F939F93AF93BF93CF93EF9398
:10187000FF9390E08091C60080930D0250911B026F
:10188000503A10F090931C0280910D028D3009F0B7
:1018900065C080911C02823009F060C090931C02E8
:1018A000852F99278D589B4FFC01329740812091BD
:1018B000170230911802241B3109DC0111978C9119
:1018C000281B3109C9019F70909318028093170259
:1018D00046E0969587954A95E1F7982F935C90930B
:1018E00019022F733070235C20931A02808198179D
:1018F00029F48C91281711F491E006C090E08091B2
:101900000A028F5F80930A02C0910C02CC2309F077
:1019100074C0992309F471C081E080930C02580FC0
:10192000509309025150E52FFF27ED58FB4F8DE0F2
:10193000808380917504823509F05FC00E94851F05
:1019400088E190E02CE00FB6F894A89580936000B1
:101950000FBE20936000C09321024FC020911C0253
:10196000822F992781309105F9F0823091051CF47E
:10197000892B21F040C0029711F13DC080910D02EA
:10198000833239F480910C02882319F481E080932A
:101990001C0280910D028093730481E080931B02EE
:1019A00080910D02992722C02F5F20931C02E52F02
:1019B000FF27ED58FB4F80910D02808309C0E52F72
:1019C000FF27ED58FB4F80910D028083503A20F4A1
:1019D0005F5F50931B0202C010921C0220910D0207
:1019E0008091170290911802820F911D9093180216
:1019F0008093170202C010921C02FF91EF91CF91C9
:101A0000BF91AF919F918F917F916F915F914F9116
:101A10003F912F910F900FBE0F901F901895AC0122
:101A2000A0E0B0E09D01A817B90748F4E5E1F5E0B2
:101A30008191280F311D1196A417B507C8F33F7087
:101A4000FD01EB5EFA4FC90156E0969587955A95D0
:101A5000E1F7835C80831196FD01EB5EFA4F2F73F3
:101A60003070822F835C8083AA5EBA4F8DE08C93A6
:101A700010920701809115058093C6000895A0E09B
:101A8000B0E0E5E4FDE00C943B7B2C859D850E8564
:101A9000BB2483E2809315059F59909316052093EC
:101AA000170533E0E32EF12C002309F49EC0CF8408
:101AB000D888BE016D5E7F4FA989BA890150109701
:101AC00009F493C01097B9F0F601EB0DF11DB39432
:101AD0009081119791F4002349F1FB016E5F7F4FD4
:101AE000DB01C080D1806E5F7F4F0D90BC91A02D37
:101AF000BB24015002C090E019C01097B9F0F60164
:101B0000EB0DF11DB3944081119791F4002341F145
:101B1000FB016E5F7F4FDB01C080D1806E5F7F4F26
:101B20000D90BC91A02DBB24015002C040E018C014
:101B30001097B1F0F601EB0DF11DB39410811197E0
:101B400081F4002371F0FB013296DB01CD90DC9033
:101B5000BF016E5F7F4FA081B181BB24015001C0E6
:101B600010E0F701EB5EFA4F892F86958695835C2E
:101B700080830894E11CF11CF701EB5EFA4F892F7A
:101B800099278370907024E0880F991F2A95E1F7B8
:101B900055279A0194E0369527959A95E1F7822B7F
:101BA000835C80830894E11CF11CF701EB5EFA4F23
:101BB0004F705070440F551F440F551F812F9927A8
:101BC00026E0969587952A95E1F7842B835C8083A0
:101BD0000894E11CF11CF701EB5EFA4F1F73135CD4
:101BE00010830894E11CF11C6ACFC7010E940F0DFD
:101BF000E9E00C94577BA3E07A2F4091090246500C
:101C0000442309F458C0E72FFF27ED58FB4F80818C
:101C10008D537F5FE72FFF27ED58FB4F20812D531A
:101C20007F5FE72FFF27ED58FB4F30813D537F5FEC
:101C3000E72FFF27ED58FB4F60816D537F5F99279A
:101C4000880F991F880F991F522F52955F70582B3C
:101C5000822F99278F709070F4E0880F991FFA9562
:101C6000E1F7232F26952695282B832F992783701C
:101C70009070E6E0880F991FEA95E1F7682B4150D4
:101C80004F3FC9F0EA2FFF27ED58FB4F5083AF5F5E
:101C900041504F3F81F0EA2FFF27ED58FB4F208343
:101CA000AF5F41504F3F39F0EA2FFF27ED58FB4F10
:101CB0006083AF5FA5CF86E794E09093080280939E
:101CC0000702A350A09306020895A2E0B0E0EBE65D
:101CD000FEE00C94417B80910C02882309F4C7C379
:101CE0000E94FB0D80917404823609F081C28091BC
:101CF000750499278137910509F4C0C08237910591
:101D0000C4F48D36910509F482C08E36910544F4F1
:101D10008B34910531F18636910509F454C168C2BE
:101D20008E36910509F45BC08037910509F49FC098
:101D30005FC28537910509F4E2C18637910544F405
:101D40008337910509F4DCC08437910539F150C21D
:101D50008737910509F410C28937910509F46AC1E2
:101D600047C2E0910702F09108028081918190932F
:101D70003303809332032091300330913103821B6F
:101D8000930B845E9D4F68E671E00E94E27A845B6B
:101D9000904090932F0380932E032AC280910902D2
:101DA000A0910702B0910802853140F080E1EEE495
:101DB000F4E00D9001928A95E1F70DC08D919D910F
:101DC0000D90BC91A02D80934E0490934F04A0934E
:101DD0005004B093510480EF809304024BC0809173
:101DE00007018823E1F38DE490E09F938F9389E7C7
:101DF00096E09F938F9381E08F938F938EE48F93E0
:101E00000E943F0D8DB79EB707968DBFF1C1A0917F
:101E10000702B09108021C91113081F48DE4E9E7CA
:101E2000F6E00D9001928A95E1F70E94AA2E19839F
:101E300080914A048F7E80934A0401C01982809168
:101E400007018823E1F381E090E09F938F93CE0117
:101E500001969F938F9381E08F938F938DE48F935F
:101E60000E943F0DADB7BEB71796ADBFC1C181E0AF
:101E700080930F028FEF80930501BAC1E0910702B2
:101E8000F091080280818F3F39F40E940D2FE0917C
:101E90000702F09108028083E0910702F0910802A6
:101EA0008081882311F481E003C0863010F085E042
:101EB0008083E0910702F091080280810E94C02D8A
:101EC000E0910702F09108028081898380910701E7
:101ED0008823E1F380E790E09F938F9388E096E07A
:101EE0009F938F9381E090E09F938F93CE01019613
:101EF0009F938F9382E08F9381E08F9381E571C1EF
:101F00002091070230910802D9018C9181508530CF
:101F100008F040C0F90181818435E1F52F5F3F4F22
:101F200080E7E8E0F6E0D9010D9001928A95E1F7AB
:101F3000F90182910E94292E809147069927AA27AC
:101F4000BB27BC01CD0124EC39E040E050E00E9409
:101F5000A37ADC01CB018093B7019093B801A093E1
:101F6000B901B093BA01809148069927AA27BB27E7
:101F7000BC01CD010E94A37ADC01CB018093B301A7
:101F80009093B401A093B501B093B6010E940D2FB8
:101F9000898301C01982809107018823E1F381E0E0
:101FA00090E09F938F93CE0101969F938F9381E052
:101FB0008F938F9383E58F930E943F0D8DB79EB7CC
:101FC00007968DBF26C0E0910702F0910802E081DC
:101FD0008E2F8150853018F48E2F0E94C02D0E94C4
:101FE0000D2F8983809107018823E1F381E090E040
:101FF0009F938F93CE0101969F938F9381E08F9350
:102000008F9386E48F930E943F0DADB7BEB71796AE
:10201000ADBF80911703882329F46EE670E08981B3
:102020000E941F3880E00E94490780912F060E947D
:102030005677DEC0E0910702F0910802808199276F
:1020400087FD909590934B0780934A07818199274C
:1020500087FD909590934D0780934C078281992737
:1020600087FD909590934F0780934E078381992722
:1020700087FD90959093510780935007848199270D
:1020800087FD9095909353078093520785819927F8
:1020900087FD9095909355078093540786819927E3
:1020A00087FD9095909357078093560787819927CE
:1020B00087FD9095909359078093580780859927BD
:1020C00087FD909590935B0780935A0781859927A8
:1020D00087FD909590935D0780935C078285992793
:1020E00087FD909590935F0780935E07838599277E
:1020F00087FD9095909361078093600779C0E09188
:102100000702F091080280810E94F2338A838823BB
:1021100019F481E0898301C0198280910701882325
:10212000E1F388E090E09F938F9387EC96E09F9394
:102130008F9321E030E03F932F938091070290919D
:1021400008029F938F933F932F93CE0102969F9304
:102150008F933F932F93CE01820F931F9F938F9363
:1021600084E08F9381E08F9385E58F930E943F0DEC
:10217000EDB7FEB773963BC0809106028930C0F17F
:1021800020910702309108022F5F3F4F88E0A7ECB3
:10219000B6E0F90101900D928A95E1F7D9018E918F
:1021A0000E9448338A83882319F481E0898301C01F
:1021B0001982809107018823E1F321E030E03F9309
:1021C0002F93CE0102969F938F933F932F93CE012F
:1021D000820F931F9F938F9382E08F9381E08F9361
:1021E00087E58F930E943F0DEDB7FEB73B96EDBF9D
:1021F0008091750499278436910509F4CDC0853600
:102200009105ACF48136910509F481C082369105BF
:102210002CF48B34910509F45DC021C182369105FF
:1022200009F482C08336910509F491C018C18C3637
:10223000910509F4FFC08D3691054CF48736910560
:1022400009F40AC18836910509F4C4C008C184376D
:10225000910529F08637910509F4FAC000C18091F3
:102260000902A0910702B0910802803140F080E19C
:10227000EEE4F4E00D9001928A95E1F70DC08D91A6
:102280009D910D90BC91A02D80934E0490934F048E
:10229000A0935004B0935104809107018823E1F387
:1022A0001F92809104018F9384E58F930E943F0DCC
:1022B0008AEF809304028FEF8093050180EA9FE00C
:1022C0000E9462169093FD018093FC010F900F9085
:1022D0000F90C5C0E0910702F091080280819181C2
:1022E0009093330380933203209130033091310374
:1022F000821B930B845E9D4F68E671E00E94E27A38
:10230000845B904090932F0380932E03A8C0E091AC
:102310000702F0910802808180930601803298F0D4
:102320008FE1809306010FC0A0910702B0910802CF
:102330008BE0E6E6F4E00D9001928A95E1F780915A
:102340006F048093F7058FEF8093050188C080911B
:10235000000290910102892B89F4E0910702F0912B
:102360000802E081EE2351F08AE0E89FC0011124C9
:102370000E9462169093410480934004E09107020A
:10238000F091080290818AE0989FC00111249093F7
:1023900001028093000215C08FEF80930501E09148
:1023A0000702F091080290818AE0989FC0011124F1
:1023B0009093030280930202892B19F081E08093AD
:1023C000110280EA9FE00E9462169093FD018093C3
:1023D000FC0145C08FEF80930501E0910702F09169
:1023E0000802908197FD08C082E080930E0210924F
:1023F000FF011092FE011AC0909580916502892B11
:102400008093650291818AE0989FC0011124909386
:10241000FF018093FE0184E080930E0280EA9FE03A
:102420000E9462169093FD018093FC0181E08093ED
:10243000120215C08FEF80930501E0910702F09121
:10244000080280818093660281E08093130207C0B6
:1024500081E08093100203C081E080931402109207
:102460000C02109208021092070210920602E3E09A
:10247000CE5F0C945D7B982F8091C00085FFFCCFD0
:102480009093C60008950F931F9388E18093C10035
:102490008091C00082608093C0008091C1008068FC
:1024A0008093C1008091C10080648093C10000E0EE
:1024B00010E00093C5008AE290E08093C400809110
:1024C0000202909103020E9462169093430480934B
:1024D00042048CED90E00E94621690937204809307
:1024E00071041092440480E58093450485E0809354
:1024F00048048BE08093460410924704109308022E
:1025000000930702109206021F910F910895A0E117
:10251000B0E0EDE8F2E10C943E7B80910701882366
:1025200009F4C1C28091FC019091FD010E946B16DB
:10253000882361F01092FF011092FE0110920302B5
:102540001092020210920102109200028091FE018C
:102550009091FF01892B41F0809113059091140512
:102560000E946B16882329F480911202882309F4B3
:1025700060C080910701882309F45BC080910E023E
:1025800000E211E08430A8F00E94991F80E590E0FD
:102590009F938F931F930F9381E08F938F9388E482
:1025A0008F930E943F0D2DB73EB7295F3F4F2DBF40
:1025B00034C01092670282E294E09F938F938EE87A
:1025C0009FE19F938F93E0913004F091310409953E
:1025D00084E190E09F938F931F930F9381E090E0AD
:1025E0009F938F938EE092E09F938F9382E08F93DF
:1025F00081E08F9388E48F930E943F0D80910E02BB
:10260000982F8F5F80930E022DB73EB7215F3F4F0B
:102610002DBF943010F010920E028091FE01909127
:10262000FF010E9462169093140580931305109287
:10263000120280911302882351F1809107018823AF
:1026400031F10E94991F80E590E09F938F9380E283
:1026500091E09F938F9321E030E03F932F938FE1A0
:1026600091E09F938F933F932F9386E692E09F9301
:102670008F9383E08F9381E08F938CE48F930E94FC
:102680003F0D109213028DB79EB70F968DBF8091AC
:1026900010028823D1F0809107018823B1F08AE0ED
:1026A00090E09F938F9384E494E09F938F9381E0D5
:1026B0008F938F9386E58F930E943F0D10921002A7
:1026C0002DB73EB7295F3F4F2DBF8091140288235D
:1026D000D9F0809107018823B9F08BE090E09F93B7
:1026E0008F9386E694E09F938F9381E08F93809100
:1026F00004018F9387E48F930E943F0D1092140280
:102700008DB79EB707968DBF80917104909172042A
:102710000E946B16882309F461C080910701882309
:1027200009F45CC0809124069927880F991F880FAF
:10273000991F7C010027F7FC0095102F80917003F2
:1027400090917103A0917203B0917303BC01CD010C
:10275000A80197010E94177B30935F0420935E04C9
:102760008091680390916903A0916A03B0916B0313
:10277000BC01CD01A80197010E94177B3093610431
:102780002093600480910103809362048091000390
:102790008093630488E090E09F938F938EE594E0AC
:1027A0009F938F9381E08F9383E08F938BE68F933A
:1027B0000E943F0D809164042DB73EB7295F3F4FC3
:1027C0002DBF853018F086E08093640483E690E0A6
:1027D0000E946216909372048093710480910202A9
:1027E00090910302892B41F080914204909143041F
:1027F0000E946B16882321F480911102882339F1FD
:1028000080910701882319F10E94153782E490E036
:102810009F938F9385EB95E09F938F9381E08F93A8
:102820008F9384E48F930E943F0D109211028DB715
:102830009EB707968DBF8091020290910302009788
:1028400031F00E9462169093430480934204809179
:10285000000290910102892B09F4B8C080914004D4
:10286000909141040E946B16882309F4AFC08091B7
:102870000701882309F4AAC0809124069927880FAC
:10288000991F880F991F7C010027F7FC0095102FD6
:102890008091700390917103A0917203B0917303C2
:1028A000BC01CD01A80197010E94177B309333042E
:1028B000209332048091680390916903A0916A0388
:1028C000B0916B03BC01CD01A80197010E94177B59
:1028D00030933504209334042091F6073091F707A4
:1028E0004091F8075091F907DA01C90163E0880FB8
:1028F000991FAA1FBB1F6A95D1F7820F931FA41FB0
:10290000B51F820F931FA41FB51F20919501309111
:1029100096014091970150919801BC01CD010E9410
:10292000177B309337042093360480913C039091B9
:102930003D03A0913E03B0913F0339E0B595A795C3
:10294000979587953A95D1F780933804809138030D
:1029500090913903A0913A03B0913B0329E0B595DA
:10296000A795979587952A95D1F7809339048091FB
:10297000400390914103A0914203B091430309E0C9
:10298000B595A795979587950A95D1F780933A04C1
:102990008EE090E09F938F9382E394E09F938F93D8
:1029A00081E08F938F9383E48F930E943F0D8091FA
:1029B0000002909101020E9462169093410480935C
:1029C00040042DB73EB7295F3F4F2DBF80910601D0
:1029D0008F3F71F1992714E0880F991F1A95E1F73D
:1029E0008E5D9D4F40E150E0BC01CE0101960E94FA
:1029F000F67880E190E09F938F93CE0101969F93AC
:102A00008F9381E090E09F938F9386E091E09F9376
:102A10008F9382E08F9381E08F9381E48F930E9464
:102A20003F0D8FEF809306018DB79EB70B968DBF3C
:102A30008091F7058823D1F0809107018823B1F0B8
:102A400081E090E09F938F9387EF95E09F938F9322
:102A500081E08F938F9382E48F930E943F0D1092B9
:102A6000F7052DB73EB7295F3F4F2DBF80910F026D
:102A70008823C9F0809107018823A9F084E390E0BE
:102A80009F938F9380E397E09F938F9381E08F9341
:102A90008F9380E58F930E943F0D10920F028DB7A8
:102AA0009EB707968DBFE6E0C05F0C945A7B1F92DD
:102AB0000F920FB60F9211242F933F935F936F9352
:102AC0007F938F939F93AF93BF93EF93FF9320E0F8
:102AD00080912202882329F08091220281508093E4
:102AE000220280911304882319F0815080931304EB
:102AF00080912A02815080932A028F3F09F05BC0A7
:102B000089E080932A0280912802909129020196FF
:102B1000909329028093280280910A018F5F81702F
:102B200080930A01882319F481E080932702349965
:102B300003C081E080932B028091230290912402B4
:102B4000892B21F180912302909124020B9750F060
:102B500080912302909124020A97909324028093FB
:102B6000230204C0109224021092230280912302B7
:102B7000909124022091080130910901822393232E
:102B8000892B11F021E008C020E006C08FEF9FEFF5
:102B9000909309018093080180910201222331F072
:102BA0008A3011F45A9A07C0479A05C08A3011F446
:102BB0005A9801C0479880912B02882309F472C06B
:102BC0002091EA01222309F06DC08091150683FF50
:102BD00069C086B19927FC01E071F07084FF14C0D0
:102BE000809125029091260201969093260280936F
:102BF00025028091250290912602895E934008F477
:102C000051C020932B024EC0809125029091260244
:102C1000892B09F443C080912502909126028A569F
:102C20009140E0F5809125029091260269E270E0E2
:102C30000E94CE7A8091250290912602860F971FDE
:102C4000909326028093250280912502909126027E
:102C50000B9750F080912502909126020A9790934D
:102C600033038093320304C0F0933303E0933203C1
:102C700080913203909133032091300330913103DE
:102C8000821B930B845E9D4F68E671E00E94E27A9E
:102C9000845B904090932F0380932E031092260222
:102CA00010922502FF91EF91BF91AF919F918F916B
:102CB0007F916F915F913F912F910F900FBE0F9079
:102CC0001F9018952091280230912902280F391F52
:102CD000C901019608952091280230912902821B92
:102CE000930B892F99278695807490700895CF93C0
:102CF000DF930E946216EC01CE010E946B168823BE
:102D0000D9F3DF91CF910895CF93DF930E9462169C
:102D1000EC0109C080910F01882329F090930F01E5
:102D20008FEC80937A00CE010E946B16982F882337
:102D300089F3DF91CF9108959FB7F8945F983E9AF9
:102D4000469A8091B0008F708093B0008091B0005F
:102D500083608093B0008091B1008B738093B10049
:102D60008091B1008B608093B1001092B2008FEF20
:102D70008093B3008091B00080688093B000809110
:102D800070008A7F809370008091700082608093D1
:102D900070009FBF08958AE090E00E9462169093B1
:102DA00033028093320282E085BD83EA84BD17BC82
:102DB00084EB88BD86E086BD80916E008160809343
:102DC0006E0008951F920F920FB60F9211242F9349
:102DD0003F934F935F936F937F938F939F93AF93A3
:102DE000BF93CF93DF93EF93FF9380910201909174
:102DF0002C02843108F011C1992309F06AC3809133
:102E0000B00086FFECC08091B0008F7B8093B00053
:102E100089EA93E090932E0280932D0280910B011A
:102E200090910C019C01220F331F280F391F8091B4
:102E3000A1019927880F991F880F991F280F391F03
:102E400037FF02C02D5F3F4FC90195958795959536
:102E5000879590930C0180930B01909320028093AF
:102E60001F0280916A0660913606209170033091AE
:102E70007103409172035091730380FF2CC0772738
:102E800088279927EA01D90157FF04C0A158BF4FED
:102E9000CF4FDF4FE7E0D595C795B795A795EA9552
:102EA000D1F79D01AE010E94A37A9B01AC0197FF6F
:102EB00004C0215C3F4F4F4F5F4F66E055954795EB
:102EC000379527956A95D1F780911F02909120023E
:102ED000820F931F2BC0772788279927EA01D901F2
:102EE00057FF04C0A158BF4FCF4FDF4F27E0D59504
:102EF000C795B795A7952A95D1F79D01AE010E9478
:102F0000A37A9B01AC0197FF04C0215C3F4F4F4F58
:102F10005F4FF6E05595479537952795FA95D1F788
:102F200080911F0290912002821B930B90932002AC
:102F300080931F0280913706282F3327220F331FDB
:102F4000220F331F80911F02909120028217930756
:102F50007CF080913806282F3327220F331F220F51
:102F6000331F80911F02909120022817390724F403
:102F70003093200220931F0220912D0230912E02C7
:102F800080911F0290912002280F391F205032405B
:102F900030932E0220932D0280911F0290912002E7
:102FA00097FD039695958795959587959093200223
:102FB00080931F0245E02D3D340718F08CED95E01D
:102FC00005C02757314030F487E791E090932E02F7
:102FD00080932D0280912D0290912E0243C2809108
:102FE000B00080648093B00080913D06282F332785
:102FF0008DED96E0289FA001299F500D389F500D20
:103000001124CA0120912F0230913002821B930BB0
:1030100090932E0280932D0259C2992309F059C230
:103020008091B00086FF23C28091B0008F7B809397
:10303000B000E0913102EE23F1F480913D06282F9B
:1030400033278DED96E0289FA001299F500D389FD2
:10305000500D1124CA0120912F0230913002821BA1
:10306000930B90932E0280932D02109230021092B7
:103070002F02469A2BC289EA93E090932E02809306
:103080002D028E2F99278330910509F4A4C1843035
:1030900091053CF48130910561F0029709F4D2C0AA
:1030A000AAC18430910509F499C1059709F4A0C11A
:1030B000A2C180910B0190910C019C01220F331F42
:1030C000280F391F8091A1019927880F991F880F18
:1030D000991F280F391F37FF02C02D5F3F4FC901CD
:1030E000959587959595879590930C0180930B0105
:1030F0009093200280931F0280916A0660913606A9
:1031000020917003309171034091720350917303C9
:1031100080FF2CC0772788279927EA01D90157FF1C
:1031200004C0A158BF4FCF4FDF4F27E0D595C795BB
:10313000B795A7952A95D1F79D01AE010E94A37A74
:103140009B01AC0197FF04C0215C3F4F4F4F5F4F85
:10315000A6E05595479537952795AA95D1F7809183
:103160001F0290912002820F931F27C07727882784
:10317000992757FF04C021583F4F4F4F5F4FF7E04B
:103180005595479537952795FA95D1F70E94A37ADB
:103190009B01AC0197FF04C0215C3F4F4F4F5F4F35
:1031A000E6E05595479537952795EA95D1F78091B3
:1031B0001F0290912002821B930B90932002809318
:1031C0001F0280913706282F3327220F331F220F2B
:1031D000331F80911F0290912002821793077CF089
:1031E00080913806282F3327220F331F220F331FD9
:1031F00080911F02909120022817390724F4309300
:10320000200220931F0280912D0290912E02209186
:103210001F0230912002820F931F805092409093A2
:103220002E0280932D0280911F029091200297FD23
:103230000396959587959595879590932002809311
:103240001F02ECC080910D0190910E019C01220F94
:10325000331F280F391F8091A0019927880F991FCC
:10326000880F991F280F391F37FF02C02D5F3F4F6E
:10327000C901959587959595879590930E018093B3
:103280000D0190931E0280931D0280916A06609149
:103290003A06A0916803B0916903C0916A03D09186
:1032A0006B0381FF2AC07727882799279D01AE01EC
:1032B000D7FF04C021583F4F4F4F5F4FA7E05595B0
:1032C000479537952795AA95D1F70E94A37A9B0138
:1032D000AC0197FF04C0215C3F4F4F4F5F4FF6E0BA
:1032E0005595479537952795FA95D1F780911D0209
:1032F00090911E02820F931F29C077278827992754
:103300009D01AE01D7FF04C021583F4F4F4F5F4F83
:10331000E7E05595479537952795EA95D1F70E94AF
:10332000A37A9B01AC0197FF04C0215C3F4F4F4F34
:103330005F4F76E055954795379527957A95D1F764
:1033400080911D0290911E02821B930B90931E028E
:1033500080931D0280913B06282F3327220F331FB5
:10336000220F331F80911D0290911E028217930736
:103370007CF080913C06282F3327220F331F220F29
:10338000331F80911D0290911E022817390724F4E3
:1033900030931E0220931D0280912D0290912E02E7
:1033A00020911D0230911E02820F931F8050924087
:1033B00090932E0280932D0280911D0290911E0207
:1033C00097FD0396959587959595879590931E0201
:1033D00080931D0223C08091C40702C080919E0784
:1033E0009927880F991F880F991F87559E4F12C0E4
:1033F0008091CC07F5CFFF27EE0FFF1FE05DF84F60
:1034000020813181220F331F80912D0290912E0255
:10341000820F931F90932E0280932D0280912D0294
:1034200090912E0255E08D3D950718F08CED95E0BA
:1034300005C08757914030F487E791E090932E02C2
:1034400080932D0220912D0230912E022C5B304072
:1034500030932E0220932D0280912F029091300202
:10346000820F931F9093300280932F022FC0809180
:10347000B00080648093B0008CEB90E090932E02BB
:1034800080932D0280912F029091300284549F4F9F
:103490009093300280932F0280912102882321F0A3
:1034A00080912003853B20F480912102823011F429
:1034B000469801C0469A809131028F5F8093310215
:1034C00090913D06981710F41092310281E080939C
:1034D0002C0220912D0230912E0241E02F3734072B
:1034E00030F08FEF8093B3002F5F30400FC02F3F3D
:1034F0003105C9F0C0F0A9014F5F50404F37510569
:1035000050F480E88093B3002058304030932E026E
:1035100020932D0212C08FEF8093B30050932E02A0
:1035200040932D020AC080912D028093B300109227
:103530002E0210922D0210922C02FF91EF91DF913A
:10354000CF91BF91AF919F918F917F916F915F913B
:103550004F913F912F910F900FBE0F901F90189594
:1035600010927C008FEC80937A000895CF93DF93C4
:1035700083E090E00E94A22DC82FDD27C531D10540
:1035800008F02A97C7BD1092380284E690E00E94A6
:10359000841680911301909114018052934010F48D
:1035A000C0E0D0E0CA3FD105F8F4C7BD82E390E0A7
:1035B0000E94841687E394E09F938F938BE392E1BC
:1035C0009F938F93E0913004F0913104099580919D
:1035D0001301909114010F900F900F900F90805253
:1035E000934010F02196DECF6C2F83E090E00E9494
:1035F000AA2DC09304068091150680FF09C08C2F68
:103600008A508B3E28F0809149048064809349045D
:10361000C7BD8CE291E00E948416DF91CF9108959E
:10362000EF92FF921F93CF9310E080ED97E00E94FE
:1036300062167C01CCE8133019F4CB3008F0C9E0F5
:1036400010E080914802909149028C5F934024F4ED
:103650008091120181500AC08091480290914902E4
:103660008750944034F0809112018F5F8093120153
:1036700001C011E080914602909147028C5F934017
:1036800024F48091110181500AC0809146029091EA
:1036900047028750944034F0809111018F5F8093EE
:1036A000110101C01F5F80914402909145028C5F1F
:1036B000934024F48091100181500AC0809144020B
:1036C0009091450287509440C4F0809110018F5F23
:1036D0008093100113C089E394E09F938F938BE351
:1036E00092E19F938F93E0913004F091310409951A
:1036F0000F900F900F900F905FC01F5F82E180933B
:10370000710280916C028E7F80936C0285EA8093B7
:10371000BC00809112018A3040F48091490481609C
:10372000809349048AE08093120180911201863FC0
:1037300040F08091490481608093490485EF809333
:103740001201809111018A3040F480914904826015
:10375000809349048AE08093110180911101863F92
:1037600040F08091490482608093490485EF809302
:103770001101809110018A3040F4809149048460E5
:10378000809349048AE08093100180911001863F64
:1037900040F08091490484608093490485EF8093D0
:1037A000100180917102882339F0C7010E946B16C5
:1037B000882309F090CFF5CF10920F018FEC809302
:1037C0007A0080910F018823E1F3CA3020F48AE067
:1037D00090E00E948416C15009F02DCF86E490E05D
:1037E0000E948416CF911F91FF90EF9008951F9231
:1037F0000F920FB60F921124AF92BF92CF92DF9229
:10380000EF92FF920F931F932F933F934F935F93EA
:103810006F937F938F939F93AF93BF93EF93FF9398
:1038200080915102282F3327442755278F5F80939B
:103830005102F9012231310508F03EC3EA5BFF4F26
:103840000C94697B809178009091790046C08091BA
:10385000780090917900DEC0809178009091790095
:10386000909353028093520209C180917903909101
:103870007A032091780030917900821B930B90930A
:10388000F9058093F8058091F8059091F9059093DA
:103890005D0280935C0210C1809178009091790064
:1038A00020917B0330917C03821B930B9093030642
:1038B00080930206809102069091030690935F0226
:1038C00080935E02FBC28091560290915702209134
:1038D000780030917900820F931F90935702809364
:1038E000560281E0ECC280915402909155022091E1
:1038F000780030917900820F931F90935502809346
:10390000540284E0DCC280911D0190911E019C0153
:10391000220F331F280F391F809178009091790072
:1039200063E070E00E94CE7A260F371F3695279508
:103930003695279530931E0120931D0185E0BFC267
:1039400080917800909179002091750330917603F1
:10395000821B930B90933F0280933E0281E0809301
:103960003D0280917800909179009093FB058093BF
:10397000FA0580913E0290913F029C01442737FD59
:103980004095542F8091340390913503A0913603D4
:10399000B0913703820F931FA41FB51F8093340388
:1039A00090933503A0933603B093370320913403EB
:1039B00030913503409136035091370357FF04C0CF
:1039C00021503C4F4F4F5F4F0AE055954795379533
:1039D00027950A95D1F78091340390913503A091F2
:1039E0003603B0913703821B930BA40BB50B809366
:1039F000340390933503A0933603B09337032EC15D
:103A00008091540290915502209178003091790074
:103A1000820F931F9093550280935402109250028C
:103A200050C2809102018A3071F4809178009091A7
:103A300079002091520230915302820F931F019618
:103A40009695879517C04091520250915302843148
:103A500058F02091780030917900240F351F8FEFB6
:103A600097E0821B930B06C08091780090917900BB
:103A7000840F951F909345028093440286E01FC2F5
:103A80008091790390917A032091780030917900A8
:103A9000821B930B9093F9058093F8058091F805AC
:103AA0009091F90520915C0230915D02820F931F85
:103AB000909343028093420287E001C28091780094
:103AC0009091790020917B0330917C03821B930BB2
:103AD000909303068093020680910206909103065C
:103AE00020915E0230915F02820F931F90934102FA
:103AF00080934002E3C12091560230915702809199
:103B0000780090917900280F391F30935702209345
:103B10005602809102018A3019F4220F331F04C02B
:103B2000220F331F220F331F309357022093560268
:103B30002091560230915702C90137FD0796A3E044
:103B400095958795AA95E1F790934902809348024D
:103B50008091580290915902820F931F97FD019610
:103B600095958795909359028093580220918503EB
:103B700030918603821B930B90931C0180931B0151
:103B800020914E0230914F0280911B0190911C01B7
:103B9000280F391F37FF02C02F5F3F4F35952795FC
:103BA00030934F0220934E029CCE209154023091CC
:103BB00055028091780090917900280F391F309339
:103BC000550220935402809102018A3019F4220F89
:103BD000331F04C0220F331F220F331F30935502AF
:103BE000209354022091540230915502C90137FDAF
:103BF000079663E0959587956A95E1F7909347025C
:103C00008093460280915A0290915B02820F931F2B
:103C100097FD01969595879590935B0280935A0244
:103C20002091830330918403821B930B90931A019C
:103C30008093190120914C0230914D02809119011D
:103C400090911A01280F391F37FF02C02F5F3F4F95
:103C50003595279530934D0220934C0283E02FC178
:103C60001092510281E080930F0180913402909173
:103C7000350201969093350280933402809178004A
:103C80009091790090931401809313018091130116
:103C900090911401AA27BB27A0906002B090610206
:103CA000C0906202D0906302A80EB91ECA1EDB1E2D
:103CB000A0926002B0926102C0926202D09263024E
:103CC000809164028F5F80936402823108F4F6C0B1
:103CD0008091150190911601A0911701B0911801E2
:103CE0007C018D0123E0EE0CFF1C001F111F2A95A3
:103CF000D1F7E81AF90A0A0B1B0BEA0CFB1C0C1D86
:103D00001D1D80913802992787FD9095A92FB92F05
:103D1000BC01CD0126EC34E240E050E00E94A37AE1
:103D2000DC01CB01E81AF90A0A0B1B0BD801C70109
:103D30000496A11DB11DB7FF05C0D801C7010B96A0
:103D4000A11DB11D13E0B595A795979587951A9577
:103D5000D1F78093150190931601A0931701B093AA
:103D600018018091FC059091FD057C010027F7FC6E
:103D70000095102F8091150190911601A0911701C7
:103D8000B0911801E81AF90A0A0B1B0BE092120312
:103D9000F09213030093140310931503209139023A
:103DA00030913A0240913B0250913C0257FF04C0CF
:103DB000215F3F4F4F4F5F4FF4E055954795379543
:103DC0002795FA95D1F78091390290913A02A09106
:103DD0003B02B0913C02821B930BA40BB50B80936A
:103DE000390290933A02A0933B02B0933C02809137
:103DF000390290913A02A0913B02B0913C028E0DA3
:103E00009F1DA01FB11F8093390290933A02A09387
:103E10003B02B0933C028091360290913702AC0194
:103E2000E5E0440F551FEA95E1F7481B590B8091D7
:103E3000390290913A02A0913B02B0913C02B7FF47
:103E400003C00F96A11DB11D74E0B595A795979578
:103E500087957A95D1F72091120330911303281B8F
:103E6000390B63E0220F331F6A95E1F7240F351FEA
:103E700037FF02C0215E3F4F45E0359527954A95B3
:103E8000E1F73093370220933602D601C501D7FE01
:103E900003C00196A11DB11DB595A795979587956E
:103EA0008093600290936102A0936202B0936302D8
:103EB00089E08093640202C01092510282E08093F4
:103EC00050028091500280937C008091510288239F
:103ED00019F08FEC80937A00FF91EF91BF91AF9131
:103EE0009F918F917F916F915F914F913F912F9112
:103EF0001F910F91FF90EF90DF90CF90BF90AF9008
:103F00000F900FBE0F901F90189590E2E0E2F1E045
:103F10008FE49193815087FFFCCF089590916702C1
:103F2000E0E2F1E0E90FF11D80839F5F909367026B
:103F30000895EF92FF920F931F93CF93DF932091F9
:103F4000650220FF0AC080916602882311F081502B
:103F500002C080911F018093660221FF0CC09091E6
:103F6000660280911F01981719F41092660203C02F
:103F70009F5F90936602822F992780FF04C081FF84
:103F800002C0109266020E94851F80916602282F4F
:103F90003327CEE8EC2ECFE1FC2EC0913004D09137
:103FA00031048A3098F481E1809367023F932F9324
:103FB00080E794E09F938F93FF92EF92FE01099523
:103FC0002DB73EB72A5F3F4F2DBF11C080E18093D0
:103FD00067023F932F9385E794E09F938F93FF921F
:103FE000EF92FE0109958DB79EB706968DBF209181
:103FF0006602822F9927AA27BB27FC01429710F05F
:104000000C94462AE85AFF4FBEE8EB2EBFE1FB2E88
:10401000C0913004D09131040C94697B10926702F6
:104020008AE794E09F938F930EE81FE1FF92EF924F
:10403000FE01099584E1809367020F900F900F9025
:104040000F9086E690E09F938F9380E590E09F939A
:104050008F931F921F92809102016AE00E94C27AA0
:10406000892F99279F938F93809102010E94C27A92
:1040700099279F938F938AE894E09F938F93FF9261
:10408000EF92E0913004F0913104099588E2809339
:1040900067022DB73EB7225F3F4F2DBF8AE796E0FC
:1040A0009F938F930E940D2F99279F938F938FE952
:1040B00094E09F938F93FF92EF92E0913004F09100
:1040C000310409958DB79EB708968DBF909149042C
:1040D000992351F08CE380936702892F99279F934E
:1040E0008F938DEA94E085C690916D02992371F0CB
:1040F0008CE380936702892F99279F938F9384EC99
:1041000094E09F938F931F930F9391C080914A04E3
:1041100084FF07C08CE38093670289ED94E00C94E0
:10412000D8298091910190919201069710F00C94FA
:104130004F2A8CE38093670286EE94E00C94D82992
:1041400080911506AEE8EA2EAFE1FA2EC091300458
:10415000D091310480FF74C01092670280911203E5
:1041600090911303A0911403B0911503BC01CD01EC
:1041700025E030E040E050E00E94177B3F932F9312
:1041800083EF94E09F938F93FF92EF92FE01099546
:1041900084E1809367022DB73EB72A5F3F4F2DBF62
:1041A00080910E0390910F03A0911003B091110321
:1041B000BC01CD0125E030E040E050E00E94177BDB
:1041C0003F932F9380E095E09F938F93FF92EF9220
:1041D000E0913004F0913104099588E28093670200
:1041E0008DB79EB706968DBF8091130190911401F3
:1041F0009F938F938DE095E09F938F93FF92EF9223
:10420000E0913004F091310409958CE380936702CA
:104210002DB73EB72A5F3F4F2DBF87B599279F9394
:104220008F938AE195E09F938F93FF92EF92E091B5
:104230003004F091310409958DB79EB706962FC7CB
:104240001092670287E295E09F938F93FF92EF921F
:10425000FE01099584E1809367020F900F900F9003
:104260000F9086E395E09F938F93FF92EF92E091FA
:104270003004F0913104099588E2809367020F9031
:104280000F900F900F908FE395E09F938F93FF9285
:10429000EF92E0913004F091310409958CE3809322
:1042A00067020F900F900F900F908EE495E09F9310
:1042B0008F93FF92EF920C94DC291092670287E5AE
:1042C00095E09F938F930EE81FE1FF92EF92FE011E
:1042D000099584E1809367020F900F900F900F90E3
:1042E0008091700390917103A0917203B091730358
:1042F000B7FF04C081509C4FAF4FBF4FFAE0B59558
:10430000A79597958795FA95D1F7BF93AF939F930C
:104310008F9384E695E09F938F931F930F93E09183
:104320003004F0913104099588E2809367022DB73B
:104330003EB7285F3F4F2DBF80916803909169037E
:10434000A0916A03B0916B03B7FF04C081509C4FEA
:10435000AF4FBF4FEAE0B595A79597958795EA953A
:10436000D1F7BF93AF939F938F9383E795E09F938C
:104370008F931F930F93E0913004F09131040995CE
:104380008CE3809367028DB79EB708968DBF8091AE
:104390003203909133039F938F9382E895E09F932C
:1043A0008F931F930F93E0913004F091310409959E
:1043B0002DB73EB72A5F3F4F0DC71092670280911D
:1043C0003407909135079F938F9380913207909196
:1043D00033079F938F9381E995E09F938F93FF928B
:1043E000EF92FE01099584E1809367028DB79EB735
:1043F00008968DBF80913807909139079F938F93CE
:1044000080913607909137079F938F9381EA95E0CB
:104410009F938F93FF92EF92E0913004F0913104DB
:10442000099588E2809367022DB73EB7285F3F4F1A
:104430002DBF80913C0790913D079F938F93809172
:104440003A0790913B079F938F9381EB95E09F9361
:104450008F93FF92EF92E0913004F091310409952F
:104460008CE3809367028DB79EB708968DBF8091CD
:104470004007909141079F938F9380913E079091C1
:104480003F079F938F9381EC95E0A2C01092670243
:1044900080910A06E82FFF27EE0FFF1FE05DF84F1F
:1044A000808191819F938F9380910906E82FFF2748
:1044B000EE0FFF1FE05DF84F808191819F938F93F6
:1044C00081ED95E09F938F93FF92EF92FE01099506
:1044D00084E1809367028DB79EB708968DBF809167
:1044E0000C06E82FFF27EE0FFF1FE05DF84F8081DD
:1044F00091819F938F9380910B06E82FFF27EE0FFA
:10450000FF1FE05DF84F8081918188589F4F9F93F6
:104510008F9381EE95E09F938F93FF92EF92E091BE
:104520003004F0913104099588E2809367022DB739
:104530003EB7285F3F4F2DBF80910E06E82FFF2723
:10454000EE0FFF1FE05DF84F8081918182599F4FF0
:104550009F938F9380910D06E82FFF27EE0FFF1F8B
:10456000E05DF84F8081918182599F4F9F938F9397
:1045700081EF95E09F938F93FF92EF92E09130044B
:10458000F091310409958CE3809367028DB79EB753
:1045900008968DBF80911006E82FFF27EE0FFF1FB2
:1045A000E05DF84F8081918182599F4F9F938F9357
:1045B00080910F06E82FFF27EE0FFF1FE05DF84FF9
:1045C0008081918182599F4F9F938F9381E096E0E4
:1045D0009F938F93FF92EF92E0913004F09131041A
:1045E00009952DB73EB7285F3F4FF4C5109267027B
:1045F00081E196E09F938F930EE81FE1FF92EF9287
:10460000FE010995809102010F900F900F900F907D
:104610008A3009F0A1C084E180936702809185030C
:10462000909186039C0197FF02C0295F3F4F287F2E
:10463000821B930B9F938F938091850390918603A8
:1046400097FD079673E0959587957A95E1F79F9387
:104650008F93209185033091860337FF02C0295F35
:104660003F4F63E0359527956A95E1F780914802C1
:1046700090914902821B930B9F938F938FE196E059
:104680009F938F931F930F93E0913004F091310427
:10469000099588E2809367028DB79EB70A968DBF11
:1046A00080918303909184039C0197FF02C0295F4E
:1046B0003F4F287F821B930B9F938F93809183039F
:1046C0009091840397FD079653E0959587955A95A9
:1046D000E1F79F938F93209183033091840337FFF9
:1046E00002C0295F3F4F43E0359527954A95E1F792
:1046F0008091460290914702821B930B9F938F9368
:1047000080E396E09F938F931F930F93E091300483
:10471000F091310409958CE3809367022DB73EB781
:10472000265F3F4F2DBF80918103909182039F931D
:104730008F93809181039091820320914402309164
:104740004502821B930B9F938F9381E496E09F9386
:104750008F931F930F93A3C38B3019F0843108F408
:10476000ADC084E1809367028091850390918603B8
:104770009C0197FF02C0215F3F4F207F821B930B5C
:1047800097FD0196959587959F938F9380918503CB
:104790009091860397FD0F9624E0959587952A952D
:1047A000E1F79F938F93209185033091860337FF24
:1047B00002C0295F3F4F83E0359527958A95E1F741
:1047C0008091480290914902821B930B9F938F9393
:1047D0008FE496E09F938F931F930F93E0913004A3
:1047E000F0913104099588E2809367022DB73EB7B6
:1047F000265F3F4F2DBF80918303909184039C01DE
:1048000097FF02C0215F3F4F207F821B930B97FDD4
:104810000196959587959F938F93809183039091AF
:10482000840397FD0F96B4E095958795BA95E1F7C7
:104830009F938F93209183033091840337FF02C0AD
:10484000295F3F4FA3E035952795AA95E1F7809121
:10485000460290914702821B930B9F938F9381E6B0
:1048600096E09F938F931F930F93E0913004F09104
:10487000310409958CE3809367028DB79EB70A9641
:104880008DBF809181039091820397FD019695954C
:1048900087959F938F9380918103909182032091BC
:1048A000440230914502821B930B9F938F9383E7C1
:1048B00096E09F938F931F930F938ECE8D3009F0C8
:1048C000EEC584E1809367028091120199279F933E
:1048D0008F93809185039091860397FD0F96E4E076
:1048E00095958795EA95E1F79F938F93209185039E
:1048F0003091860337FF02C0295F3F4F73E0359543
:1049000027957A95E1F78091480290914902821BA0
:10491000930B9F938F9382E896E09F938F931F93BF
:104920000F93E0913004F0913104099588E280936F
:1049300067028DB79EB70A968DBF809111019927A6
:104940009F938F93809183039091840397FD0F969B
:1049500064E0959587956A95E1F79F938F932091F1
:1049600083033091840337FF02C0295F3F4F53E038
:10497000359527955A95E1F7809146029091470227
:10498000821B930B9F938F9386E996E09F938F935F
:104990001F930F93E0913004F091310409958CE35B
:1049A000809367022DB73EB7265F3F4F2DBF8091A2
:1049B000100199279F938F93809181039091820397
:1049C00097FD0196959587959F938F93809181038D
:1049D000909182032091440230914502821B930BF7
:1049E0009F938F938AEA96E09F938F931F930F93E1
:1049F000E0913004F091310409958DB79EB70A9685
:104A00004EC3109267028EEB96E09F938F93FF92B6
:104A1000EF92FE01099584E1809367020F900F9059
:104A20000F900F9080917B0390917C039F938F93C5
:104A300080914002909141029F938F938BEC96E07E
:104A40009F938F93FF92EF92E0913004F0913104A5
:104A5000099588E2809367022DB73EB7285F3F4FE4
:104A60002DBF8091790390917A039F938F938091CA
:104A70004202909143029F938F938AED96E09F9319
:104A80008F93FF92EF92E0913004F09131040995F9
:104A90008CE3809367028DB79EB708968DBF809197
:104AA0007503909176039F938F9380913E0290912E
:104AB0003F029F938F9389EE96E08ACD1092670212
:104AC00080911D0190911E016AE070E00E94E27ADF
:104AD0009F938F9380911D0190911E016AE070E079
:104AE0000E94E27A7F936F9388EF96E09F938F9373
:104AF000FF92EF92FE01099584E1809367028DB7E2
:104B00009EB708968DBF80916D0890916E086AE0FF
:104B100070E00E94CE7A9F938F9380916D08909160
:104B20006E086AE070E00E94CE7A7F936F938CE00B
:104B300097E09F938F93FF92EF92E0913004F09172
:104B40003104099588E2809367022DB73EB7285F4C
:104B50003F4F2DBF80916F08909170089F938F9366
:104B600080E297E09F938F93FF92EF92E091300461
:104B7000F091310409958CE3809367028DB79EB75D
:104B800006968DBF80917108909172089F938F93C4
:104B900080E397E02EC11092670282E497E09F9332
:104BA0008F93FF92EF92FE01099584E18093670253
:104BB0000F900F900F900F908091300790913107D8
:104BC0009F938F938BE497E09F938F93FF92EF9245
:104BD000E0913004F0913104099588E280936702F6
:104BE0008DB79EB706968DBF8091200399279F931E
:104BF0008F938BE597E09F938F93FF92EF92E091D5
:104C00003004F091310409958CE3809367022DB74D
:104C10003EB72A5F3F4F2DBF80912F0799270197FD
:104C20009F938F938BE697E0FECA109267028BE703
:104C300097E09F938F93FF92EF92FE01099584E195
:104C4000809367020F900F900F900F9080912E032A
:104C500090912F039F938F9383E897E09F938F9377
:104C6000FF92EF92E0913004F0913104099588E2CF
:104C7000809367022DB73EB72A5F3F4F2DBF8091CB
:104C80003203909133039F938F9381E997E09F9331
:104C90008F93FF92EF92E0913004F09131040995E7
:104CA0008CE3809367028DB79EB706968DBF809187
:104CB0003003909131039F938F938FE997E099C0D0
:104CC000109267028091210399279F938F938DEA19
:104CD00097E09F938F93FF92EF92FE01099584E1F5
:104CE000809367028DB79EB706968DBF8091220391
:104CF00099279F938F9389EB97E09F938F93FF92D0
:104D0000EF92E0913004F0913104099588E28093AC
:104D100067022DB73EB72A5F3F4F2DBF8091230317
:104D200099279F938F9385EC97E09F938F93FF92A2
:104D3000EF92E0913004F091310409958CE3809377
:104D400067028DB79EB706968DBF80912403992781
:104D50009F938F9381ED97E04CC0109267028091F2
:104D6000250399279F938F938DED97E09F938F93C2
:104D7000FF92EF92FE01099584E1809367028DB75F
:104D80009EB706968DBF8091260399279F938F9398
:104D900089EE97E09F938F93FF92EF92E09130041A
:104DA000F0913104099588E2809367022DB73EB7F0
:104DB0002A5F3F4F2DBF8091270399279F938F93A1
:104DC00085EF97E09F938F93FF92EF92E0913004ED
:104DD000F091310409958CE3809367028DB79EB7FB
:104DE00006968DBF8091280399279F938F9381E02A
:104DF00098E09F938F93FF92EF92D5CA109267022B
:104E00008DE098E09F938F93FF92EF92FE010995BA
:104E100084E1809367020F900F900F900F90809124
:104E2000A10199279F938F9385E198E09F938F939A
:104E3000FF92EF92E0913004F0913104099588E2FD
:104E4000809367028DB79EB706968DBF80911F0233
:104E5000909120029F938F9383E298E09F938F938A
:104E6000FF92EF92E0913004F091310409958CE3C8
:104E7000809367022DB73EB72A5F3F4F2DBF8091C9
:104E8000380699279F938F938091370699279F9390
:104E90008F9381E398E09F938F93FF92EF92E0913D
:104EA0003004F091310409958DB79EB70896F7C08C
:104EB000109267028FE398E09F938F93FF92EF9297
:104EC000FE01099584E1809367020F900F900F9087
:104ED0000F9080916A04992787FD90959F938F93F7
:104EE00080916904992787FD90959F938F938FE414
:104EF00098E09F938F93FF92EF92E0913004F091AE
:104F00003104099588E2809367022DB73EB7285F88
:104F10003F4F2DBF80916B04992787FD90959F93FC
:104F20008F9380916C0499279F938F938FE598E0DE
:104F30009F938F93FF92EF92E0913004F0913104B0
:104F400009958CE3809367028DB79EB708968DBF55
:104F50008091700499279F938F9380916D04992776
:104F600087FD90959F938F938FE698E031CB1092B9
:104F700067028FE798E09F938F93FF92EF92FE0175
:104F8000099584E1809367020F900F900F900F9026
:104F90008091EA0699278F7790709F938F938091E5
:104FA000E20699278F7790709F938F938091DA060E
:104FB00099278F7790709F938F938091D20699272E
:104FC0008F7790709F938F938FE898E09F938F9344
:104FD000FF92EF92E0913004F0913104099588E25C
:104FE000809367028DB79EB70C968DBF80910A079C
:104FF00099278F7790709F938F93809102079927BD
:105000008F7790709F938F938091FA0699278F776F
:1050100090709F938F938091F20699278F7790706D
:105020009F938F9380EA98E09F938F93FF92EF92E4
:10503000E0913004F091310409958CE3809367028C
:105040002DB73EB7245F3F4F2DBF80912A07992788
:105050008F7790709F938F938091220799278F77F6
:1050600090709F938F9380911A0799278F779070F4
:105070009F938F938091120799278F7790709F93BA
:105080008F9381EB98E09F938F93FF92EF92E09143
:105090003004F091310409958DB79EB70C968DBF01
:1050A000FEC11092670282EC98E09F938F93FF926B
:1050B000EF92FE01099584E1809367020F900F90B3
:1050C0000F900F908091EE06992787FD90959F9302
:1050D0008F938091E606992787FD90959F938F93F4
:1050E0008091DE06992787FD90959F938F938091FD
:1050F000D606992787FD90959F938F9381ED98E031
:105100009F938F93FF92EF92E0913004F0913104DE
:10511000099588E2809367022DB73EB7245F3F4F21
:105120002DBF80910E07992787FD90959F938F93B0
:1051300080910607992787FD90959F938F93809183
:10514000FE06992787FD90959F938F938091F60691
:10515000992787FD90959F938F9382EE98E09F9378
:105160008F93FF92EF92E0913004F0913104099512
:105170008CE3809367028DB79EB70C968DBF8091AC
:105180002E07992787FD90959F938F9380912607EF
:10519000992787FD90959F938F9380911E0799275C
:1051A00087FD90959F938F9380911607992787FD90
:1051B00090959F938F9383EF98E09F938F93FF92A7
:1051C000EF92E0913004F091310409952DB73EB78C
:1051D000245F3F4F2DBF63C11092670284E099E0C6
:1051E0009F938F930EE81FE1FF92EF92FE010995C6
:1051F00084E1809367020F900F900F900F90809141
:10520000EA06881F8827881F97E0899FC00111241C
:105210008D969F938F938091E206881F8827881F21
:1052200096E0899FC00111248D969F938F93809162
:10523000DA06881F8827881F95E0899FC0011124FE
:105240008D969F938F938091D206881F8827881F01
:105250009927880F991F880F991F8D969F938F9379
:1052600083E199E09F938F93FF92EF92E091300456
:10527000F0913104099588E2809367028DB79EB75B
:105280000C968DBF80910A07881F8827881F9BE096
:10529000899FC00111248D969F938F93809102075F
:1052A000881F8827881F9AE0899FC00111248D9646
:1052B0009F938F938091FA06881F8827881F99E013
:1052C000899FC00111248D969F938F938091F20640
:1052D000881F8827881F992723E0880F991F2A9500
:1052E000E1F78D969F938F9387E299E09F938F9339
:1052F000FF92EF92E0913004F091310409958CE334
:10530000809367022DB73EB7245F3F4F2DBF80913A
:105310001207881F8827881F9CE0899FC0011124DD
:105320008D969F938F938BE399E09F938F93FF923A
:10533000EF92E0913004F0913104099580911A07C1
:105340002DB73EB72A5F3F4F2DBF87FF12C080E4C5
:10535000809367028CE499E09F938F93FF92EF9282
:10536000E0913004F091310409950F900F900F9067
:105370000F908091220787FF12C084E48093670218
:105380008FE499E09F938F931F930F93E0913004E4
:10539000F091310409950F900F900F900F9080912C
:1053A0002A0787FF7CC088E48093670282E599E042
:1053B0009F938F931F930F93E0913004F0913104EA
:1053C00009950F900F900F900F9069C0109267028F
:1053D00085E599E09F938F93FF92EF92FE010995E7
:1053E00084E1809367020F900F900F900F9080914F
:1053F000F7019091F8019F938F9383E699E09F9333
:105400008F93FF92EF92E0913004F091310409956F
:1054100088E2809367028DB79EB706968DBF809114
:10542000F9019091FA019F938F9380E799E09F9300
:105430008F93FF92EF92E0913004F091310409953F
:1054400089E4809367022DB73EB72A5F3F4F2DBF97
:105450008DE799E09F938F93FF92EF92E091300454
:10546000F09131040995809165020F900F900F9093
:105470000F9083FF14C01092FA011092F90160E0BE
:1054800070E08EE090E00E94BB2D09C080911F016A
:10549000281719F4215020931F01109266021092D0
:1054A0006502E6E0CDB7DEB70C945A7BF999FECFE2
:1054B00092BD81BDF89A80B599270895F999FECFDC
:1054C0001FBA92BD81BD60BD0FB6F894FA9AF99AE1
:1054D0000FBE08954AEA20E030E02617370740F46F
:1054E000FC018191480F2F5F3F4F26173707C8F304
:1054F000842F99270895EAEA40E050E046175707BD
:1055000078F49C01F999FECF32BD21BDF89A80B59F
:10551000E80F4F5F5F4F2F5F3F4F4617570790F3DE
:105520008E2F9927089581E080930B0682E0809367
:105530000A0683E08093090684E080930C0685E0E8
:1055400080930D0686E080930E0687E080930F0619
:1055500088E08093100689E0809311068AE08093AA
:1055600012068BE0809313068CE080931406089556
:105570001F93CF93DF9384E5809308068091020107
:10558000843150F08AE08093280610924A068BE11D
:10559000809324068EE40AC083E08093280680E28C
:1055A00080934A068EE18093240685E58093470622
:1055B000809348068AE68093150683E080936B0605
:1055C000AEE1A09316068FEF80931806EFE0E0930C
:1055D0001906A093170610921B06F8E0F0931C061C
:1055E00080E480931D0610921E0684E180931A06C3
:1055F0008EE080931F06B0E1B09320061CE010936C
:105600002106F093220686EE8093230680E880939D
:10561000250650E55093260686E980932706509389
:10562000290680932A0676E070932B0681E2809308
:105630002C068DE280932D069AE590932E0680E24B
:105640008093300610923106109232061092330683
:105650001092340610924C0610924D0610924E068F
:1056600010924F0634E63093350648E240933606F2
:1056700061E060936A061092370627EF20933806A0
:1056800070933D068DE780933E0680933F0680939E
:1056900040063093390640933A0610923B06209319
:1056A0003C0682E380934106909342068093430632
:1056B00010926906909344065093450660934606FF
:1056C000B093490630934B068FE58093500683EFE5
:1056D000809352068AEA8093540680935506E0939D
:1056E0005106E09353068EEF80935606309357068B
:1056F000909358069093590690935A068BE48093A2
:105700005B0680935C0680935D0610925E06709344
:105710005F06F093600690936106A0936206309353
:1057200063063093640682E08093650660932F06DB
:105730001092670610926806ACE6B6E0E0E7F1E08A
:10574000ED01019009921A95E1F760E770E0CD0153
:10575000845690400E946A2A80937806DF91CF9108
:105760001F910895CF93DF9384E58093080680917D
:105770000201843150F08AE08093280610924A0694
:105780008BE1809324068EE40AC083E08093280690
:1057900080E280934A068EE18093240685E580931B
:1057A0004706809348068AE68093150683E0809337
:1057B0006B067EE1709316068FEF809318069FE0CC
:1057C000909319067093170610921B0668E0609379
:1057D0001C0680E480931D0610921E0690931A0604
:1057E0008AE080931F0680E18093200656E0509364
:1057F00021066093220686EE8093230680E880933C
:1058000025062AE52093260688E78093270620931D
:10581000290680932A0650932B0681E280932C065A
:105820008DE280932D0620932E06E0E2E093300671
:1058300010923106109232061092330610923406FE
:1058400010924C0610924D0610924E0610924F0682
:1058500044E64093350638E230933606F1E0F093A3
:105860006A061092370697EF9093380650933D06DC
:105870008DE780933E0680933F06809340064093D9
:10588000390630933A0610923B0690933C0682E329
:105890008093410620934206809343061092690646
:1058A0002093440680E5809345068CE3809346066A
:1058B000E09349069BE490934B068FE58093500656
:1058C00083EF809352068AEA8093540680935506AC
:1058D00084E180935106809353068EEF80935606A1
:1058E00040935706209358062093590620935A0652
:1058F00090935B0690935C0690935D0610925E0613
:1059000050935F0660936006209361067093620671
:10591000409363064093640682E080936506F093AB
:105920002F061092670610926806ACE6B6E08CE08F
:10593000E7E7F1E0ED01019009928A95E1F760E770
:1059400070E0CD01845690400E946A2A80937806C8
:10595000DF91CF910895CF93DF9384E5809308067C
:1059600080910201843150F08AE0809328061092E1
:105970004A068BE1809324068EE40AC083E080937C
:10598000280680E280934A068EE18093240685E50E
:1059900080934706809348068AE68093150683E045
:1059A00080936B066EE1609316068FEF8093180666
:1059B0009FE0909319066093170610921B0678E0FB
:1059C00070931C0680E480931D0610921E0690932F
:1059D0001A0670931F0690E19093200656E05093AC
:1059E00021067093220686EE8093230680E880933A
:1059F000250634E63093260688E780932706309301
:105A0000290680932A0650932B0681E280932C0668
:105A10008DE280932D062AE520932E069093300682
:105A2000109231061092320610923306109234060C
:105A300010924C0610924D0610924E0610924F0690
:105A40003093350648E240933606E1E0E0936A067B
:105A50001092370697EF9093380650933D068DE7E6
:105A600080933E0680933F0680934006309339062C
:105A700040933A0610923B0690933C0682E3809353
:105A800041062093420680934306109269062093B4
:105A9000440680E58093450696E49093460680E2AE
:105AA0008093490690934B068FE58093500683EFD1
:105AB000809352068AEA8093540680935506609339
:105AC0005106609353068EEF809356063093570627
:105AD000209358062093590620935A068BE480930E
:105AE0005B0680935C0680935D0610925E06509381
:105AF0005F067093600620936106609362063093A0
:105B000063063093640682E080936506E0932F0677
:105B10001092670610926806ACE6B6E08CE0EFE7FC
:105B2000F1E0ED01019009928A95E1F760E770E0FC
:105B3000CD01845690400E946A2A80937806DF91B6
:105B4000CF910895F999FECF92BD81BDF89A80B5A5
:105B500099270895F999FECF1FBA92BD81BD60BD06
:105B60000FB6F894FA9AF99A0FBE089566E57AE2AC
:105B70000E94317908954EE55AE20E946B790895AA
:105B8000EF92FF920F931F93CF93C82F81508530D0
:105B900008F0C3E081E7C89F8001112483EFE82E5D
:105BA0008FEFF82EE00EF11E60E770E0C7010E9453
:105BB0007B2A682F98012D593F4F8FB39927AC014D
:105BC0004270507081FDF9CF32BD21BDF89A80B589
:105BD000861711F0CA0121C08FB399279C0122704A
:105BE000307081FDF9CFF2BCE1BCF89A80B5843504
:105BF00011F0C90112C081E7C89FC00111240D979F
:105C000026E53AE241E750E0BC0188E096E00E94D8
:105C10000C790E940D6A81E090E0CF911F910F9165
:105C2000FF90EF900895282F863010F025E003C0F4
:105C3000882309F421E0F999FECF1FBA82E090E0B1
:105C400092BD81BD20BD0FB6F894FA9AF99A0FBEA5
:105C50000895CF93C82F80910806843509F042C07B
:105C6000C63010F0C5E003C0CC2309F43BC060E7A8
:105C700070E088E096E00E946A2A8093780681E7C7
:105C8000C89FC00111242EE53AE241E750E068E0E8
:105C900076E00D970E9449792EE53AE24CE050E01B
:105CA00069E076E080E590E00E9449796CE070E080
:105CB00089E096E00E946A2A282FF999FECF1FBA40
:105CC0008CE590E092BD81BD20BD0FB6F894FA9AA4
:105CD000F99A0FBE8C2F0E94132E0E940D6A81E04C
:105CE00090E002C080E090E0CF9108956DE470E014
:105CF00088EE93E00E947B2A482F8FB399279C015E
:105D00002270307081FDF9CF85E394E092BD81BDB2
:105D1000F89A80B5841779F48FB399279C01227083
:105D2000307081FDF9CF88EE93E092BD81BDF89A85
:105D300080B5813011F0C901089526E53AE24EE4BC
:105D400050E068EE73E089E796E00E940C7981E00C
:105D500090E00895809179068130A9F46DE470E0B7
:105D600089E796E00E946A2A8093C6062EE53AE209
:105D70004EE450E069E776E088EE93E00E944979CE
:105D800081E090E0089580E090E00895CF93DF9364
:105D900081E080937906E9E7F6E08FE015861686C4
:105DA0001786108A8150349687FFF8CF80E480935D
:105DB00086068093870610928806809389068093D2
:105DC0008A0690EC90938B0610928C0680938D0639
:105DD00080938E0610928F06909390069093910672
:105DE0008093920610929306809394069093950662
:105DF000AAE7B6E087E0E9E8F1E0ED010190099259
:105E00008A95E1F76DE470E0CD0101970E946A2A5E
:105E10008093C606DF91CF910895F999FECF82E075
:105E200090E092BD81BDF89A80B5282F863078F039
:105E300023E0322FF999FECF1FBA82E090E092BDA5
:105E400081BD30BD0FB6F894FA9AF99A0FBE822F31
:105E500099270895DF92EF92FF920F931F93CF93AC
:105E6000FF24DF2CEF2C81E090E00E94A22D8435EE
:105E700039F031E0E32E64E581E090E00E94AA2D44
:105E80006CE070E080E590E00E947B2AC82FF999D1
:105E9000FECF8CE590E092BD81BDF89A80B58C175D
:105EA00011F421E0D22EC1E001E010E0EE2029F44F
:105EB0008C2F0E94C02D8823C1F591E0F92E1F93ED
:105EC0000F9385E899E09F938F938BE392E19F93E3
:105ED0008F93E0913004F091310409958DB79EB70E
:105EE00006968DBF0230110549F0033011054CF4C0
:105EF0000130110531F40E94B82A05C00E94B22B6E
:105F000002C00E94AB2CDD2059F026E53AE24CE0BD
:105F100050E060E570E089E096E00E940C7902C0F4
:105F20000E94932A8C2F0E94292ECF5F0F5F1F4F54
:105F3000C63008F4BBCFFF2019F083E00E94132E77
:105F40000E940D2FC82F0E94C02D8C2F99279F9340
:105F50008F938BEA99E09F938F930BE312E11F934A
:105F60000F93E0913004F091310409958DB79EB7FD
:105F700006968DBFEE2021F40E94762E882399F498
:105F800084EC99E09F938F931F930F93E0913004DB
:105F9000F091310409950E94C62E0E94AA2E0F90FE
:105FA0000F900F900F901092070690E0E6E8F6E051
:105FB000CFE08081349618160CF49F5FC150C7FF64
:105FC000F8CF90930706892F99279F938F938AE79D
:105FD00096E09F938F9385EE99E09F938F931F9305
:105FE0000F93E0913004F091310409958DB79EB77D
:105FF00008968DBF86E09AE09F938F931F930F932F
:10600000E0913004F091310409950F900F900F90BA
:106010000F90CF911F910F91FF90EF90DF90089517
:106020009FB7F8943998389A88B1836088B980917D
:10603000B9008C7F8093B9008AE28093B8001092F7
:10604000710210926F0210926E02EFECF6E08BE09C
:106050001082118212821382148215821682178294
:106060008150389687FFF4CF9FBF08951092710238
:1060700084E98093BC0010926F0210926E0280E857
:106080008093BC001092BD001092BA001092BB0029
:106090001092B9001092B8000E9410301092BB000C
:1060A00085E88093BC0080916C02826080936C02D2
:1060B00008951F920F920FB60F9211242F933F93C2
:1060C0004F935F938F939F93EF93FF938091710210
:1060D000282F3327442755278F5F80937102F901BA
:1060E0002731310508F0B3C2E659FF4F0C94697BA4
:1060F00080916F028C3090F480916F028F5F80935B
:106100006F0280916F02E82FFF27EE0FFF1FEE0F47
:10611000FF1FE758F94F8585181654F780916F02D5
:106120008C3070F010926B0210926A0210926F0223
:1061300085E08093710280916E02880F8D5A04C0B1
:1061400080916F02880F8E5A8093BB0085E874C2DD
:1061500080916F02E82FFF2783E0EE0FFF1F8A95E3
:10616000E1F7E153F94F81818093BB0085E880938B
:10617000BC0080916F02E82FFF27EE0FFF1FEE0F8C
:10618000FF1FEE0FFF1FE153F94F808180FF91C089
:1061900080916F02E82FFF27EE0FFF1FEE0FFF1F0A
:1061A000EE0FFF1FE153F94F8281882329F0809180
:1061B0000706873008F45FC280916A0290916B02F3
:1061C000892B09F058C28091680290916902892B4D
:1061D00009F051C26EC080916F0221E030E002C030
:1061E000220F331F8A95E2F780916802909169022D
:1061F00028233923232B79F080916F02E82FFF2782
:10620000EE0FFF1FEE0FFF1FEE0FFF1FE153F94FC1
:1062100080E184830DC080916F02E82FFF27EE0F8D
:10622000FF1FEE0FFF1FEE0FFF1FE153F94F148208
:1062300080916F02E82FFF2753E0EE0FFF1F5A9562
:10624000E1F7E153F94F8481282F332743E0220FF0
:10625000331F4A95E1F780916F02E82FFF2793E003
:10626000EE0FFF1F9A95E1F7E153F94F8281877096
:10627000822B8093BB0085E88093BC0020916F0245
:1062800081E090E002C0880F991F2A95E2F72091E3
:106290006A0230916B0282239323892B51F087ECA1
:1062A00096E0909375028093740288E08093760262
:1062B000E2C184E080C1E0917402F09175028191A5
:1062C0008093BB0085E88093BC00F0937502E09357
:1062D000740280917602815080937602882309F4BB
:1062E000CAC183E068C18091B900803351F58091C3
:1062F0007202882329F480916F028F5F809372026B
:1063000080916F02E82FFF2783E0EE0FFF1F8A9531
:10631000E1F7E153F94F838199278F7790708F3799
:1063200091057CF480916F02E82FFF27EE0FFF1F8D
:10633000EE0FFF1FEE0FFF1FE153F94F83818F5FB9
:1063400083831092710284E98093BC008AE090E01C
:10635000909392018093910180916F028F5F80935F
:106360006F021092710262C18091B9008034A9F16C
:1063700080916E02E82FFF27EE0FFF1FEE0FFF1F29
:10638000EE0FFF1FE153F94F83818F778383809155
:106390006E028F5F80936E0280916E028C30A0F04F
:1063A00010926E021092690210926802809173023C
:1063B0008F5F809373028C3038F01092730280915B
:1063C0006C028D7F80936C0280916C02816080935F
:1063D0006C021092710284E971C080916E02E82F04
:1063E000FF27EE0FFF1FEE0FFF1FEE0FFF1FE15302
:1063F000F94F83818068838380916E02E82FFF27A5
:10640000EE0FFF1FEE0FFF1FEE0FFF1FE153F94FBF
:10641000808180FF2FC080916E02E82FFF2753E01C
:10642000EE0FFF1F5A95E1F7E153F94F8481992749
:10643000009751F04097D9F587EC96E0909375025C
:106440008093740288E031C080916E02992743E006
:10645000880F991F4A95E1F78C52994F90937502D6
:106460008093740290916E02809173029817E1F408
:1064700083E01BC080916E02992733E0880F991F3B
:106480003A95E1F78C52994F90937502809374027C
:1064900080916C0281FD06C090916E028091730222
:1064A000981711F482E001C081E080937602809118
:1064B0007602813011F485E801C085EC8093BC0040
:1064C0008091720280936D0210927202D4C0E091AA
:1064D0007402F09175028091BB00808380917402F8
:1064E0009091750201969093750280937402809149
:1064F0007602815080937602823010F085EC58C08D
:10650000813011F485E854C080916C0281FF2DC068
:106510008091E80280FD1DC080916E02E82FFF2768
:1065200023E0EE0FFF1F2A95E1F7E153F94F868133
:106530008A3F79F480916E02E82FFF2793E0EE0FF7
:10654000FF1F9A95E1F7E153F94F808181608083C5
:106550000CC080916E02E82FFF2783E0EE0FFF1F33
:106560008A95E1F7E153F94F108280916E028F5FB7
:1065700080936E0280916E028C30A0F010926E02B9
:106580001092690210926802809173028F5F80936B
:1065900073028C3038F01092730280916C028D7F00
:1065A00080936C021092710284E98093BC0049C010
:1065B0008093BC0086E0809371025DC088E9C4CD01
:1065C00080917002880F805FBFCD80917002992703
:1065D0008130910561F0823091051CF4892B21F006
:1065E0004AC0029739F047C080911201ADCD809129
:1065F0001101AACD80911001A7CD80E8A5CD109200
:10660000710284E98093BC008AE090E0909392014B
:106610008093910180917002823088F480917002A1
:106620008F5F8093700282E18093710280916C028F
:106630008E7F80936C0285EA8093BC001CC0109210
:10664000700280916C02816080936C0214C0109281
:10665000710284E98093BC0080916C028160809318
:106660006C028AE090E090939201809391011092E5
:106670006F0210926E02FF91EF919F918F915F9147
:106680004F913F912F910F900FBE0F901F90189533
:106690001F93CF93DF93182F80911703882321F442
:1066A00080910402882319F081E090E097C01D30AA
:1066B00008F092C01123B1F0E12FFF2723E0EE0F85
:1066C000FF1F2A95E1F7E153F94F35978081359601
:1066D00088230CF081C03897808180FD03C083E05F
:1066E00090E07CC08091C706823019F084E090E091
:1066F00075C067E070E087EC96E00E946A2A90918E
:10670000CE06891719F085E090E068C080ED97E02B
:106710000E946216EC0180916C0280FD05C0CE01E2
:106720000E946B168823B9F3112319F48FEF90E0C0
:106730000BC0212F33272150304081E090E002C070
:10674000880F991F2A95E2F790936B0280936A0253
:10675000A1E0B0E0EFECF6E040E050E06BE0CD010E
:10676000042E02C0880F991F0A94E2F720916A0252
:1067700030916B0282239323892B11F011821282B4
:1067800061504F5F5F4F389667FFE9CF10926F02FD
:106790001092710280916C028E7F80936C0285EA68
:1067A0008093BC0080916C0280FD05C0CE010E94E8
:1067B0006B168823B9F380916A0290916B02892B42
:1067C00029F0CE010E946B16882311F380916A0292
:1067D00090916B02009711F082E090E0DF91CF91F1
:1067E0001F9108950F931F93CF93DF93982F80915C
:1067F0001703882321F480910402882319F081E093
:1068000090E092C09D30A0F4992319F486E090E0C6
:106810008BC0C92FDD27FE0133E0EE0FFF1F3A9535
:10682000E1F7E153F94F35978081359687FD03C035
:1068300082E090E079C03897808180FD03C083E0DA
:1068400090E072C080ED97E00E9462168C0180910A
:106850006C0280FD05C0C8010E946B168823B9F345
:10686000219721E030E0C90102C0880F991FCA9525
:10687000E2F79093690280936802D901EFECF6E0A9
:1068800040E050E06BE0CD01042E02C0880F991F5C
:106890000A94E2F7209168023091690282239323DF
:1068A000892B11F01182128261504F5F5F4F389631
:1068B00067FFE9CF10926E021092C7061092CE06C3
:1068C0001092710280916C028E7F80936C0285EA37
:1068D0008093BC0080916C0280FD05C0C8010E94BD
:1068E0006B168823B9F38091680290916902892B15
:1068F00029F0C8010E946B16882311F38091C70606
:10690000823019F084E090E00FC067E070E087EC1F
:1069100096E00E946A2A9091CE06891719F085E0C8
:1069200090E002C080E090E0DF91CF911F910F9145
:10693000089589E1A4E6B7E0E0E3F7E01182108270
:10694000329611961C921E921296815087FFF6CFB6
:106950001092820310928103109284031092830399
:10696000109286031092850308951F920F920FB61E
:106970000F9211240F931F932F933F934F935F9385
:106980006F937F938F939F93AF93BF93CF93DF9337
:10699000EF93FF9380916B0682FDCFC040918600FC
:1069A000509187008091780290917902481B590B91
:1069B000809186009091870090937902809378026D
:1069C000CA018D549440A0917A02B0917B02835FFA
:1069D0009A4178F480917A0280932F07149714F0EB
:1069E0001092930181E090E090937B0280937A0271
:1069F00007C2AD30B1050CF003C2CA018B5F9040F5
:106A0000845B914008F074C0425D5140FD01EA0F83
:106A1000FB1FE05DF84F80819181FA01E81BF90BC3
:106A2000CF01F7FF03C0909581959F4F06975CF4C7
:106A300080912003883C20F480912003865F01C070
:106A400088EC80932003FD01EA0FFB1FE05DF84F07
:106A5000808191819C01220F331F280F391F240F41
:106A6000351F37FF02C02D5F3F4FE901D595C79510
:106A7000D595C795CA0101968C179D0714F42197E7
:106A800006C041505040C417D5070CF421968091A0
:106A90002003833CE0F08D010A0F1B1FF801E05D2D
:106AA000F84F808191819E01281B390BC90163E059
:106AB00070E00E94E27ACB01880F991F860F971F22
:106AC0000C59184FD80111969C938E9307C0AA0FAA
:106AD000BB1FAC59B84F11961C921E92E0917A02DE
:106AE000F0917B02EE0FFF1FE05DF84FD183C08372
:106AF00020917A0230917B022F5F3F4F30937B02CF
:106B000020937A0280910201843108F079C1253006
:106B1000310511F45D9A01C05D9880917A029091DF
:106B20007B028630910511F45C9A01C05C9807974E
:106B300011F45B9A65C15B9863C1409186005091E6
:106B4000870080917C0290917D02481B590B8091B7
:106B500086009091870090937D0280937C02CA0109
:106B60008D5494406091E602835F9A4108F07AC0A8
:106B70006093770280917702843008F453C090913B
:106B80002F0780917702981709F04CC05091E702C7
:106B90005B3008F43FC0109293011092E60240E08F
:106BA0005F31C0F0E42FFF27EE0FFF1F9F012E542F
:106BB0003D4FDF01A05DB84F8D919C91D9018D9320
:106BC0009C93DF01AC59B84F8D919C91E453FD4FDC
:106BD00091838083E42FFF27EE0FFF1F9F01205D2D
:106BE000384FDF01A258BD4F8D919C91D90111966C
:106BF0009C938E93DF01A856BD4F8D919C91EC59CB
:106C0000F84F91838083842F8F5F482F8D3040F21F
:106C10008093E6028091E7028F3FB9F08F5F809307
:106C2000E70213C08091E702853620F08AE0809366
:106C3000E70202C01092E702809102018A3011F04F
:106C4000843110F0289A01C0289881E08093E602F0
:106C500080911703882309F0D3C080917702809335
:106C60002F07CEC06D3008F0A3C0CA018B5F9040E3
:106C7000845B914008F07EC0425D5140E62FFF27C3
:106C8000EE0FFF1FE258FD4F80819181FA01E81B52
:106C9000F90BCF0105960B97B0F48091E7028A318A
:106CA00020F080912003865F05C08B3028F0809112
:106CB00020038E5F8093200380912003893C18F08D
:106CC00088EC80932003E62FFF27EE0FFF1FE2588A
:106CD000FD4F808191819C01220F331F280F391FA6
:106CE000240F351F37FF02C02D5F3F4FE901D595B7
:106CF000C795D595C795CA0101968C179D0714F4C1
:106D0000219706C041505040C417D5070CF4219676
:106D1000809120038E3BD8F0E62FFF27EE0FFF1F58
:106D2000DF01A258BD4F8D919C919E01281B390B0C
:106D3000C90163E070E00E94E27ACB01880F991FDD
:106D4000860F971FE856FD4F9183808308C0E62F7A
:106D5000FF27EE0FFF1FE856FD4F11821082809132
:106D6000E602E82FFF27EE0FFF1FE258FD4FD18309
:106D7000C08309C0809102018A3011F0843110F083
:106D8000289A01C0289880910201843188F480916A
:106D9000E602853011F45D9A05C05D98863011F4E5
:106DA0005C9A05C05C98873011F45B9A01C05B98CF
:106DB0008091E602843120F48F5F8093E60220C048
:106DC0008431F1F4809102018A3011F0843110F0A5
:106DD000289A01C028988EE18093E6022CE0C4E650
:106DE000D7E0A2EBB2E0E0E3F7E08D919D919183D3
:106DF00080833296198218822296215027FFF5CF80
:106E0000FF91EF91DF91CF91BF91AF919F918F91C2
:106E10007F916F915F914F913F912F911F910F91B2
:106E20000F900FBE0F901F901895EF92FF920F9347
:106E30001F93809124069927880F991F880F991F07
:106E40007C010027F7FC0095102F80917003909132
:106E50007103A0917203B0917303BC01CD01A8012D
:106E600097010E94177B3093B8052093B705809156
:106E7000680390916903A0916A03B0916B03BC0110
:106E8000CD01A80197010E94177B3093BA0520938A
:106E9000B9058091EA079091EB0797FD03969595C8
:106EA0008795959587959093BC058093BB058091B8
:106EB000FA079091FB0797FD039695958795959511
:106EC00087959093BE058093BD0580918103909135
:106ED00082032091440230914502821B930B9093D0
:106EE000C0058093BF058091120390911303A09178
:106EF0001403B0911503BC01CD0125E030E040E062
:106F000050E00E94177B3093C2052093C105809109
:106F10003E0290913F029093C4058093C3058091F7
:106F20003203909133039093C8058093C7058091F5
:106F30001D0190911E019093CA058093C90580910F
:106F4000200399279093CC058093CB058091F60779
:106F50009091F707A091F807B091F907209195015A
:106F6000309196014091970150919801BC01CD015B
:106F70000E94177B3093CE052093CD058091D006DB
:106F800099279093D0058093CF058091D8069927B3
:106F90009093D2058093D1058091E0069927909334
:106FA000D4058093D3058091E80699279093D60560
:106FB0008093D50580911F02909120029093E00567
:106FC0008093DF0580916D0890916E089093E405A1
:106FD0008093E30580917108909172089093E60583
:106FE0008093E5058091730899279093F20580932B
:106FF000F10580910104909102049093F40580932F
:10700000F3058091FF03909100049093F60580931F
:10701000F50580914904882321F480914A0488234E
:1070200021F08091B605816003C08091B6058E7F06
:107030008093B6051F910F91FF90EF9008951F93D5
:10704000CF93DF93182FEB01809117038823A1F4CE
:1070500011501F3F89F0D0932402C09323028091E6
:10706000230290912402892BD1F7CE018C0F9D1F12
:107070000E947716115078F7DF91CF911F910895F4
:10708000CF93DF93809102018D3011F40E94101B89
:1070900010927A0080914802909149029093B10732
:1070A0008093B00780914602909147029093A20787
:1070B0008093A10780914402909145029093F0073C
:1070C0008093EF072091400230914102C901880F5F
:1070D000991F880F991F820F931F820F931F909300
:1070E000EB078093EA072091420230914302C901E5
:1070F000880F991F880F991F820F931F820F931F6C
:107100009093FB078093FA078FEC80937A00A1E2BB
:10711000B3E0CDE0D6E097E08991E82FFF27EE0FAE
:10712000FF1FE05DF84F0190F081E02DE259FF4F25
:107130001E161F061CF0E0E0F0E005C0EF3FF10571
:1071400014F0EFEFF0E08C91282F3327E217F307CC
:1071500014F4815004C02E173F0714F48F5F8C93F2
:107160009150119697FFD8CF809147069927AA276B
:10717000BB27BC01CD0124EC39E040E050E00E9487
:10718000A37ADC01CB018093B7019093B801A0935F
:10719000B901B093BA01809148069927AA27BB2765
:1071A000BC01CD010E94A37ADC01CB018093B30125
:1071B0009093B401A093B501B093B601DF91CF9144
:1071C0000895A0E0B0E0E7EEF8E30C94387B882E59
:1071D000C0E0D0E07E016E0110924904469AD0933F
:1071E0007C03C0937B03D0937A03C0937903D0933D
:1071F0007603C0937503D0938603C0938503D09321
:107200008403C0938303D0938203C09381031092BD
:107210009E0110929D01109238020E94403884E62F
:1072200090E00E9484160E9440388091150680FFED
:1072300010C08091130190911401875B934038F442
:1072400080911301909114018E5E924010F40E947F
:10725000B61A0FE18AE090E00E9484168091440201
:1072600090914502C80FD91F809148029091490220
:10727000E80EF91E8091460290914702C80ED91E71
:10728000015007FFE7CF9701205F3F4F36952795C5
:10729000369527953093860320938503C601409643
:1072A000969587959695879590938403809383030D
:1072B0006096F5E0D695C795FA95E1F7D0938203ED
:1072C000C09381039093800380937F0330937E0368
:1072D00020937D03882009F441C08091EA079091B2
:1072E000EB0797FF03C0909581959F4F6CE070E08E
:1072F0000E94E27A9B0170937C0360937B038091F0
:10730000FA079091FB0797FF03C0909581959F4FD7
:107310006CE070E00E94E27A70937A0360937903E4
:107320008091FA059091FB05909376038093750305
:10733000B90184E090E00E94BB2D609179037091C7
:107340007A0386E090E00E94BB2D609175037091F6
:10735000760388E090E00E94BB2D65C084E090E059
:107360000E94B62D90937C0380937B0386E090E08F
:107370000E94B62D90937A038093790388E090E081
:107380000E94B62D9C0190937603809375038091A3
:107390007B0390917C038150984050F48091790355
:1073A00090917A038150984018F421503440D8F1DC
:1073B00087E29AE09F938F938BE392E19F938F9361
:1073C000E0913004F091310409958091EA079091A1
:1073D000EB0797FF03C0909581959F4F6CE070E09D
:1073E0000E94E27A70937C0360937B038091FA079A
:1073F0009091FB0797FF03C0909581959F4F6CE09C
:1074000070E00E94E27A70937A036093790380912E
:10741000FA059091FB0590937603809375030F9086
:107420000F900F900F901092B1071092B00710922A
:10743000A2071092A1071092F0071092EF0784E6BE
:1074400090E00E94841680914002909141029C013C
:10745000220F331F220F331F280F391F280F391F08
:107460003093EB072093EA07809142029091430208
:107470008C01000F111F000F111F080F191F080F9B
:10748000191F1093FB070093FA0780912406C82E5A
:10749000DD24EE24FF24442737FD4095542FC701F7
:1074A000B6010E94A37A4B015C0160937003709354
:1074B000710380937203909373039801442737FDFF
:1074C0004095542FC701B6010E94A37ADC01CB017D
:1074D0008093680390936903A0936A03B0936B034E
:1074E00080924C0390924D03A0924E03B0924F03B2
:1074F0008093440390934503A0934603B0934703BE
:1075000010924003109241031092420310924303E1
:107510008091150190911601A0911701B091180169
:107520009093FD058093FC0510923702109236026D
:1075300010923403109235031092360310923703E1
:107540008091320390913303909331038093300301
:107550000E94A46582E390E090932402809323022A
:10756000809147069927AA27BB27BC01CD0124ECAF
:1075700039E040E050E00E94A37ADC01CB0188565C
:10758000954CAF4FBF4F8093B7019093B801A09334
:10759000B901B093BA01809148069927AA27BB2761
:1075A000BC01CD010E94A37ADC01CB018856954C29
:1075B000AF4FBF4F8093B3019093B401A093B50137
:1075C000B093B60110929A01109299018091320302
:1075D00090913303AA2797FDA095BA2F209195018A
:1075E000309196014091970150919801BC01CD01D5
:1075F0000E94A37ADC01CB018093F6079093F707F2
:10760000A093F807B093F90710922B0310922A0366
:1076100081E0809301010E940D6A8091E8028460FC
:107620008093E8028FEF809368081092690880E2E7
:1076300080936A08C1E2D3E0ADE0B6E007E08D9147
:10764000E82FFF27EE0FFF1FE05DF84F808191814B
:1076500082598993015007FFF2CF84E6809320037B
:1076600080912102882311F0469A579A80918503D0
:107670009091860380569940815C9B4228F08091CE
:10768000490481608093490480918303909184032D
:1076900080569940815C9B4228F080914904826029
:1076A0008093490480918103909182038C52914090
:1076B0008957954028F0809149048460809349045B
:1076C00080917B0390917C038C529140835C91402C
:1076D00028F080914904886080934904809179035F
:1076E00090917A038C529140835C914028F0809174
:1076F00049048061809349048091750390917603D9
:10770000805092408355914028F0809149048062D6
:1077100080934904ECE0CDB7DEB70C94547BABE02A
:10772000B0E0E5E9FBE30C94327B8091810390911A
:1077300082032091440230914502821B930B909367
:10774000F0078093EF0780914E0290914F0297FDD2
:1077500007969C01F3E035952795FA95E1F730936C
:10776000B1072093B00780914C0290914D0297FD94
:107770000796E3E095958795EA95E1F79093A20740
:107780008093A1073093BC072093BB079093B40765
:107790008093B3078091EA079091EB07AC01440F07
:1077A000551F480F591F2091400230914102C901D5
:1077B000880F991F880F991F820F931F820F931FA5
:1077C000480F591F57FF02C04D5F5F4F55954795B2
:1077D000559547955093EB074093EA078091FA0738
:1077E0009091FB07AC01440F551F480F591F209182
:1077F000420230914302C901880F991F880F991FD7
:10780000820F931F820F931F480F591F57FF02C00B
:107810004D5F5F4F55954795559547955093FB079D
:107820004093FA072091400230914102C901880F2C
:10783000991F880F991F820F931F820F931F9C011E
:10784000442737FD4095542F809160039091610348
:10785000A0916203B0916303820F931FA41FB51F11
:107860008093600390936103A0936203B0936303DA
:107870002091420230914302C901880F991F880F5D
:10788000991F820F931F820F931F9C01442737FD7E
:107890004095542F80915C0390915D03A0915E030D
:1078A000B0915F03820F931FA41FB51F80935C03E9
:1078B00090935D03A0935E03B0935F038091C5072F
:1078C0009091C6072091400230914102820F931F90
:1078D0009093C6078093C5078091F2079091F307B4
:1078E0002091420230914302820F931F9093F3073D
:1078F0008093F2078091770390917803019690939B
:107900007803809377038091FA059091FB0520918D
:10791000750330917603821B930B9C01442737FD3E
:107920004095542F8091580390915903A0915A0388
:10793000B0915B03820F931FA41FB51F8093580360
:1079400090935903A0935A03B0935B038FEC8093F9
:107950007A0010920F012090480330904903409024
:107960004A0350904B0329E422162BE6320621E00D
:10797000420620E052064CF088E49BE6A1E0B0E02D
:1079800089839A83AB83BC8316C098EB291694E94C
:1079900039069EEF49069FEF59064CF428EB34E96F
:1079A0004EEF5FEF29833A834B835C8304C02982C7
:1079B0003A824B825C828091500390915103A09156
:1079C0005203B09153038D839E83AF83B88789544C
:1079D0009B46A140B04044F0E8E46E2EEBE67E2EDC
:1079E000E1E08E2E912C16C02D813E814F8158856D
:1079F000285B34494E4F5F4F4CF478EB672E74E9A7
:107A0000772E7EEF872E7FEF972E04C06D807E80CD
:107A10008F809884A091EF07B091F007BB87AA8769
:107A2000FD01CF01AA2797FDA095BA2F2091400311
:107A3000309141034091420350914303280F391F75
:107A40004A1F5B1F2093400330934103409342033E
:107A5000509343032091F6073091F7074091F807C0
:107A60005091F907280F391F4A1F5B1F2093F60713
:107A70003093F7074093F8075093F9079091150654
:107A800092FD04C080910103833310F01092CD0762
:107A9000F0910703F987FF2309F0A7C1809106033E
:107AA000882309F0A2C18091CD07882309F49DC1E4
:107AB00096FF9BC18091A1079091A207AA2797FDED
:107AC000A095BA2FBC01CD01A40193010E94A37A15
:107AD0009B01AC0197FF04C02150384F4F4F5F4FBF
:107AE0006BE055954795379527956A95D1F7809125
:107AF0009D01E82EFF2400271127CA01B901A80122
:107B000097010E94A37ADC01CB01809391039093AB
:107B10009203A0939303B0939403B7FF04C08150E2
:107B2000904FAF4FBF4F5C016D013CE0D594C794BF
:107B3000B794A7943A95D1F7A0929103B09292038B
:107B4000C0929303D09294038091B0079091B107B3
:107B5000AA2797FDA095BA2FBC01CD0129813A81B2
:107B60004B815C810E94A37A97FF04C06150784FDB
:107B70008F4F9F4F2BE095958795779567952A9521
:107B8000D1F7A80197010E94A37ADC01CB01809371
:107B9000950390939603A0939703B0939803B7FF30
:107BA00004C08150904FAF4FBF4F9C01AD010CE01E
:107BB00055954795379527950A95D1F720939503C5
:107BC00030939603409397035093980380919103C9
:107BD00090919203909399078093980780919503D1
:107BE0009091960390939D0780939C072A193B09D7
:107BF0004C095D09209395033093960340939703B6
:107C0000509398038091F6079091F707A091F80799
:107C1000B091F907820F931FA41FB51F8093F60739
:107C20009093F707A093F807B093F90780919C0110
:107C30008823F1F457FF04C02F5F3F4F4F4F5F4F32
:107C4000559547953795279580914003909141032D
:107C5000A0914203B0914303821B930BA40BB50B7D
:107C60008093400390934103A0934203B093430356
:107C70002A853B8579010027F7FC0095102F80911C
:107C8000950390919603A0919703B0919803E80E05
:107C9000F91E0A1F1B1FC801B701A40193010E940E
:107CA000A37A9B01AC0197FF04C02150384F4F4F7E
:107CB0005F4FBBE05595479537952795BA95D1F716
:107CC00080919E01A82EBB24CC24DD24CA01B901D9
:107CD000A60195010E94A37ADC01CB018093890360
:107CE00090938A03A0938B03B0938C03B7FF04C0D7
:107CF0008150904FAF4FBF4F3C014D01ACE0959488
:107D0000879477946794AA95D1F7609289037092CB
:107D10008A0380928B0390928C03C801B70129815A
:107D20003A814B815C810E94A37A97FF04C0615025
:107D3000784F8F4F9F4FFBE0959587957795679587
:107D4000FA95D1F7A60195010E94A37ADC01CB0137
:107D500080938D0390938E03A0938F03B093900331
:107D6000B7FF04C08150904FAF4FBF4FAC01BD0172
:107D7000ECE07595679557954795EA95D1F740934F
:107D80008D0350938E0360938F03709390032A8525
:107D90003B8537FF03C0309521953F4F2134310596
:107DA000E4F1D401C30197FE07C0B095A09590956A
:107DB00081959F4FAF4FBF4F81389105A105B10508
:107DC00084F4DB01CA0177FF07C0B095A0959095B8
:107DD00081959F4FAF4FBF4F81389105A105B105E8
:107DE000E4F081E080932C0318C010929D0710925C
:107DF0009C07109299071092980710928D03109289
:107E00008E0310928F0310929003109289031092A8
:107E10008A0310928B0310928C0380918D039091B2
:107E20008E03A0918F03B0919003BC01CD0124E695
:107E300030E040E050E00E94177BE0908903F09032
:107E40008A03E21AF30AF092AF07E092AE0780913C
:107E5000890390918A03A0918B03B0918C03BC019C
:107E6000CD0124E630E040E050E00E94177BDA01CB
:107E7000C90120918D0330918E038C01021B130BDD
:107E80001093A4070093A307809195019091960108
:107E9000A0919701B0919801BC01CD0128E631E095
:107EA00040E050E00E94A37A2091F6073091F70756
:107EB0004091F8075091F9072617370748075907E7
:107EC00064F0261B370B480B590B2093F6073093B1
:107ED000F7074093F8075093F9072091F607309180
:107EE000F7074091F8075091F90757FF0CC0260F8C
:107EF000371F481F591F2093F6073093F707409309
:107F0000F8075093F9076091A1077091A2076E0DD1
:107F10007F1D9B01442737FD4095542F80914403DA
:107F200090914503A0914603B0914703820F931FA0
:107F3000A41FB51F8093440390934503A093460369
:107F4000B093470380910C0390910D03681B790B4C
:107F5000CB01AA2797FDA095BA2F820D931DA41DD2
:107F6000B51D8093480390934903A0934A03B093AF
:107F70004B03C090B301D090B401E090B501F090F4
:107F8000B601C816D906EA06FB06C4F488EA91E6EB
:107F9000A0E0B0E08C199D09AE09BF0980934803A9
:107FA00090934903A0934A03B0934B0380934403F7
:107FB00090934503A0934603B093470322273327AA
:107FC000A9012C193D094E095F0980914803909140
:107FD0004903A0914A03B0914B0382179307A4076A
:107FE000B507B4F4D701C601885A9146A040B04005
:107FF0008093480390934903A0934A03B0934B03A3
:108000008093440390934503A0934603B0934703A2
:108010006091B0077091B107600F711F9B014427F9
:1080200037FD4095542F80914C0390914D03A091C2
:108030004E03B0914F03820F931FA41FB51F80936F
:108040004C0390934D03A0934E03B0934F03809144
:108050000A0390910B03681B790BCB01AA2797FDAC
:10806000A095BA2F2D813E814F815885820F931F95
:10807000A41FB51F8093500390935103A093520304
:10808000B0935303E090B701F090B8010091B901AB
:108090001091BA01E816F9060A071B07C4F488EA2A
:1080A00091E6A0E0B0E08E199F09A00BB10B809380
:1080B000500390935103A0935203B09353038093C2
:1080C0004C0390934D03A0934E03B0934F0322278C
:1080D0003327A9012E193F09400B510B8091500302
:1080E00090915103A0915203B091530382179307CB
:1080F000A407B507B4F4D801C701885A9146A04037
:10810000B0408093500390935103A0935203B093D7
:10811000530380934C0390934D03A0934E03B0936D
:108120004F038091400390914103A0914203B0918D
:1081300043038093540390935503A0935603B09345
:1081400057038091500390915103A0915203B09135
:1081500053038093700390937103A0937203B093C1
:1081600073038091480390914903A0914A03B09111
:108170004B038093680390936903A0936A03B093C1
:108180006B0380914C0390914D03A0914E03B091ED
:108190004F0380936C0390936D03A0936E03B09391
:1081A0006F038091440390914503A0914603B091E1
:1081B00047038093640390936503A0936603B09391
:1081C000670380911B0190911C0197FD079633E096
:1081D000959587953A95E1F79093B1078093B0070D
:1081E0008091190190911A0197FD079623E09595CA
:1081F00087952A95E1F79093A2078093A107809134
:1082000002018A3009F062C08091480290914902CF
:10821000835F934034F088E592E09093B1078093B8
:10822000B00780914802909149028A5F934034F0F0
:1082300080E293E09093B1078093B0078091480269
:10824000909149020F9734F488EA9DEF9093B1071B
:108250008093B0078091480290914902079734F4C7
:1082600080EE9CEF9093B1078093B0078091460217
:1082700090914702835F934034F088E592E09093B9
:10828000A2078093A10780914602909147028A5FDE
:10829000934034F080E293E09093A2078093A1078B
:1082A00080914602909147020F9734F488EA9DEF3F
:1082B0009093A2078093A107809146029091470274
:1082C00007970CF067C080EE9CEF60C08091480279
:1082D00090914902815D974034F080EB94E0909357
:1082E000B1078093B0078091480290914902805E67
:1082F000974034F080E496E09093B1078093B00704
:1083000080914802909149020F9734F480E59BEFE9
:108310009093B1078093B0078091480290914902F1
:10832000079734F480EC99EF9093B1078093B007EE
:108330008091460290914702815D974034F080EB36
:1083400094E09093A2078093A107809146029091B8
:108350004702805E974034F080E496E09093A20755
:108360008093A10780914602909147020F9734F4C1
:1083700080E59BEF9093A2078093A107809146022E
:1083800090914702079734F480EC99EF9093A207FD
:108390008093A107E091A801EE2309F4B7C04091B2
:1083A0001B0150911C018091990390919A03481BE5
:1083B000590B5093A00340939F0320911B013091D0
:1083C0001C01280F391F37FF02C02F5F3F4F359523
:1083D000279530939A0320939903413851051CF057
:1083E00080E890E005C040585F4F34F480E89FEF8C
:1083F0009093A00380939F038E2F9927A0919F03B2
:10840000B091A003A89FA001A99F500DB89F500D47
:10841000112457FF02C0415F5F4F14E05595479507
:108420001A95E1F78091B0079091B107840F951FDD
:108430009093B1078093B0076091190170911A0170
:1084400080919B0390919C03681B790B70939E0312
:1084500060939D034091190150911A01480F591FD3
:1084600057FF02C04F5F5F4F5595479550939C0350
:1084700040939B03613871051CF080E890E005C0D3
:1084800060587F4F34F480E89FEF90939E03809371
:108490009D032E2F332780919D0390919E03829FF1
:1084A000B001839F700D929F700D1124AB0177FF77
:1084B00002C0415F5F4FE4E055954795EA95E1F7CB
:1084C0008091A1079091A207840F951F9093A20716
:1084D0008093A107A29FC001A39F900DB29F900D12
:1084E00011249C0180911B0190911C01820F931F0C
:1084F00090931C0180931B018091190190911A01A6
:10850000860F971F90931A01809319010091B3076A
:108510001091B40780919807909199071016110651
:108520005CF59C0197FF04C022273327281B390BD9
:10853000C901AA2797FDA095BA2F20919C01332746
:1085400044275527BC01CD010E94A37A9B01AC01B1
:1085500097FF04C0215C3F4F4F4F5F4F76E055952A
:108560004795379527957A95D1F78091AE079091E9
:10857000AF07820F931F27C097FF03C09095819587
:108580009F4FAA2797FDA095BA2F20919C013327D2
:1085900044275527BC01CD010E94A37A9B01AC0161
:1085A00097FF04C0215C3F4F4F4F5F4F66E05595EA
:1085B0004795379527956A95D1F78091AE079091A9
:1085C000AF07821B930B9093AF078093AE07E090A9
:1085D000BB07F090BC0780919C0790919D071E14EB
:1085E0001F045CF59C0197FF04C022273327281B3A
:1085F000390BC901AA2797FDA095BA2F20919C019C
:10860000332744275527BC01CD010E94A37A9B0143
:10861000AC0197FF04C0215C3F4F4F4F5F4F96E086
:1086200055954795379527959A95D1F78091A3074A
:108630009091A407820F931F27C097FF03C09095C6
:1086400081959F4FAA2797FDA095BA2F20919C0155
:10865000332744275527BC01CD010E94A37A9B01F3
:10866000AC0197FF04C0215C3F4F4F4F5F4F86E046
:1086700055954795379527958A95D1F78091A3070A
:108680009091A407821B930B9093A4078093A30758
:108690008091150687FF44C09985992309F040C051
:1086A000809106038823E1F5A1E0EA16A1E0FA062D
:1086B0004CF08091B0079091B1078E0D9F1D8050B6
:1086C00091400DC0B0E0EB16BFEFFB0664F4809163
:1086D000B0079091B1078E0D9F1D80509F4F9093D2
:1086E000B1078093B007E1E001301E074CF08091A4
:1086F000A1079091A207800F911F805091400CC05C
:10870000FFEF00301F0764F48091A1079091A2074A
:10871000800F911F80509F4F9093A2078093A107D5
:10872000A1E2B3E06DE076E057E0FB018191BF018B
:10873000E82FFF27EE0FFF1FE05DF84F0190F0815B
:10874000E02DE259FF4FEF3FF10521F01CF0EFEF74
:10875000F0E004C0F7FF02C0E0E0F0E04C91242F0D
:108760003327E217F307B1F0CF01821B930B97FD7C
:10877000079613E0959587951A95E1F7242F280F12
:108780002C93822F9927E817F90714F4215001C080
:108790002F5F2C935150119657FFC7CFE2E1C55F71
:1087A0000C944E7B80911703882301F58091E80299
:1087B0008C7F8093E802AEE4B4E0EFECF6E09BE05F
:1087C00080910402882309F48C938D918183128215
:1087D0009150389697FFF4CF80910402882359F086
:1087E0008091040281508093040205C08091E802C8
:1087F00081608093E80210926F0210927102809162
:108800006C028E7F80936C0285EA8093BC00089591
:1088100080911706883F38F0EFEFF0E0E81BF10990
:10882000EF5DFC4F80818093AE018091AE01882383
:1088300029F0843618F084E68093AE018091190601
:10884000883F38F0EFEFF0E0E81BF109EF5DFC4FF7
:1088500080818093AC018091AC01882329F084361B
:1088600018F084E68093AC0180912606883F38F0AA
:10887000EFEFF0E0E81BF109EF5DFC4F80818093A2
:10888000A7018091A7018B3010F48AE002C08F3FCE
:1088900011F48093A70180915106883F38F0EFEFE3
:1088A000F0E0E81BF109EF5DFC4F80818093C70782
:1088B0008091C707823010F481E002C08F3F11F42D
:1088C0008093C70780915306883F38F0EFEFF0E0C0
:1088D000E81BF109EF5DFC4F80818093ED078091EB
:1088E000ED07823010F481E002C08F3F11F48093D5
:1088F000ED0780913E06883F38F0EFEFF0E0E81B8F
:10890000F109EF5DFC4F80818093C40780913F06A1
:10891000883F38F0EFEFF0E0E81BF109EF5DFC4F26
:10892000808180939E0780914006883F38F0EFEF6A
:10893000F0E0E81BF109EF5DFC4F80818093CC07EC
:1089400080911806883F38F0EFEFF0E0E81BF1095E
:10895000EF5DFC4F80818093AD0180911B06883FC5
:1089600038F0EFEFF0E0E81BF109EF5DFC4F80819C
:108970008093AB0180911D06883F38F0EFEFF0E067
:10898000E81BF109EF5DFC4F80818093A901809184
:108990002506883F38F0EFEFF0E0E81BF109EF5DC6
:1089A000FC4F80818093AA0180912706883F38F090
:1089B000EFEFF0E0E81BF109EF5DFC4F8081809361
:1089C000A60180912806883F38F0EFEFF0E0E81B21
:1089D000F109EF5DFC4F80818093A8018091290609
:1089E000883F38F0EFEFF0E0E81BF109EF5DFC4F56
:1089F00080818093A50180912A06883F38F0EFEFAF
:108A0000F0E0E81BF109EF5DFC4F80818093A40149
:108A100080913006883F38F0EFEFF0E0E81BF10975
:108A2000EF5DFC4F80818093A20180913106883FE9
:108A300038F0EFEFF0E0E81BF109EF5DFC4F8081CB
:108A40008093010380913206883F38F0EFEFF0E029
:108A5000E81BF109EF5DFC4F80818093000380915A
:108A60003306883F38F0EFEFF0E0E81BF109EF5DE7
:108A7000FC4F80818093FF0280913406883F38F05C
:108A8000EFEFF0E0E81BF109EF5DFC4F8081809390
:108A9000FE0280914C06883F38F0EFEFF0E0E81BD3
:108AA000F109EF5DFC4F80818093FD0280914D06BE
:108AB000883F38F0EFEFF0E0E81BF109EF5DFC4F85
:108AC00080818093FC0280914E06883F38F0EFEF62
:108AD000F0E0E81BF109EF5DFC4F80818093FB0221
:108AE00080914F06883F38F0EFEFF0E0E81BF10986
:108AF000EF5DFC4F80818093FA0280913506883FBC
:108B000038F0EFEFF0E0E81BF109EF5DFC4F8081FA
:108B10008093A10180913906883F38F0EFEFF0E0B3
:108B2000E81BF109EF5DFC4F80818093A0018091EB
:108B30004106883F38F0EFEFF0E0E81BF109EF5D08
:108B4000FC4F808180939F0180914406883F38F0DC
:108B5000EFEFF0E0E81BF109EF5DFC4F80818093BF
:108B60009E0180914506883F38F0EFEFF0E0E81B6A
:108B7000F109EF5DFC4F808180939D018091460655
:108B8000883F38F0EFEFF0E0E81BF109EF5DFC4FB4
:108B9000808180939C0180914B06883F38F0EFEFF5
:108BA000F0E0E81BF109EF5DFC4F808180939B01B1
:108BB00080916606883F38F0EFEFF0E0E81BF1099E
:108BC000EF5DFC4F80818093FD078091A201282FEB
:108BD00033272F5F3F4F8CE398E2B9010E94E27A7E
:108BE0007093B2016093B10180910103833380F0EF
:108BF00080910003282F33272F5F3F4F8CE398E2AB
:108C0000B9010E94E27A7093B0016093AF0104C091
:108C10007093B0016093AF01809156068093AD07C9
:108C20008091CD07882311F48093AD0780912306AE
:108C30008093EE07809122068093B5079091680695
:108C4000933320F181E08093F902983F58F0EFEFE1
:108C5000F0E0E91BF109EF5DFC4F8081823310F4F5
:108C60001092F90280913B0890913C0897FF08C050
:108C70008091F902882321F080914904806803C023
:108C8000809149048F778093490402C01092F902C1
:108C900080913B0890913C0897FF1DC0809117037D
:108CA0008823C9F08091F9028823A9F080910801F6
:108CB000909109018F5F9F4F71F488E99AE3909337
:108CC00024028093230280E094EA90930901809328
:108CD00008011092F9028091F902882339F08091FD
:108CE0009E01823D18F4825E80939E010895A5E363
:108CF000B0E0EDE7F6E40C94327B0E948F3B3091BC
:108D000002013C3010F4299A01C0299840911803BF
:108D10005091190359A348A38091B50799270A9642
:108D20004817590714F499A388A380912003843627
:108D300008F05CC08091BD039091BE03009731F0B4
:108D400001979093BE038093BD0307C01092170351
:108D50008091E8028F7E8093E8023A3011F034313E
:108D600010F0289A01C028988091E9029091EA02B7
:108D7000895E9340C0F180912D06682F772779A3F3
:108D800068A38091E80280618093E80280910906DF
:108D9000A82FBB27AA0FBB1FFD01EC59F84F11826A
:108DA000108280910A06282F3327220F331FC90112
:108DB0008C59984FFC0111821082A05DB84F11961A
:108DC0001C921E92205D384FD90111961C921E9262
:108DD00080910C06E82FFF27EE0FFF1FE05DF84F94
:108DE00011821082A2C2109217039FC280912003A9
:108DF0008D3808F49AC28091E8028F7E8093E80251
:108E000090912E0682E3989FC00111249093BE0397
:108E10008093BD03E8A1F9A1B9978CF08091170365
:108E2000882369F08091E9029091EA02FFEF8F3F79
:108E30009F0729F001969093EA028093E9028091BE
:108E4000E9029091EA028F3F910509F038F51092FE
:108E50003C0310923D0310923E0310923F03109288
:108E600038031092390310923A0310923B03109288
:108E7000A9031092AA031092AB031092AC031092B4
:108E800040031092410310924203109243038A3F21
:108E9000910549F481E08093C30305C08091E80205
:108EA00082608093E80280910B06E82FFF27EE0F87
:108EB000FF1FE05DF84F80819181813591050CF4B1
:108EC00041C120911703222309F03CC180910C0677
:108ED000E82FFF27EE0FFF1FE05DF84F80819181A3
:108EE0008C3491050CF406C18091BF038F5F809391
:108EF000BF03893C08F426C13C3010F4299801C016
:108F0000299A109217031092BF031092EA0210924E
:108F1000E90230910906E32FFF27EE0FFF1FE05D06
:108F2000F84F8081918187349105B4F480910A06CD
:108F3000E82FFF27EE0FFF1FE05DF84F8081918142
:108F40000190F081E02DF7FF03C0F095E195FF4F10
:108F5000E734F1050CF478C041E020910A06A22F15
:108F6000BB27AA0FBB1FA05DB84F8D919C91119795
:108F70008734910544F0E32FFF27EE0FFF1FE05DDC
:108F8000F84F808191818D919C918734910574F087
:108F900080910906E82FFF27EE0FFF1FE05DF84FD5
:108FA00080819181873491050CF042E0E22FFF2708
:108FB000EE0FFF1FE05DF84F8081918186349105AF
:108FC00074F480910906E82FFF27EE0FFF1FE05D84
:108FD000F84F80819181873491050CF043E0E22FB6
:108FE000FF27EE0FFF1FE05DF84F808191818A5BC4
:108FF0009F4F74F480910906E82FFF27EE0FFF1FA3
:10900000E05DF84F80819181873491050CF044E058
:10901000E22FFF27EE0FFF1FE05DF84F8081918167
:109020008A5B9F4F74F480910906E82FFF27EE0FAB
:10903000FF1FE05DF84F80819181863491050CF42B
:1090400045E0842F0E94132E80910A06E82FFF2707
:10905000EE0FFF1FE05DF84F808191810190F0815C
:10906000E02DF7FF03C0F095E195FF4F7E97BCF42C
:1090700080910906E82FFF27EE0FFF1FE05DF84FF4
:10908000808191818A5B9F4F54F481E080936404D6
:1090900088EE93E0909324028093230253C00E94B1
:1090A0000D2F0E94C02D80E00E94490780912F065D
:1090B0000E9456778091150680FF10C080911301A1
:1090C00090911401875B934038F480911301909143
:1090D00014018E5E924010F40E94B61A1092210282
:1090E00080E00E94E13881E08093C20380932102F6
:1090F000579A1FC080819181855B9F4F0CF58091AD
:10910000BF038F5F8093BF03893CE0F03C3010F4D5
:10911000299801C0299A109217031092BF03109248
:10912000EA021092E90281E00E94E13881E0809336
:10913000C2030E940D2F68E770E00E941F3802C032
:109140002093BF0380910B06E82FFF27EE0FFF1F30
:10915000E05DF84F808191818B5A9F4F0CF0E5C004
:1091600020911703E0910C06222309F0C2C0FF27CB
:10917000EE0FFF1FE05DF84F80819181855B9F4F6F
:109180000CF0B4C08091C0038F5F8093C003893C12
:1091900008F4CBC02093C00380914904882309F0D0
:1091A0009EC08091C203882309F499C081E090E0B9
:1091B0009093EA028093E90281E080931703109272
:1091C000A9031092AA031092AB031092AC03109261
:1091D0004003109241031092420310924303809186
:1091E0002406E82EFF24002711278091EA0790919A
:1091F000EB079C01442737FD4095542FC801B70168
:109200000E94A37ADC01CB01809350039093510319
:10921000A0935203B09353038091FA079091FB07F8
:109220009C01442737FD4095542FC801B7010E9487
:10923000A37ADC01CB018093480390934903A09368
:109240004A03B0934B038091700390917103A091F6
:109250007203B091730380934C0390934D03A093DA
:109260004E03B0934F038091680390916903A091DE
:109270006A03B0916B038093440390934503A093DA
:109280004603B093470310923C0310923D031092A3
:109290003E0310923F03109238031092390310924C
:1092A0003A0310923B038091E80288608093E802C1
:1092B000909167068FE0989F90011124809132036E
:1092C00090913303820F931F68E671E00E94E27A67
:1092D00097FD0196959587958093740326C08CED34
:1092E00095E090932402809323021FC02093C00333
:1092F0001CC0FF27EE0FFF1FE05DF84F80819181BA
:109300008C34910584F08091C1038F5F8093C103F9
:10931000893C58F0109217031092C1031092EA0290
:109320001092E90202C01092C10380919301815012
:1093300080939301809193018F3F21F08091E80207
:1093400084FF25C40E940844B0900103E0910906FF
:109350004091CC035091CD0322E32B1508F05AC065
:109360009A01220F331F240F351FFF27EE0FFF1F17
:10937000E05DF84F8091FF02482F55278081918151
:10938000849FB001859F700D949F700D1124260F4E
:10939000371F8091ED029091EE02281B390B37FFA9
:1093A00002C02D5F3F4F3595279535952795309312
:1093B000CD032093CC038091CE039091CF039C01E9
:1093C000220F331F280F391F80910A06E82FFF272D
:1093D000EE0FFF1FE05DF84F80819181849FD001E7
:1093E000859FB00D949FB00D11242A0F3B1F8091D3
:1093F000EB029091EC02281B390B37FF02C02D5F66
:109400003F4F35952795359527953093CF0320937A
:10941000CE0357C09A01220F331F240F351FFF2799
:10942000EE0FFF1FE05DF84F80911F06482F552774
:1094300080819181849FF001859FF00D949FF00DB4
:1094400011242E0F3F1F37FF02C02D5F3F4FB90180
:1094500075956795759567957093CD036093CC036B
:109460008091CE039091CF039C01220F331F280FD0
:10947000391F80910A06E82FFF27EE0FFF1FE05DDE
:10948000F84F80819181849FD001859FB00D949F7A
:10949000B00D11242A0F3B1F37FF02C02D5F3F4F35
:1094A000C90195958795959587959093CF0380935E
:1094B000CE037093EE026093ED029093EC028093E2
:1094C000EB028091CD07882309F442C02091CC03A0
:1094D0003091CD033093EE022093ED024091CE0304
:1094E0005091CF035093EC024093EB028091090618
:1094F000E82FFF27EE0FFF1FEC59F84F8091200651
:10950000682F772780819181869FF001879FF00DDA
:10951000969FF00D11242E0F3F1F3093CD03209303
:10952000CC0380910A06E82FFF27EE0FFF1FEC59AE
:10953000F84F80819181869F9001879F300D969F83
:10954000300D1124420F531F5093CF034093CE038D
:109550009E012F5F3F4F8FE1E2ECF1E0D9010190D6
:109560000D928A95E1F78091F9024091CC035091D8
:10957000CD03882309F44BC0CA0157FD0396DC01D3
:10958000B595A795B595A7958091CE039091CF03FA
:1095900097FD0396FC01F595E795F595E795809184
:1095A000EB01682F772767FD70956A9F90016B9F8D
:1095B000300D7A9F300D112480910504482F5527D6
:1095C00047FD50954E9FC0014F9F900D5E9F900D9F
:1095D0001124280F391F37FF02C0295F3F4F03E0D6
:1095E000359527950A95E1F730931F0320931E03C5
:1095F0006E9F90016F9F300D7E9F300D11244A9F0A
:10960000C0014B9F900D5A9F900D112448C080912E
:109610006706682F7727DE01A60FB71FFD01978128
:109620009093EB01620F731FDB018C918093050413
:10963000A92FBB27A7FDB095A49F9001A59F300D32
:10964000B49F300D1124E82FFF27E7FDF0956091BE
:10965000CE037091CF03E69FC001E79F900DF69F68
:10966000900D1124280F391F37FF02C0295F3F4F8B
:1096700013E0359527951A95E1F730931F03209352
:109680001E03A69F9001A79F300DB69F300D112499
:10969000E49FC001E59F900DF49F900D1124281BBD
:1096A000390B37FF02C0295F3F4FF3E0359527950F
:1096B000FA95E1F730931D0320931C0380910C066B
:1096C000E82FFF27EE0FFF1FE05DF84F80819181AB
:1096D000909581959F4F90931B0380931A0383303D
:1096E000910514F0029705C0BFEF8E3F9B0734F43D
:1096F000029690931B0380931A0304C010921B03DD
:1097000010921A0380910104909102042091FD03AC
:109710003091FE03820F931FC0901E03D0901F0351
:10972000C81AD90AD0921F03C0921E038091FF036A
:10973000909100042091FB033091FC03820F931F52
:1097400000911C0310911D03081B190B10931D039E
:1097500000931C0380910B06E82FFF27EE0FFF1FDD
:10976000E05DF84FE080F180E8E7F0E0EE0EFF1EEC
:10977000F0921903E09218038091A7019927AA2774
:1097800097FDA095BA2FBC01CD010E94177ADC018C
:10979000CB0120E030E040E251E4BC01CD010E9469
:1097A0008579DC01CB01BC01CD010E94E979DC01A6
:1097B000CB018093F4078091A6018093CD0780911F
:1097C000A5019927AA2797FDA095BA2FBC01CD0125
:1097D0000E94177ADC01CB0120E030E040E251E446
:1097E000BC01CD010E948579DC01CB01BC01CD011A
:1097F0000E94E979DC01CB018093A8078091A40144
:109800008093BD078091700480FF5CC08091FD074C
:10981000813808F457C080916904282F332727FD29
:10982000309580911F06482F5527249FC001259F02
:10983000900D349F900D1124C80ED91ED0921F0395
:10984000C0921E0380916A04992787FD9095849F9A
:109850009001859F300D949F300D1124020F131F2E
:1098600010931D0300931C0380916B04282F332752
:1098700027FD309580911A0390911B03820F931F4F
:1098800090931B0380931A0380916D04282F332734
:1098900027FD309580911A069927289FA001299FBE
:1098A000500D389F500D112450939A014093990107
:1098B00080916C0499278E159F0524F490931903C9
:1098C00080931803809118039091190397FF04C0A7
:1098D00010921903109218038091150682FD03C09F
:1098E00052E35B1510F41092CD0740911E03509186
:1098F0001F03CA0157FD03969C01359527953595A1
:10990000279537FF03C0309521953F4F8091F10295
:109910009091F20282179307B4F4CA0157FF03C073
:10992000909581959F4F97FD039695958795959571
:1099300087959093F2028093F1028536910544F069
:1099400084E690E001C001979093F2028093F102C7
:1099500040911C0350911D03CA0157FD03969C01C1
:10996000359527953595279537FF03C03095219577
:109970003F4F8091EF029091F00282179307B4F469
:10998000CA0157FF03C0909581959F4F97FD03969D
:1099900095958795959587959093F0028093EF0222
:1099A0008536910544F084E690E001C001979093DC
:1099B000F0028093EF028091E80284FF08C01092C9
:1099C000F2021092F1021092F0021092EF02509106
:1099D0000A06E52FFF27EE0FFF1FE05DF84F4091CD
:1099E0004206242F3327808191812817390744F4B8
:1099F0008091690682FF04C081E08093050313C053
:109A0000E52FFF27EE0FFF1FE05DF84F842F99270A
:109A100020914306821B9109208131812817390743
:109A200014F41092050340910A06E42FFF27EE0F6D
:109A3000FF1FE05DF84F50914206852F992722279E
:109A40003327281B390B808191818217930744F4B7
:109A50008091690683FF04C081E08093040316C0EF
:109A600080910403882391F0E42FFF27EE0FFF1F5E
:109A7000E05DF84F809143069927851B910920816D
:109A800031818217930714F4109204035091090650
:109A9000E52FFF27EE0FFF1FE05DF84F40914206D4
:109AA000242F3327808191812817390744F480912E
:109AB000690680FF04C081E08093020317C0809193
:109AC0000203882399F0E52FFF27EE0FFF1FE05DCB
:109AD000F84F842F992720914306821B91092081FA
:109AE00031812817390714F41092020340910906B6
:109AF000E42FFF27EE0FFF1FE05DF84F5091420665
:109B0000852F992722273327281B390B80819181A4
:109B10008217930744F48091690681FF04C081E0B5
:109B20008093030316C080910303882391F0E42FF0
:109B3000FF27EE0FFF1FE05DF84F80914306992746
:109B4000851B9109208131818217930714F41092AB
:109B5000030380910503882319F480910403811184
:109B600081E08093060380910203882321F4809191
:109B70000303882351F081E08093070310920603CA
:109B8000109205031092040302C080930703809192
:109B90000603882321F480910703882369F08091CC
:109BA0004106992768A179A18617970714F499A30C
:109BB00088A381E080932C038091E80284FF1AC07F
:109BC00010921B0310921A0310921F0310921E038F
:109BD00010921D0310921C039AE59093F40788E7F6
:109BE0008093CD079093A8078093BD07109206033A
:109BF000109207038091C0079091C107A091C207FE
:109C0000B091C307209170033091710340917203AA
:109C100050917303820F931FA41FB51F8093C00739
:109C20009093C107A093C207B093C3078091C80760
:109C30009091C907A091CA07B091CB072091680302
:109C40003091690340916A0350916B03820F931F17
:109C5000A41FB51F8093C8079093C907A093CA0794
:109C6000B093CB078091B7079091B807A091B9073F
:109C7000B091BA0720916C0330916D0340916E034F
:109C800050916F032AA33BA34CA35DA3820F931FA4
:109C9000A41FB51F8093B7079093B807A093B90787
:109CA000B093BA078091A9079091AA07A091AB073A
:109CB000B091AC07409164035091650360916603D5
:109CC000709167034EA35FA368A779A7840F951FC0
:109CD000A61FB71F8093A9079093AA07A093AB076D
:109CE000B093AC07509107035AA7552349F48091CC
:109CF0000603882329F48091CD07882309F080C0CA
:109D00001092600310926103109262031092630339
:109D100010925C0310925D0310925E0310925F0339
:109D20001092C0071092C1071092C2071092C30789
:109D30001092C8071092C9071092CA071092CB0759
:109D40001092B7071092B8071092B9071092BA078D
:109D50001092A9071092AA071092AB071092AC07B5
:109D60001092700310927103109272031092730399
:109D7000109268031092690310926A0310926B03A9
:109D800010925003109251031092520310925303F9
:109D9000109248031092490310924A0310924B0309
:109DA0001092400310924103109242031092430319
:109DB00010925403109255031092560310925703B9
:109DC00010924C0310924D0310924E0310924F03C9
:109DD00010924403109245031092460310924703D9
:109DE000109235021092340210920B0310920A0363
:109DF00010920D0310920C036AA5662309F003C2AA
:109E000080910603882309F0FEC18091FA059091A4
:109E1000FB05815092402CF480911703882309F4AC
:109E2000F2C18091CD07882309F4EDC190906808B4
:109E3000A09024068091EA079091EB079BAB8AAB38
:109E4000A091FA07B091FB07BDABACAB609170037A
:109E50007091710380917203909173032090680355
:109E60003090690340906A0350906B03BFEF9B16DC
:109E700009F4D7C0BB24CC24DD24A60195010E949F
:109E8000177B79018A01EAA9FBA9CF01AA2797FDCF
:109E9000A095BA2FE81AF90A0A0B1B0BC201B101EF
:109EA000A60195010E94177B59016A012CA93DA9C1
:109EB000C901AA2797FDA095BA2FA81AB90ACA0AFC
:109EC000DB0A292C332427FC3094432C532CC80163
:109ED000B701A20191010E94A37A97FF04C06150CB
:109EE0007E4F8F4F9F4F3B014C0109E09594879423
:109EF000779467940A95D1F7C601B501A201910143
:109F00000E94A37A97FF04C061507E4F8F4F9F4FEE
:109F10005B016C0119E0D594C794B794A7941A9586
:109F2000D1F78091F1029091F202813491053CF4D5
:109F30008091EF029091F00281349105D4F0D40128
:109F4000C30197FE03C00196A11DB11D3C014D0147
:109F50009594879477946794D601C501D7FE03C082
:109F60000196A11DB11D5C016D01D594C794B794F4
:109F7000A79480910C06E82FFF27EE0FFF1FE05DEE
:109F8000F84F808191810190F081E02DF7FF03C0AF
:109F9000F095E195FF4F7A97A4F0C401B30123E057
:109FA00030E040E050E00E94177B39014A01C601D1
:109FB000B50123E030E040E050E00E94177B5901FA
:109FC0006A0180916A08282F332727FD3095432F97
:109FD000532F261537054805590514F439014A0150
:109FE000992787FD9095909581959F4FAA2797FD7A
:109FF000A095BA2F681679068A069B0614F43C01D0
:10A000004D012A153B054C055D0514F459016A0103
:10A01000A816B906CA06DB060CF0CDC05C016D01BE
:10A02000CAC0EA2CFF2400271127A80197010E942B
:10A03000177B39014A014AA95BA9CA01AA2797FDE2
:10A04000A095BA2F681A790A8A0A9B0AC201B1013F
:10A05000A80197010E94177B59016A016CA97DA98B
:10A06000CB01AA2797FDA095BA2FA81AB90ACA0A48
:10A07000DB0AD401C30197FE03C00F96A11DB11DD9
:10A080003C014D01F4E09594879477946794FA9598
:10A09000D1F7D601C501D7FE03C00F96A11DB11D92
:10A0A0005C016D01E4E0D594C794B794A794EA9558
:10A0B000D1F78091F1029091F202813491053CF444
:10A0C0008091EF029091F00281349105A4F0C401D7
:10A0D000B30123E030E040E050E00E94177B3901FB
:10A0E0004A01C601B50123E030E040E050E00E94A3
:10A0F000177B59016A0180910C06E82FFF27EE0FAC
:10A10000FF1FE05DF84F808191810190F081E02D8B
:10A11000F7FF03C0F095E195FF4F7A97A4F0C401D3
:10A12000B30123E030E040E050E00E94177B3901AA
:10A130004A01C601B50123E030E040E050E00E9452
:10A14000177B59016A0171E2671671048104910459
:10A150002CF070E2672E712C812C912C80EE681609
:10A160008FEF78068FEF88068FEF980644F460EE45
:10A17000662E6FEF762E6FEF862E6FEF962E91E2A2
:10A18000A916B104C104D1042CF050E2A52EB12CC3
:10A19000C12CD12CA0EEAA16AFEFBA06AFEFCA06BB
:10A1A000AFEFDA0644F440EEA42E4FEFB42E4FEF9B
:10A1B000C42E4FEFD42E8091500390915103A09163
:10A1C0005203B091530386199709A809B9098093DE
:10A1D000500390935103A0935203B0935303809183
:10A1E000480390914903A0914A03B0914B038A1907
:10A1F0009B09AC09BD098093480390934903A09340
:10A200004A03B0934B0380913402909135028F3F03
:10A21000910509F008F4C9C5BAA5BB2309F053C5D7
:10A2200080910603882309F04EC580912C03882372
:10A2300009F049C5E0914A06EBA7EE2309F443C5AE
:10A240008091CD07882309F43EC58091C007909185
:10A25000C107A091C207B091C307B7FF04C08150E6
:10A260009F4FAF4FBF4FE92EFA2E0B2F112707FD3F
:10A270001A95E092C007F092C1070093C2071093AD
:10A28000C3078091C8079091C907A091CA07B091F0
:10A29000CB07B7FF04C081509F4FAF4FBF4F892FEF
:10A2A0009A2FAB2FBB27A7FDBA958CA79DA7AEA76A
:10A2B000BFA78093C8079093C907A093CA07B0931C
:10A2C000CB0780912406A82EBB24CC24DD2420912A
:10A2D0006003309161034091620350916303C601B2
:10A2E000B5010E94A37A97FF04C061507F4F8F4F42
:10A2F0009F4F672E782E892E992487FC9A9460921E
:10A3000060037092610380926203909263032091D4
:10A310005C0330915D0340915E0350915F03C60181
:10A32000B5010E94A37A97FF04C061507F4F8F4F01
:10A330009F4F272E382E492E552447FC5A942092A1
:10A340005C0330925D0340925E0350925F03809104
:10A35000580390915903A0915A03B0915B03B7FF42
:10A3600004C081509F4FAF4FBF4F892F9A2FAB2F03
:10A37000BB27A7FDBA958093580390935903A093E8
:10A380005A03B0935B03D801C70186199709A8093E
:10A39000B9098093B5039093B603A093B703B09324
:10A3A000B80320914906E22EFF2400271127BC01A3
:10A3B000CD01A80197010E94177B59016A012093E2
:10A3C000C4033093C5034093C6035093C7038CA5C1
:10A3D0009DA5AEA5BFA582199309A409B5098093CF
:10A3E000B9039093BA03A093BB03B093BC03BC0121
:10A3F000CD01A80197010E94177B2093C8033093D9
:10A40000C9034093CA035093CB03D601C501D7FEBD
:10A4100004C081509F4FAF4FBF4F892F9A2FAB2F52
:10A42000BB27A7FDBA9590930B0380930A0357FFB0
:10A4300004C021503F4F4F4F5F4FBB2757FDBA9588
:10A44000A52F942F832F90930D0380930C0380915D
:10A45000F1029091F20281349105DCF48091EF02D7
:10A460009091F00281349105A4F480910C06E82FBC
:10A47000FF27EE0FFF1FE05DF84F80819181019073
:10A48000F081E02DF7FF03C0F095E195FF4F7A973B
:10A49000E4F0809168088F3FC1F480910A039091A5
:10A4A0000B0397FD01969595879590930B038093E9
:10A4B0000A0380910C0390910D0397FD01969595E9
:10A4C000879590930D0380930C038091B70790912B
:10A4D000B807A091B907B091BA07B7FF04C081507F
:10A4E0009F4FAF4FBF4F892F9A2FAB2FBB27A7FD91
:10A4F000BA958093B7079093B807A093B907B09324
:10A50000BA078091A9079091AA07A091AB07B091D3
:10A51000AC07B7FF04C081509F4FAF4FBF4F892F8B
:10A520009A2FAB2FBB27A7FDBA958093A9079093CD
:10A53000AA07A093AB07B093AC07809170039091EA
:10A540007103A0917203B09173032AA13BA14CA1A6
:10A550005DA1281B390B4A0B5B0B2093AD03309395
:10A56000AE034093AF035093B00380916803909182
:10A570006903A0916A03B0916B03EEA0FFA008A548
:10A5800019A5E81AF90A0A0B1B0BE092B103F09225
:10A59000B2030093B3031093B4032093B503309335
:10A5A000B6034093B7035093B803E092B903F09217
:10A5B000BA030093BB031093BC0380914C039091AA
:10A5C0004D03A0914E03B0914F03821B930BA40B3C
:10A5D000B50B80934C0390934D03A0934E03B0931F
:10A5E0004F038091440390914503A0914603B0919D
:10A5F00047038E199F09A00BB10B809344039093DE
:10A600004503A0934603B0934703FBA5FF23E1F066
:10A6100020912A0330912B03213831054CF0809191
:10A62000810390918203019690938203809381032A
:10A6300020583F4F4CF48091810390918203019701
:10A64000909382038093810310922B0310922A032C
:10A6500081E090E09093D1038093D003A090B50364
:10A66000B090B603C090B703D090B803D601C5012F
:10A67000D7FE07C088279927DC018A199B09AC09F6
:10A68000BD0981509240A040B04034F084E090E099
:10A690009093D1038093D0038091D6039091D703F8
:10A6A000A091D803B091D9032091C0073091C10780
:10A6B0004091C2075091C307821B930BA40BB50BAB
:10A6C000815E914BAF4FBF4F8F539C49A040B0402C
:10A6D00028F08091690889310CF4FFC071E0A71659
:10A6E00070E1B70670E0C70670E0D7060CF473C0DF
:10A6F0008091D203882309F46AC0D601C501D7FE30
:10A7000007C088279927DC018A199B09AC09BD0974
:10A710009C01AD01B7FF04C021503E4F4F4F5F4F2A
:10A7200009E055954795379527950A95D1F780917A
:10A73000D0039091D103820F931F9093D103809304
:10A74000D003D601C501D7FE03C00796A11DB11DD8
:10A7500013E0B595A795979587951A95D1F78093AE
:10A76000C4039093C503A093C603B093C70389584D
:10A770009341A040B04064F088E893E1A0E0B0E0ED
:10A780008093C4039093C503A093C603B093C703FB
:10A790002091C4033091C5034091C6035091C70373
:10A7A00057FF04C021503F4F4F4F5F4F232F342F8F
:10A7B000452F552747FD5A9580910A0390910B0329
:10A7C000820F931F90930B0380930A0306C081E0CE
:10A7D0008093D20302C01092D203F0E0AF16F0EFE4
:10A7E000BF06FFEFCF06FFEFDF060CF073C08091CE
:10A7F000D303882309F46AC0D601C501D7FE07C078
:10A8000088279927DC018A199B09AC09BD099C019D
:10A81000AD01B7FF04C021503E4F4F4F5F4FF9E0ED
:10A820005595479537952795FA95D1F78091D0039F
:10A830009091D103820F931F9093D1038093D00303
:10A84000D601C501D7FE03C00796A11DB11DE3E0E7
:10A85000B595A79597958795EA95D1F78093C40309
:10A860009093C503A093C603B093C70388579C4E2B
:10A87000AF4FBF4F64F488E79CEEAFEFBFEF80931C
:10A88000C4039093C503A093C603B093C70320915C
:10A89000C4033091C5034091C6035091C70357FFCD
:10A8A00004C021503F4F4F4F5F4F232F342F452F70
:10A8B000552747FD5A9580910A0390910B03820F0B
:10A8C000931F90930B0380930A0311C081E0809340
:10A8D000D3030DC01092D3030AC01092D10310927B
:10A8E000D00388EE93E09093BC018093BB014BA50D
:10A8F000242F33278091D0039091D1032817390753
:10A9000024F43093D1032093D003E0916908EE231F
:10A9100079F02E2F332727FD30958091D003909129
:10A92000D1032817390724F43093D1032093D0039F
:10A930004091B5035091B6036091B7037091B8038D
:10A94000413851056105710574F08091850390913E
:10A9500086032091D0033091D103820F931F9093EF
:10A9600086038093850340585F4F6F4F7F4F74F489
:10A9700080918503909186032091D0033091D1037B
:10A98000821B930B909386038093850381E090E074
:10A990009093D1038093D003A090B903B090BA03F1
:10A9A000C090BB03D090BC03D601C501D7FE07C041
:10A9B00088279927DC018A199B09AC09BD098150B8
:10A9C0009240A040B04034F084E090E09093D103F6
:10A9D0008093D0038091DA039091DB03A091DC0394
:10A9E000B091DD032091C8073091C9074091CA0793
:10A9F0005091CB07821B930BA40BB50B815E914B3F
:10AA0000AF4FBF4F8F539C49A040B04018F0E93181
:10AA10000CF4FFC031E0A31630E1B30630E0C3060A
:10AA200030E0D3060CF473C08091D403882309F47A
:10AA30006AC0D601C501D7FE07C088279927DC0167
:10AA40008A199B09AC09BD099C01AD01B7FF04C07F
:10AA500021503E4F4F4F5F4F69E0559547953795D1
:10AA600027956A95D1F78091D0039091D103820FF9
:10AA7000931F9093D1038093D003D601C501D7FED5
:10AA800003C00796A11DB11D23E0B595A795979525
:10AA900087952A95D1F78093C8039093C903A09313
:10AAA000CA03B093CB0389589341A040B04064F0EF
:10AAB00088E893E1A0E0B0E08093C8039093C903D5
:10AAC000A093CA03B093CB032091C8033091C9036C
:10AAD0004091CA035091CB0357FF04C021503F4F10
:10AAE0004F4F5F4F232F342F452F552747FD5A9542
:10AAF00080910C0390910D03820F931F90930D038F
:10AB000080930C0306C081E08093D40302C01092AE
:10AB1000D40350E0A51650EFB5065FEFC5065FEF12
:10AB2000D5060CF073C08091D503882309F46AC060
:10AB3000D601C501D7FE07C088279927DC018A19ED
:10AB40009B09AC09BD099C01AD01B7FF04C02150B0
:10AB50003E4F4F4F5F4F09E05595479537952795E5
:10AB60000A95D1F78091D0039091D103820F931F62
:10AB70009093D1038093D003D601C501D7FE03C0C3
:10AB80000796A11DB11D13E0B595A79597958795DB
:10AB90001A95D1F78093C8039093C903A093CA0371
:10ABA000B093CB0388579C4EAF4FBF4F64F488E7F8
:10ABB0009CEEAFEFBFEF8093C8039093C903A093BF
:10ABC000CA03B093CB032091C8033091C9034091CD
:10ABD000CA035091CB0357FF04C021503F4F4F4F42
:10ABE0005F4F232F342F452F552747FD5A958091CE
:10ABF0000C0390910D03820F931F90930D0380938C
:10AC00000C0311C081E08093D5030DC01092D503D1
:10AC10000AC01092D1031092D00388EE93E0909373
:10AC2000BC018093BB017BA5272F33278091D003E4
:10AC30009091D1032817390724F43093D10320933E
:10AC4000D00380916908882379F0282F332727FDC6
:10AC500030958091D0039091D1032817390724F4BF
:10AC60003093D1032093D0034091B9035091BA039C
:10AC70006091BB037091BC034138510561057105BA
:10AC800074F080918303909184032091D0033091DC
:10AC9000D103820F931F90938403809383034058C2
:10ACA0005F4F6F4F7F4FCCF480918303909184036B
:10ACB0002091D0033091D103821B930B9093840396
:10ACC000809383030AC010920D0310920C0310921C
:10ACD0000B0310920A0310922C038091CD07882356
:10ACE00041F410920D0310920C0310920B0310927A
:10ACF0000A038091C0079091C107A091C207B0914B
:10AD0000C3078093D6039093D703A093D803B0933F
:10AD1000D9038091C8079091C907A091CA07B09143
:10AD2000CB078093DA039093DB03A093DC03B0930B
:10AD3000DD0310926003109261031092620310927F
:10AD4000630310925C0310925D0310925E031092F5
:10AD50005F03109258031092590310925A031092F5
:10AD60005B031092C0071092C1071092C2071092A5
:10AD7000C3071092C8071092C9071092CA07109211
:10AD8000CB071092B7071092B8071092B90710922C
:10AD9000BA071092A9071092AA071092AB07109257
:10ADA000AC07109235021092340200911A031091F0
:10ADB0001B03C80117FF04C088279927801B910B2C
:10ADC00040976CF088EE93E09093BC018093BB01B8
:10ADD0008091150684FD03C081E08093C303F09049
:10ADE0002106AF2CBB24CC24DD24B801882777FDB5
:10ADF0008095982F980117FF04C022273327201B26
:10AE0000310B442737FD4095542F0E94A37A9B01B4
:10AE1000AC01C601B5010E94A37A97FF04C061503E
:10AE20007E4F8F4F9F4FE9E0959587957795679572
:10AE3000EA95D1F79B018F2D9927809FD001819FA3
:10AE4000B00D909FB00D1124CD01B7FD03969595DF
:10AE5000879595958795280F391F442737FD40958D
:10AE6000542F2093A9033093AA034093AB0350932C
:10AE7000AC038091400390914103A0914203B091B3
:10AE80004303821B930BA40BB50B80934003909359
:10AE90004103A0934203B09343038155934CA040D8
:10AEA000B04064F080E593ECA0E0B0E08093400314
:10AEB00090934103A0934203B093430380914003D6
:10AEC00090914103A0914203B0914303805B9C4366
:10AED000AF4FBF4F64F480EB9CE3AFEFBFEF8093C5
:10AEE000400390934103A0934203B0934303A09087
:10AEF0003203B0903303A114B10409F477C18091F7
:10AF0000150683FF73C18091700390917103A09126
:10AF10007203B0917303B7FF04C081509E4FAF4FCF
:10AF2000BF4F69E0B595A795979587956A95D1F735
:10AF30006C0197FF04C0D094C194D108D394809140
:10AF4000680390916903A0916A03B0916B03B7FF06
:10AF500004C081509E4FAF4FBF4F59E0B595A795A4
:10AF6000979587955A95D1F7BC0197FF03C07095C7
:10AF700061957F4FC616D7060CF46B01B601D7FE5C
:10AF800002C0695F7F4F2B0143E0559447944A9577
:10AF9000E1F722E030E0420E531E4CE152E0A40EF5
:10AFA000B51E75010027F7FC0095102F64EE7DEFAC
:10AFB000A60EB71E8091F6079091F707A091F807AB
:10AFC000B091F9076090950170909601809097017B
:10AFD00090909801BC01CD01A40193010E94177BC0
:10AFE000E21AF30A040B150BC801B70128E631E099
:10AFF00040E050E00E94177BDC01CB013CE4E32EF3
:10B000003FEFF32EE80EF91E0091BB011091BC0139
:10B010000115110589F579E1C716D1046CF5809108
:10B020002A0390912B038E0D9F1D90932B038093E9
:10B030002A038091C3038823F9F0C501AA2797FD4D
:10B04000A095BA2FBC01CD01A40193010E94A37A5F
:10B05000DC01CB018093F6079093F707A093F807E4
:10B06000B093F907BC01CD010E94177B30933103E7
:10B07000209330031092C303C70124E0880F991F67
:10B080002A95E1F7B2010E94E27ACB01AA2797FD47
:10B09000A095BA2F2091F6073091F7074091F80755
:10B0A0005091F907280F391F4A1F5B1F2093F6079D
:10B0B0003093F7074093F8075093F907F090AA01EF
:10B0C0006F2D7727C69EC001C79E900DD69E900D0E
:10B0D000112497FD4F966C0185E0D594C7948A950D
:10B0E000E1F76C197D096B0177FD7AC00115110537
:10B0F00009F06FC00091F1021091F2028091EF020D
:10B100009091F002080F191F17FF02C0095F1F4F2F
:10B11000B3E015950795BA95E1F7005C1F4FCA019A
:10B12000B901A40193010E94177BDA01C9012091A2
:10B13000300330913103442737FD4095542F821B53
:10B14000930BA40BB50B845E9D4FAF4FBF4FBC015B
:10B15000CD0128E631E040E050E00E94177BDC01A1
:10B16000CB01845B90408C9DD0018D9DB00D9C9D4A
:10B17000B00D1124CD01B8010E94E27A83E0F89E5F
:10B1800060011124C616D70614F4B60108C088273A
:10B1900099278C199D09681779070CF4BC019B014C
:10B1A000442737FD4095542F8091400390914103EF
:10B1B000A0914203B0914303820F931FA41FB51FB8
:10B1C0008093400390934103A0934203B0934303C1
:10B1D0000DC0015010401093BC010093BB0106C08C
:10B1E00084EF91E09093BC018093BB0180912C038C
:10B1F000882381F0109238031092390310923A0399
:10B2000010923B0310923C0310923D0310923E03B8
:10B2100010923F03109107031123F1F48091CD07A1
:10B22000282F33274427552780917003909171036D
:10B23000A0917203B0917303BC01CD010E94A37A67
:10B24000DC01CB01BC01CD0128EF3AE240E050E047
:10B250000E94177B290102C0442455240091060353
:10B260000023F1F48091CD07282F33274427552759
:10B270008091680390916903A0916A03B0916B0378
:10B28000BC01CD010E94A37ADC01CB01BC01CD0140
:10B2900028EF3AE240E050E00E94177B190102C01B
:10B2A000222433248091A3079091A407893C91051F
:10B2B0001CF088EC90E005C088539F4F34F488E37D
:10B2C0009FEF9093A4078093A3078091AE0790917E
:10B2D000AF07893C91051CF088EC90E005C08853CD
:10B2E0009F4F34F488E39FEF9093AF078093AE07AE
:10B2F0008091CD072091F4076091B0077091B1075C
:10B30000882309F064C0CB01AA2797FDA095BA2F26
:10B31000A22EBB24CC24DD24BC01CD01A6019501C5
:10B320000E94A37A97FF04C0615C7F4F8F4F9F4FAD
:10B33000A6E09595879577956795AA95D1F770932F
:10B34000B1076093B0078091A1079091A207AA2747
:10B3500097FDA095BA2FBC01CD01A60195010E94D1
:10B36000A37A97FF04C0615C7F4F8F4F9F4FF6E039
:10B370009595879577956795FA95D1F77093A2077C
:10B380006093A1078091EF079091F007880F991FB4
:10B39000AA2797FDA095BA2F2091A8073327442705
:10B3A0005527BC01CD010E94A37A97FF04C0615CC0
:10B3B0007F4F8F4F9F4FE6E09595879577956795DF
:10B3C000EA95D1F77093F0076093EF07B9C0CB010E
:10B3D000AA2797FDA095BA2FA22EBB24CC24DD244A
:10B3E000BC01CD01A60195010E94A37A9B01AC018D
:10B3F0008091A3079091A407AA2797FDA095BA2F43
:10B4000067E0880F991FAA1FBB1F6A95D1F7280F05
:10B41000391F4A1F5B1F57FF04C0215C3F4F4F4F2E
:10B420005F4FA6E05595479537952795AA95D1F793
:10B43000C201820F931F9093B1078093B007809150
:10B44000A1079091A207AA2797FDA095BA2FBC014A
:10B45000CD01A60195010E94A37A9B01AC018091C8
:10B46000AE079091AF07AA2797FDA095BA2FF7E0F6
:10B47000880F991FAA1FBB1FFA95D1F7280F391FF4
:10B480004A1F5B1F57FF04C0215C3F4F4F4F5F4F68
:10B49000E6E05595479537952795EA95D1F7C1018F
:10B4A000820F931F9093A2078093A1078091EF07CB
:10B4B0009091F007880F991FAA2797FDA095BA2FA2
:10B4C0002091A807332744275527BC01CD010E94AE
:10B4D000A37A5B016C0197FF08C02FE330E040E0E6
:10B4E00050E0A20EB31EC41ED51E76E0D594C794BC
:10B4F000B794A7947A95D1F78091BD07282F332769
:10B50000442755278091540390915503A0915603E9
:10B51000B0915703BC01CD010E94A37ADC01CB019D
:10B52000BC01CD0120EF35E540E050E00E94177BE3
:10B53000DA01C9018A0D9B1D9093F0078093EF07F4
:10B540008091B0079091B1078150904134F080E034
:10B5500090E19093B1078093B0078091B0079091EC
:10B56000B1078050904F34F480E090EF9093B10792
:10B570008093B0078091A1079091A20781509041DC
:10B5800034F080E090E19093A2078093A10780912E
:10B59000A1079091A2078050904F34F480E090EF83
:10B5A0009093A2078093A1078091EF079091F007F5
:10B5B0008150904134F080E090E19093F0078093C7
:10B5C000EF078091EF079091F0078050904F34F48F
:10B5D00080E090EF9093F0078093EF078091000157
:10B5E000482F552780911D0190911E01481759073A
:10B5F00094F420911D0130911E01E8A1F9A1E49F6E
:10B60000C001E59F900DF49F900D1124B9010E9497
:10B61000CE7A79A368A328A139A1220F331F220F64
:10B62000331F39A328A34091150640FFB3C600235A
:10B6300009F0B0C6112309F0ADC6CC24DD244601C3
:10B6400080910803909109039093E2058093E105AE
:10B6500020918703309188032115310509F03FC0FF
:10B6600080911301909114018959934058F087B546
:10B67000803F20F480913802815011C081E0809396
:10B68000E9034EC080911301909114018436910515
:10B6900008F587B58031D0F0809138028F5F8093B4
:10B6A00038029FE089029001112480910406821BD8
:10B6B00087BD8CE291E090932402809323028EE573
:10B6C00091E090938803809387032AC081E0809360
:10B6D000E80326C01093E8031093E90321C080918A
:10B6E000120390911303A0911403B091150354E039
:10B6F000880F991FAA1FBB1F5A95D1F78093390253
:10B7000090933A02A0933B02B0933C02D09237024E
:10B71000C092360221503040309388032093870333
:10B720002091AD0141FF29C0223320F08091010317
:10B730008D38E0F08091C10181508093C1018F3F2D
:10B7400009F042C010922D038091120390911303CF
:10B75000A0911403B091150380930E0390930F03EF
:10B76000A0931003B093110381E004C081E08093A3
:10B770002D0388EC8093C10127C08091990190919D
:10B780009A01820F911D20911A063327829FA001F2
:10B79000839F500D929F500D1124CA01AA2797FD37
:10B7A000A095BA2F80930E0390930F03A0931003DC
:10B7B000B0931103809101038D3818F010922D037E
:10B7C00003C081E080932D038091700390917103F9
:10B7D000A0917203B0917303E0909501F0909601EF
:10B7E0000091970110919801BC01CD01A80197012A
:10B7F0000E94177B59016A01809168039091690347
:10B80000A0916A03B0916B03BC01CD01A80197011F
:10B810000E94177BB901C5010E940E713C01CC97B3
:10B820001CF04CE3642E712CC3010E94096D3C0195
:10B8300080E28093940180912D03882309F436C41B
:10B840008091E80299279C012071307084FD2EC4FC
:10B8500060916B0660FD04C08091150681FD07C0F4
:10B8600008A119A13093DF032093DE0397C18091D3
:10B87000E80281FF69C14091BD015091BE01CA013A
:10B880000F96209118033091190382179307ACF596
:10B890008091E803882389F58091EA0381FF13C032
:10B8A0008D7F8093EA038091120390911303A091FE
:10B8B0001403B091150380930E0390930F03A0938C
:10B8C0001003B09311038091EA0381608093EA032F
:10B8D000241B350B2F50304037FF03C03095219586
:10B8E0003F4F8091DE039091DF03820F931F90936F
:10B8F000DF038093DE038BE26EC0CA010F97281727
:10B900003907ACF58091E903882389F58091EA0332
:10B9100080FF13C08E7F8093EA0380911203909181
:10B920001303A0911403B091150380930E03909319
:10B930000F03A0931003B09311038091EA03826078
:10B940008093EA03241B350B215F3F4F37FF03C071
:10B95000309521953F4F8091DE039091DF03821B4C
:10B96000930B9093DF038093DE038DE234C020912C
:10B97000EA03822F992783709070892B59F12C7FCD
:10B980002093EA031092DF031092DE03209112034A
:10B9900030911303409114035091150320930E032B
:10B9A00030930F03409310035093110361FF06C0BF
:10B9B00084EF91E0909324028093230280911603F8
:10B9C000882341F423333105410551051CF081E002
:10B9D000809316038DE3809394012091DE033091D0
:10B9E000DF03C90137FF04C088279927821B930B07
:10B9F000815092400CF491C080911A069927289F9B
:10BA0000D001299FB00D389FB00D1124CD0160E009
:10BA100075E00E94E27ACB01AA2797FDA095BA2F84
:10BA200020910E0330910F034091100350911103A8
:10BA3000280F391F4A1F5B1F20930E0330930F03FB
:10BA400040931003509311031092DF031092DE0312
:10BA5000A0901203B0901303C0901403D09015036C
:10BA6000D601C50180509440A040B0408217930792
:10BA7000A407B5075CF4D601C50180509C4FAF4FB9
:10BA8000BF4F281739074A075B0744F080930E031E
:10BA900090930F03A0931003B093110380916B0652
:10BAA00081FF06C084E690E09093240280932302F5
:10BAB00080911E06882389F540910803509109035F
:10BAC00057FF02C04D5F5F4F559547955595479578
:10BAD00080911D0190911E01209100013327489F04
:10BAE000F001499FF00D589FF00D1124CF01B901CD
:10BAF0000E94E27A7093BE016093BD0166347105C5
:10BB00001CF486E490E005C06739710534F086E9DD
:10BB100090E09093BE018093BD0180918703909146
:10BB20008803892BB9F18091120390911303A0919E
:10BB30001403B091150380930E0390930F03A09309
:10BB40001003B093110326C0809112039091130348
:10BB5000A0911403B091150380599140A040B040CA
:10BB600080930E0390930F03A0931003B0931103DF
:10BB700080911E06882311F0992702C088E790E083
:10BB80009093BE018093BD0128A139A13093090390
:10BB9000209308030091080310910903A090120359
:10BBA000B0901303C0901403D090150320910E039E
:10BBB00030910F0340911003509111032A153B055A
:10BBC0004C055D0524F080916B0680FDB1C280912B
:10BBD000870390918803892B39F000910803109115
:10BBE0000903CC24DD24D7C0D601C501821B930BE9
:10BBF000A40BB50B8093AD039093AE03A093AF035A
:10BC0000B093B003823030E893073FEFA3073FEFD4
:10BC1000B3072CF481E090E8AFEFBFEF09C08F5F6E
:10BC20009F47A040B04064F08FEF9FE7A0E0B0E0F6
:10BC30008093AD039093AE03A093AF03B093B00392
:10BC4000C090AD03D090AE038091AC01282F332774
:10BC5000442755278091AD039091AE03A091AF0387
:10BC6000B091B003BC01CD010E94A37A97FF04C03C
:10BC7000615E7F4F8F4F9F4F25E095958795779514
:10BC800067952A95D1F76093AD037093AE038093C7
:10BC9000AF039093B00365305EEF75075FEF8507E4
:10BCA0005FEF95072CF484E09EEFAFEFBFEF09C084
:10BCB000605074408040904064F080E094E0A0E0E8
:10BCC000B0E08093AD039093AE03A093AF03B09325
:10BCD000B0038090AD039090AE0320913602309176
:10BCE000370237FF02C0295F3F4F83E03595279524
:10BCF0008A95E1F7BFEF22383B071CF421E83FEFBC
:10BD000005C02038310514F020E830E0C901AA2729
:10BD100097FDA095BA2F2091AE01332744275527D0
:10BD2000BC01CD010E94A37A97FF04C06D5F7F4FD5
:10BD30008F4F9F4FB2E09595879577956795BA9508
:10BD4000D1F79B01EFEF61307E071CF420E03FEF5D
:10BD500006C06F3F710519F014F020E031E08091CA
:10BD6000EA03882349F0C90137FD03969C01359504
:10BD70002795359527950DC080916B0680FF09C0EA
:10BD8000C90137FD07969C01F3E035952795FA9593
:10BD9000E1F7820E931E2091AB01222309F454C0D7
:10BDA000609134037091350380913603909137038D
:10BDB00097FF04C061587F4F8F4F9F4FE7E09595E5
:10BDC000879577956795EA95D1F7332744275527C7
:10BDD0000E94A37A97FF04C0615E7F4F8F4F9F4FF1
:10BDE00055E095958795779567955A95D1F7609326
:10BDF000AD037093AE038093AF039093B0036138AB
:10BE0000FFEF7F07FFEF8F07FFEF9F072CF480E81E
:10BE10009FEFAFEFBFEF0AC06F3F7105810591053E
:10BE200069F064F080E091E0A0E0B0E08093AD03C1
:10BE30009093AE03A093AF03B093B0038091AD0392
:10BE40009091AE03880E991E8091A901282F332767
:10BE500080916C08992787FD9095289FA001299FC4
:10BE6000500D389F500D11249A0157FF02C02158E0
:10BE70003F4F220F232F221F330B5FEF213835074F
:10BE80001CF420E83FEF06C02F3F310519F014F0F5
:10BE900020E031E0820E931EC401AA2797FDA095F1
:10BEA000BA2FE0900803F09009039701442737FD6B
:10BEB0004095542FBC01CD010E94A37A97FF04C086
:10BEC00061507E4F8F4F9F4F29E0959587957795CD
:10BED00067952A95D1F7061B170B8091DE03909189
:10BEE000DF03892B09F060C01E141F040CF05CC036
:10BEF0009601D7FE03C0309521953F4F2D33310574
:10BF000040F48091E2039091E3038017910774F568
:10BF100026C02C53304085E0369527958A95E1F769
:10BF20002031310510F02FE030E04091E2035091D4
:10BF3000E3031C141D04E4F480E190E0821B930BE6
:10BF4000489F9001499F300D589F300D1124B4E057
:10BF500036952795BA95E1F72017310720F580919E
:10BF6000BF019091C00108171907F4F08C011CC0A3
:10BF7000205F3F4F8091BF019091C001829FB0012F
:10BF8000839F700D929F700D11249B01A4E0369544
:10BF90002795AA95E1F74017510714F08A0104C0CC
:10BFA0000217130708F08901C801AA2797FDA09579
:10BFB000BA2FFDE0880F991FAA1FBB1FFA95D1F772
:10BFC0009301442737FD4095542FBC01CD010E94B9
:10BFD000177B2093B1033093B2034093B303509384
:10BFE000B4030091B1031091B2038091E0039091EA
:10BFF000E1039C01220F331F280F391F200F311F2F
:10C0000037FF02C02D5F3F4FA901559547955595C4
:10C0100047955093E1034093E00380911606282F43
:10C020003327220F331F220F331F241735076CF4D9
:10C030008091EE07282F3327220F331F220F331F43
:10C04000205530404217530724F03093E1032093EA
:10C05000E00380916B0680FF14C08091E003909113
:10C06000E103A8A1B9A18A179B0724F0B093E103CB
:10C07000A093E003E091E003F091E103F9A3E8A3CA
:10C0800057C028A139A12E193F0937FF02C02D5FE3
:10C090003F4F35952795359527954091E003509171
:10C0A000E103420F531F59A348A342C080911E06CB
:10C0B000882301F5609108037091090377FF02C09E
:10C0C0006D5F7F4F759567957595679540911D01DB
:10C0D00050911E0180910001282F3327649FC001D9
:10C0E000659F900D749F900D1124B9010E94E27A12
:10C0F000CB0101C099279093BE018093BD0180912F
:10C10000BD019091BE01873491051CF486E490E056
:10C1100005C08639910534F086E990E09093BE0120
:10C120008093BD0168A179A17093E1036093E0035E
:10C130008091E80299279C012270307081FF1CC118
:10C140008091E4039091E503A091E603B091E703A9
:10C150000097A105B10521F0809116038130B1F45B
:10C16000E8A1F9A1CF01AA2797FDA095BA2F1EE05B
:10C17000880F991FAA1FBB1F1A95D1F78093E4035C
:10C180009093E503A093E603B093E7038091160331
:10C19000813019F482E08093160328A139A1C901E6
:10C1A000AA2797FDA095BA2F9301442737FD409504
:10C1B000542FBC01CD010E94A37ADC01CB018093F6
:10C1C000B1039093B203A093B303B093B403B7FF4A
:10C1D00004C08150904EAF4FBF4F5C016D01FDE038
:10C1E000D594C794B794A794FA95D1F7A092B103C8
:10C1F000B092B203C092B303D092B4036091E9024B
:10C200007091EA023FE0603A730750F58091E403D1
:10C210009091E503A091E603B091E7039C01AD0185
:10C22000EAE05695479537952795EA95D1F7821B11
:10C23000930BA40BB50BA601950104E0220F331F4D
:10C24000441F551F0A95D1F7820F931FA41FB51FD6
:10C250008093E4039093E503A093E603B093E70390
:10C2600060547F4118F58091E4039091E503A0911B
:10C27000E603B091E7039C01AD011CE0569547959C
:10C28000379527951A95D1F7821B930BA40BB50B05
:10C29000A6019501F2E0220F331F441F551FFA95A6
:10C2A000D1F7820F931FA41FB51F29C080913602BA
:10C2B00090913702809136029091370297FF03C028
:10C2C000909581959F4F843691050CF58091E403FC
:10C2D0009091E503A091E603B091E7039C01AD01C5
:10C2E000EEE05695479537952795EA95D1F7821B4D
:10C2F000930BA40BB50B8A0D9B1DAC1DBD1D80932C
:10C30000E4039093E503A093E603B093E7038091E1
:10C31000E4039091E503A091E603B091E7037EE08A
:10C32000B695A795979587957A95D1F79093090338
:10C330008093080340911C06442399F055279C01E3
:10C34000BA010E94E27AC901861B970B9093E3031E
:10C350008093E203260F371F3093C0012093BF0163
:10C3600019C01092E3031092E2038FEF93E09093D1
:10C37000C0018093BF010EC0109216031092E40317
:10C380001092E5031092E6031092E703309309033D
:10C39000209308035091B50758AB252F3327220F60
:10C3A000331F220F331F285D3F4F68A179A1261745
:10C3B000370714F039A328A37091EE0779AB872FC4
:10C3C0009927880F991F880F991F80559040A8A121
:10C3D000B9A18A179B0714F499A388A380916D02D1
:10C3E000882321F4809173088F3FA1F08091E902A6
:10C3F0009091EA020297C09768F4E8A1F9A11E168D
:10C400001F0644F481E090E09093EA028093E902F1
:10C4100039A328A328A139A13093C6052093C505C7
:10C420008091A9039091AA03A091AB03B091AC03B2
:10C4300042E0880F991FAA1FBB1F4A95D1F7C090F1
:10C44000EF07D090F007C81AD90A213A31058CF0CD
:10C45000C90137FD0196959587958C159D050CF4BE
:10C460006C01909581959F4FC816D90694F46C0184
:10C4700010C031E5C316D1041CF000E5C02ED12C4C
:10C4800040EBC4164FEFD40624F410EBC12E1FEF7F
:10C49000D12E59A9252F3327220F331F220F331FE7
:10C4A000C90168A179A1861B970B8C159D050CF419
:10C4B0006C0188A199A1821B930BC816D9060CF4B4
:10C4C0006C012091B0073091B10740911E0350914B
:10C4D0001F03241B350B3093BF072093BE07B0907A
:10C4E0002B068B2D9927829FD001839FB00D929FA1
:10C4F000B00D1124CD01B7FD07967C01A3E0F594A2
:10C50000E794AA95E1F70091CD07002309F465C0EF
:10C51000441A550A9201442737FD4095542F8091C3
:10C520003C0390913D03A0913E03B0913F03820FE5
:10C53000931FA41FB51F80933C0390933D03A093CA
:10C540003E03B0933F0381509D47A040B04064F04C
:10C5500080E09DE7A0E0B0E080933C0390933D0332
:10C56000A0933E03B0933F0380913C0390913D0321
:10C57000A0913E03B0913F0380509348AF4FBF4F0F
:10C5800064F480E093E8AFEFBFEF80933C039093B7
:10C590003D03A0933E03B0933F038091B10190917E
:10C5A000B2019C01442737FD4095542F80913C03F4
:10C5B00090913D03A0913E03B0913F03BC01CD019A
:10C5C0000E94177BE20EF31E1092A1031092A203A9
:10C5D0001092A3031092A40361C0442737FD409535
:10C5E000542F8091A1039091A203A091A303B09135
:10C5F000A403820F931FA41FB51F8093A1039093E0
:10C60000A203A093A303B093A40381509D47A0402D
:10C61000B04064F080E09DE7A0E0B0E08093A1032B
:10C620009093A203A093A303B093A4038091A103CA
:10C630009091A203A091A303B091A40380509348CA
:10C64000AF4FBF4F64F480E093E8AFEFBFEF80934C
:10C65000A1039093A203A093A303B093A40380919A
:10C66000AF019091B0019C01442737FD4095542FB4
:10C670008091A1039091A203A091A303B091A40380
:10C68000BC01CD010E94177BE20EF31E10923C0309
:10C6900010923D0310923E0310923F0310919B01B4
:10C6A000612F7727882799279601D7FE04C0222774
:10C6B00033272C193D0937FF02C02F5F3F4F3595B7
:10C6C000279548A159A1240F351F442737FD4095D0
:10C6D000542F0E94A37A97FF04C0615C7F4F8F4F55
:10C6E0009F4FE6E09595879577956795EA95D1F701
:10C6F0009B016E157F050CF47B01309521953F4F12
:10C70000E216F3060CF479012091A1073091A207FB
:10C7100040911C0350911D03241B350B3093A0073F
:10C7200020939F078B2D9927829FB001839F700DC7
:10C73000929F700D1124CB0177FD07965C0163E099
:10C74000B594A7946A95E1F7002309F465C0241A0B
:10C75000350A9101442737FD4095542F80913803C5
:10C7600090913903A0913A03B0913B03820F931F3C
:10C77000A41FB51F8093380390933903A0933A0305
:10C78000B0933B0381509D47A040B04064F080E0EF
:10C790009DE7A0E0B0E08093380390933903A09325
:10C7A0003A03B0933B038091380390913903A091F1
:10C7B0003A03B0913B0380509348AF4FBF4F64F4AE
:10C7C00080E093E8AFEFBFEF809338039093390395
:10C7D000A0933A03B0933B038091B1019091B201D1
:10C7E0009C01442737FD4095542F80913803909148
:10C7F0003903A0913A03B0913B03BC01CD010E94E3
:10C80000177BA20EB31E1092A5031092A6031092DE
:10C81000A7031092A80361C0442737FD4095542F09
:10C820008091A5039091A603A091A703B091A803BE
:10C83000820F931FA41FB51F8093A5039093A60397
:10C84000A093A703B093A80381509D47A040B04098
:10C8500064F080E09DE7A0E0B0E08093A5039093B2
:10C86000A603A093A703B093A8038091A50390917A
:10C87000A603A091A703B091A80380509348AF4F9F
:10C88000BF4F64F480E093E8AFEFBFEF8093A50360
:10C890009093A603A093A703B093A8038091AF0140
:10C8A0009091B0019C01442737FD4095542F809111
:10C8B000A5039091A603A091A703B091A803BC0182
:10C8C000CD010E94177BA20EB31E10923803109266
:10C8D000390310923A0310923B03612F7727882780
:10C8E00099279601D7FE04C0222733272C193D092A
:10C8F00037FF02C02F5F3F4F3595279548A159A1BB
:10C90000240F351F442737FD4095542F0E94A37AEA
:10C9100097FF04C0615C7F4F8F4F9F4F26E0959536
:10C920008795779567952A95D1F79B016A157B05C1
:10C930000CF45B01309521953F4FA216B3060CF421
:10C9400059018FEC682E86E0782E06E8802E06E0EE
:10C95000902E1BE0312EBEEC4B2EB7E05B2ED401A7
:10C960002C9112160CF0DAC0203419F408A119A188
:10C970001EC0E8A1F9A1CF01AA2797FDA095BA2F63
:10C98000332727FD3095432F532FBC01CD010E9443
:10C99000A37A97FF04C0615C7F4F8F4F9F4FA6E043
:10C9A0009595879577956795AA95D1F78B01F401B1
:10C9B0002181203419F40E0D1F1D22C0203C19F4D2
:10C9C0000E191F091DC0C701AA2797FDA095BA2FF0
:10C9D000332727FD3095432F532FBC01CD010E94F3
:10C9E000A37A97FF04C0615C7F4F8F4F9F4FF6E0A3
:10C9F0009595879577956795FA95D1F7060F171F47
:10CA0000F4012281203419F40A0D1B1D22C0203CA0
:10CA100019F40A191B091DC0C501AA2797FDA09585
:10CA2000BA2F332727FD3095432F532FBC01CD015B
:10CA30000E94A37A97FF04C0615C7F4F8F4F9F4F86
:10CA4000E6E09595879577956795EA95D1F7060F76
:10CA5000171FF4012381203419F40C0D1D1D22C071
:10CA6000203C19F40C191D091DC0C601AA2797FD09
:10CA7000A095BA2F332727FD3095432F532FBC01A4
:10CA8000CD010E94A37A97FF04C0615C7F4F8F4F56
:10CA90009F4F56E095958795779567955A95D1F76D
:10CAA000060F171FD2018D919C918017910754F4A6
:10CAB000BC01600F711F77FF02C06F5F7F4F8B015A
:10CAC00015950795B8A98B2F9927880F991F880F5F
:10CAD000991F8017910754F4E9A98E2F9927880F81
:10CAE000991F880F991F081719070CF08C01C801AE
:10CAF00017FD03969595879595958795F301818305
:10CB0000880F991F880F991F9801281B390BC9019D
:10CB1000880F8283D2010D931C9303C0F30111820D
:10CB200012823A9422E030E0420E531E44E050E07C
:10CB3000840E951E68E070E0660E771E37FE0FCFFC
:10CB4000E2E1CB5C0C944E7B8091F7039091F8036B
:10CB5000A091F903B091FA038093EF039093F0034F
:10CB6000A093F103B093F2038091F3039091F40347
:10CB7000A091F503B091F6038093EB039093EC033F
:10CB8000A093ED03B093EE03089510920204109267
:10CB90000104109200041092FF03089584B1806A8A
:10CBA00084B93D9A82E58CBD1DBC459A81E0809395
:10CBB00000088AEA8093110883E8809312088AE0CB
:10CBC00080931308109215081092140810921708F9
:10CBD0001092160810926B08109233080895309145
:10CBE0000008332309F085C00DB407FE82C084E03D
:10CBF00080932202459A2EB58091060499278130B0
:10CC0000910589F0823091051CF4892B21F03EC0FA
:10CC10000297B9F03BC030933208209307042138C3
:10CC2000A9F581E008C0253549F480910704820FF9
:10CC30008093070482E08093060428C030930604A2
:10CC400025C080913208E82FFF27E25BF74F208351
:10CC50008F5F80933208909107048A31A0F02917E2
:10CC600069F48AE1AEE4B8E0E4E3F8E00D90019203
:10CC70008A95E1F781E08093330802C0309333084E
:10CC80001092060403C0920F90930704209110089D
:10CC9000203208F028C04598000000000000000085
:10CCA0000000000000000000000000000000000084
:10CCB0000000000000000000000000000000000074
:10CCC0000000000000000000E0910908F0910A084F
:10CCD000E20FF11D80818EBD809130089081890F17
:10CCE0008093300803C081E0809300082F5F209379
:10CCF00010080895EF92FF920F931F9380912406DE
:10CD00009927880F991F880F991F7C010027F7FC2E
:10CD10000095102F8091700390917103A091720380
:10CD2000B0917303BC01CD01A80197010E94177B4C
:10CD3000309315082093140880916803909169033B
:10CD4000A0916A03B0916B03BC01CD01A8019701CA
:10CD50000E94177B30931708209316082091F6073E
:10CD60003091F7074091F8075091F907DA01C901AE
:10CD7000E3E0880F991FAA1FBB1FEA95D1F7820F26
:10CD8000931FA41FB51F820F931FA41FB51F2091CF
:10CD90009501309196014091970150919801BC0105
:10CDA000CD010E94177B30931D0820931C088091B1
:10CDB0008103909182032091440230914502821BAD
:10CDC000930B9093230880932208E0917703F091CE
:10CDD00078038091C5079091C607BF010E94E27A4F
:10CDE000CB019B01220F331F220F331F280F391F46
:10CDF000280F391F37FF02C02D5F3F4F359527950C
:10CE00003595279530931908209318088091F207DB
:10CE10009091F307BF010E94E27A9B01220F331F1A
:10CE2000220F331F260F371F260F371F37FF02C071
:10CE30002D5F3F4F359527953595279530931B08E6
:10CE400020931A0810927803109277031092C60765
:10CE50001092C5071092F3071092F2078091130801
:10CE600099278D30910509F466C08E3091055CF4E8
:10CE70008B30910509F48EC08C3091050CF00FC1F8
:10CE80000A9761F0A8C18F30910509F47CC18F30F9
:10CE900091050CF45CC1409799F19DC1809101030B
:10CEA0008093240880910003809325088091FF02DD
:10CEB000809326088091FE02809327088091FD02CE
:10CEC000809328088091FC02809329088091FB02BE
:10CED00080932A088091FA0280932B088091E802BF
:10CEE00080932C088091E802837F8093E8020E945F
:10CEF0000D2F80932D088091740380932E086BC1B1
:10CF000080916D0890916E08909325088093240875
:10CF10008091710890917208909327088093260859
:10CF200080911D0190911E0180932808809100013D
:10CF30008093290850C18091AD0780932408809187
:10CF40005706809325088091580680932608809183
:10CF500059068093270880915A068093280880916B
:10CF60005E068093290880915F0680932A0880914D
:10CF7000600680932B088091630680932C08809133
:10CF8000610680932D088091620680932E0880911F
:10CF90006406DAC0F89480910B06E82FFF27EE0FA5
:10CFA000FF1FE05DF84F0190F081E02DE038F105C2
:10CFB0001CF0EFE7F0E006C02FEFE138F20714F4C1
:10CFC000E1E8FFEFE093240880910C06E82FFF27AB
:10CFD000EE0FFF1FE05DF84F0190F081E02DE0388B
:10CFE000F1051CF0EFE7F0E006C06FEFE138F6075F
:10CFF00014F4E1E8FFEFE093250880910A06E82F9A
:10D00000FF27EE0FFF1FE05DF84F0190F081E02D4C
:10D01000E038F1051CF0EFE7F0E006C08FEFE138F3
:10D02000F80714F4E1E8FFEFE09326088091090681
:10D03000E82FFF27EE0FFF1FE05DF84F0190F08112
:10D04000E02DE038F1051CF0EFE7F0E006C02FEF2F
:10D05000E138F20714F4E1E8FFEF7894E093270851
:10D0600080912103809328088091220380932908CE
:10D070008091230380932A088091240380932B08B6
:10D080008091250380932C088091260380932D089E
:10D090008091270380932E088091280355C08091AA
:10D0A0006404863018F01092640485E080932408AC
:10D0B0008091650680932508809112039091130357
:10D0C000A0911403B0911503BC01CD0125E030E01F
:10D0D00040E050E00E94177B3093270820932608F9
:10D0E00080910E0390910F03A0911003B091110352
:10D0F000BC01CD0125E030E040E050E00E94177B0C
:10D10000309329082093280880915B0680932A0891
:10D1100080915C0680932B0880915D0680932C089B
:10D120008091200380932D088091300790913107E2
:10D1300080932E088091C5059091C60597FD0396B2
:10D14000959587959595879580932F0844C0109263
:10D15000240880E58093250885E0809326088EE0EA
:10D1600080932708809102018093280880914904C8
:10D170008093290880914A0480932A0880914B0467
:10D1800080932B0828C080913D06809324088091CD
:10D190006A06809325088091A101809326088091DA
:10D1A000360680932708809137068093280880915F
:10D1B0003806809329088091A00180932A088091E5
:10D1C0003A0680932B0880913B0680932C0880912F
:10D1D0003C0680932D0880913308882309F4CFC042
:10D1E0008AEF8093EA014091350850913608CA01D0
:10D1F00081509E4F8F5F9340B0F42091370830915B
:10D200003808C90181509E4F8F5F934060F4809130
:10D21000150685FF08C05093020440930104309323
:10D2200000042093FF0380913B0890913C0821E08B
:10D230008936920724F490933303809332038091CC
:10D240003203909133032091300330913103821BDC
:10D25000930B845E9D4F68E671E00E94E27A845BE6
:10D26000904090932F0380932E0320913F0830919C
:10D27000400880912302909124028217930740F482
:10D2800080916404882321F43093240220932302A4
:10D290008091340899278836910549F1893691059E
:10D2A00024F48736910531F072C08936910509F46E
:10D2B00045C06DC080914108809368088091420804
:10D2C00080936A088091430880936908809144089C
:10D2D00080936B088091450880936C088091460884
:10D2E0008093EB01809147088093050450C08091A2
:10D2F000410880930B088091420880930C0880912C
:10D30000430880930D088091440880930E08809113
:10D31000450880930F088091B50590914608892BA8
:10D320008093B50590914708909303048091B605CA
:10D3300083709C70892B8093B60529C08091410829
:10D3400080930108809142088093020880914308ED
:10D3500080930308809144088093040880914508D5
:10D36000909146089093060880930508809147089D
:10D3700090914808909308088093070808C010927D
:10D38000020410920104109200041092FF031F91F6
:10D390000F91FF90EF90089580910008882309F481
:10D3A0003BC0459881E198E090930A088093090872
:10D3B00090910404E92FFF27EF51FE4F9F5F909358
:10D3C0000404808180931308993010F010920404B3
:10D3D000109200080E947A6681E080931008000095
:10D3E000000000000000000000000000000000003D
:10D3F000000000000000000000000000000000002D
:10D40000000000000000000000000000000080910B
:10D410001108809330088EBD089587B18C6087B95C
:10D42000429843981092090480E88093ED0110928D
:10D4300008048093EC01089580910E04815080933C
:10D440000E048F3F09F0F4C094E090930E04809195
:10D45000E802807BE1F080915406882349F08091B6
:10D460001104882311F49093090481E0809311043E
:10D47000809155068823B9F080911204882319F40D
:10D4800084E08093080481E0809312040CC08093B0
:10D490001104809312048091500680930F048091B0
:10D4A00052068093100480911104882309F040C033
:10D4B00080916906282F332724FF07C08091170326
:10D4C000882319F425FD4DC04EC090915106983F18
:10D4D00050F08091C7078D3D30F080910F04882374
:10D4E0000CF43FC040C0983F48F08091C7078A3095
:10D4F00028F480910F048823B4F133C0809109048B
:10D500008150809309048F3F79F58091C70781503E
:10D51000809309048091ED01813011F480E801C00D
:10D5200086958093ED018091ED0190910F0417C0D5
:10D53000809109048150809309048F3FA9F489E008
:10D54000809309048091ED01813011F480E801C0DD
:10D5500086958093ED018091ED0190915406892389
:10D5600011F0429A01C0429880911204882309F078
:10D5700043C080916906282F332724FF07C080917C
:10D580001703882319F426FD50C034C09091530628
:10D59000983F50F08091ED078D3D30F08091100460
:10D5A00088230CF442C026C0983F48F08091ED07D4
:10D5B0008A3028F4809110048823E4F036C08091EA
:10D5C00008048150809308048F3F91F58091ED0706
:10D5D0008150809308048091EC01813011F480E83F
:10D5E00001C086958093EC018091EC01909110042C
:10D5F0008923D9F443980895809108048150809339
:10D6000008048F3FA9F489E0809308048091EC011D
:10D61000813011F480E801C086958093EC018091FF
:10D62000EC0190915506892311F0439A089543988F
:10D6300008954FB724E130E0F8948091C9008F77C6
:10D640008093C9008091C9008F7B8093C90080912D
:10D65000C9008F7D8093C9005A9A52985B9A539A59
:10D66000832F99278093CD002093CC008091C80010
:10D6700082608093C80080E18093C9008091CA00D5
:10D680008F778093CA008091CA008F7B8093CA00F5
:10D690008091CA008F7D8093CA008091CA008F7EDE
:10D6A0008093CA008091CA00877F8093CA008091CE
:10D6B000C9008B7F8093C9008091CA0084608093E9
:10D6C000CA008091CA0082608093CA008091C8001D
:10D6D00087FF03C08091CE00F9CF8091C900806898
:10D6E0008093C9004FBF0895EF92FF920F931F934D
:10D6F000CF93DF93482F00E010E08091EE0181305E
:10D7000061F41092EE0184E48093130410921504E6
:10D7100010921404109216042BC1809113048823D4
:10D7200019F421E030E001C098019091140499238C
:10D7300071F4232B11F081E010C084E48093130472
:10D74000909315049093140490931604FAC09130AA
:10D7500069F4232B09F0EBC082E0809314048091DC
:10D7600015048F5F8093150483E0E9C09230D1F4F3
:10D77000232B09F0DCC083E080931304409316044C
:10D7800090911504923039F41092170447FF03C0AA
:10D7900081E08093170483E0809314049F5F90934B
:10D7A0001504CFC0933009F0C2C0232B09F0BFC0CD
:10D7B0009093130482E080931404809115048F5F8A
:10D7C0008093150420911604822F9927782F6627BD
:10D7D000842F9927682B792B80912F06813049F46B
:10D7E0007370CB018050924063E070E00E94E27A57
:10D7F00017C0823061F47770CB018050944066E0AE
:10D8000070E00E94E27A2695269526950BC07370EB
:10D8100068567140CB0177FD0196BC0175956795FF
:10D8200026952695022F11270F7010700F5F1F4F3E
:10D830000D30110508F074C07801E00EF11EF701FB
:10D84000E05DF84F808191819B01281B390BC90154
:10D8500037FF03C0909581959F4F069794F4809170
:10D860002003883C30F480912003865F809320035E
:10D8700008C088EC8093200380916F008F7D809397
:10D880006F00F701E05DF84F808191819C01220FCC
:10D89000331F280F391F260F371F37FF02C02D5F98
:10D8A0003F4FE901D595C795D595C795CB01019611
:10D8B0008C179D0714F4219706C061507040C6175D
:10D8C000D7070CF4219680912003843BD0F0F70118
:10D8D000E05DF84F80819181FE01E81BF90BCF01DB
:10D8E00063E070E00E94E27ACB01880F991F860FF7
:10D8F000971F24E637E0E20EF31EF7019183808341
:10D9000007C024E637E0E20EF31EF7011182108211
:10D91000000F111F005D184FF801D183C08311C0A3
:10D920000231110570F081E08093EE010AC081E0C0
:10D930008093EE01109215041092170484E48093F2
:10D94000130480911504803198F080911704882386
:10D9500031F48091EE01882311F4809393011092A9
:10D960001504109217041092140484E48093130495
:10D97000E6E0CDB7DEB70C945A7BCF93FC0197FF5E
:10D9800005C0CFEFF095E195FF4F01C0C1E028E65B
:10D9900031E0CF01B9010E94E27AFC018B3591059B
:10D9A00054F08B5590408A35910538F484EB90E023
:10D9B0008E1B9F0BFC0141E00DC0CF01855B9040A9
:10D9C0008A35910518F4E45BF04003C02E1B3F0B31
:10D9D000F9014FEFEE0FFF1FE15CF54F25913491F8
:10D9E0008C2F992787FD9095289FB001299F700D56
:10D9F000389F700D1124842F992787FD9095689F7B
:10DA0000A001699F500D789F500D1124CA01CF913C
:10DA100008952AE530E0281B390BC9010E94BD6C2E
:10DA20000895CF93DF9380E00E94F27280911D01F0
:10DA300090911E016AE070E00E94E27A9F938F93BA
:10DA400080911D0190911E016AE070E00E94E27ACF
:10DA50007F936F938DE09BE09F938F93C5EED2E70A
:10DA6000DF93CF93E0913004F091310409952DB705
:10DA70003EB7285F3F4F2DBF8091EA018823B9F15F
:10DA800086E00E94F27280910508909106086AE093
:10DA900070E00E94CE7A7F936F938FED90E09F931A
:10DAA0008F938091F6079091F707A091F807B091B6
:10DAB000F90720919501309196014091970150917D
:10DAC0009801BC01CD010E94177B3F932F9386E103
:10DAD0009BE09F938F93DF93CF93E0913004F0917D
:10DAE000310409958DB79EB70A968DBF12C086E0A6
:10DAF0000E94F27282E29BE09F938F93DF93CF9319
:10DB0000E0913004F091310409950F900F900F903F
:10DB10000F90809103048823C1F086E00E94F27286
:10DB20008091030499279F938F9389E29BE09F93B1
:10DB30008F93DF93CF93E0913004F09131040995F6
:10DB40002DB73EB72A5F3F4F2DBF80E10E94F27292
:10DB50008091F5019091F6016CE370E00E94CE7A1D
:10DB60009F938F938091F5019091F6016CE370E0A3
:10DB70000E94CE7A7F936F93809171089091720882
:10DB80009F938F9384E39BE09F938F93C5EED2E79F
:10DB9000DF93CF93E0913004F091310409958091A7
:10DBA00015062DB73EB7265F3F4F2DBF80FF29C01A
:10DBB0008AE10E94F2728091940199279F938F933A
:10DBC0008091120390911303A0911403B091150357
:10DBD000BC01CD0124E630E040E050E00E94177B1C
:10DBE0003F932F9381E49BE09F938F93DF93CF9399
:10DBF000E0913004F091310409958DB79EB70896F5
:10DC00008DBFDF91CF910895CF93DF9380E00E9485
:10DC1000F2728091EE06992787FD90959F938F93DE
:10DC20008091E606992787FD90959F938F93809129
:10DC3000DE06992787FD90959F938F938091D60656
:10DC4000992787FD90959F938F9388E49BE09F93FE
:10DC50008F93C5EED2E7DF93CF93E0913004F0913C
:10DC60003104099580E10E94F2722DB73EB7245F1E
:10DC70003F4F2DBF80910E07992787FD90959F9369
:10DC80008F9380910607992787FD90959F938F9397
:10DC90008091FE06992787FD90959F938F938091A1
:10DCA000F606992787FD90959F938F9388E59BE0D3
:10DCB0009F938F93DF93CF93E0913004F0913104E1
:10DCC0000995809107062DB73EB7245F3F4F2DBFC2
:10DCD000853098F480E10E94F27288E69BE09F9381
:10DCE0008F93DF93CF93E0913004F0913104099545
:10DCF0000F900F900F900F9018C08730B0F488E10C
:10DD00000E94F2728FED90E09F938F9389E79BE0E2
:10DD10009F938F93DF93CF93E0913004F091310480
:10DD200009958DB79EB706968DBFDF91CF91089567
:10DD30000F931F9380E00E94F2722AE030E08091FE
:10DD40006D0890916E08B9010E94CE7A9F938F93CF
:10DD500080916D0890916E08B9010E94CE7A7F93F0
:10DD60006F9380911D0190911E01B9010E94E27A8A
:10DD70009F938F9380911D0190911E01B9010E9484
:10DD8000E27A7F936F9382E89BE09F938F9305EEF7
:10DD900012E71F930F93E0913004F091310409953D
:10DDA00080E10E94F2728DB79EB70C968DBF809174
:10DDB0007108909172089F938F9380916F08909152
:10DDC00070089F938F9385E99BE09F938F931F9398
:10DDD0000F93E0913004F091310409958DB79EB70F
:10DDE00008968DBF1F910F9108950F931F93CF93A6
:10DDF000DF938091EA01C5EED2E7882309F478C069
:10DE000080E00E94F2728091020899279F938F937D
:10DE10008091040899279F938F9381EA9BE09F93B9
:10DE20008F938E01DF93CF93E0913004F091310412
:10DE300009958DB79EB708968DBF809103088330F2
:10DE400031F48CE00E94F27280EB9BE005C08CE024
:10DE50000E94F27285EB9BE09F938F93DF93CF93A9
:10DE6000E0913004F091310409950F900F900F90DC
:10DE70000F908091010881FF12C08CE00E94F27225
:10DE80008AEB9BE09F938F931F930F93E091300455
:10DE9000F091310409950F900F900F900F9080E151
:10DEA0000E94F2728FED90E09F938F93809107080C
:10DEB000909108089F938F93809105089091060890
:10DEC0006AE070E00E94CE7A7F936F938FEB9BE0C5
:10DED0009F938F9385EE92E79F938F93E091300409
:10DEE000F091310409958DB79EB70A968DBF12C087
:10DEF00082E00E94F2728FEC9BE09F938F93DF93FE
:10DF0000CF93E0913004F091310409950F900F9078
:10DF10000F900F90DF91CF911F910F910895CF93A4
:10DF2000C82F209118042093190499278F32910546
:10DF300009F1803391051CF44F97A1F02CC08F3468
:10DF4000910501F18F38910531F5222319F481E013
:10DF500090E038C086E0289FF0011124EB50F54F87
:10DF6000849117C086E0289FF0011124EA50F54FF4
:10DF700084910FC086E0289FF0011124E950F54FED
:10DF8000849107C086E0289FF0011124E850F54FE6
:10DF90008491809318049091180480911904981327
:10DFA000C0E00E94F8729091180486E0989FF001FA
:10DFB0001124E750F54F259134918C2FF9010995E3
:10DFC00080E090E0CF91089510926E0810926D0855
:10DFD00010927208109271081092700810926F08D7
:10DFE000109273088AE090E00E94621690931B04DE
:10DFF00080931A040895CF93DF9380911A0490912F
:10E000001B040E946B16882309F4AFC080911A0488
:10E0100090911B040A9690931B0480931A04E0E0ED
:10E02000F0E09F0190E05FEFAFECB6E04BE0ED0178
:10E030008B8187FF0BC09F5F8D81E80FF11D898168
:10E04000280F311D8E81851708F4582F41501896DE
:10E0500047FFEDCF50937308232B41F52091200407
:10E06000309121044091220450912304BB27A52F15
:10E07000942F832F90931F0480931E04AA27BB27FD
:10E08000281B390B4A0B5B0BCF01AA27BB27280F94
:10E09000391F4A1F5B1F20932004309321044093B3
:10E0A000220450932304E5E0F0E013C020911E0405
:10E0B00030911F042E173F0718F4E21BF30B02C028
:10E0C000E0E0F0E0892F9927880F991FE80FF91FEA
:10E0D0003596F0936E08E0936D08EF3FF10578F404
:10E0E00080911D0190911E018E9F90018F9F300D98
:10E0F0009E9F300D1124C90164E670E013C0CF016A
:10E10000969587959695879520911D0130911E01D2
:10E11000289FA001299F500D389F500D1124CA013E
:10E1200069E170E00E94CE7A7093700860936F0886
:10E1300020911C0430911D042E0F3F1F30931D04AD
:10E1400020931C045EE02131350778F0809171083E
:10E1500090917208019690937208809371082051F3
:10E160003E4030931D0420931C04DF91CF9108950D
:10E17000002422273327442751E0BB27EE27FF271F
:10E18000A0E1660F771F881F991F001C221F331FF5
:10E19000441F660F771F881F991F001C221F331F03
:10E1A000441F2AF4050E2B1F3E1F4F1F04C0051AE3
:10E1B0002B0B3E0B4F0B550FBB1FEE1F587F5560AF
:10E1C00047FD5250AA95E9F6E695B7955795E6951D
:10E1D000B7955795852F9B2F08952227332741E028
:10E1E000552768E0880F991F221F331F880F991F3A
:10E1F000221F331F1AF4240F351F02C0241B350BB6
:10E20000440F551F487F456037FD42506A9551F7CE
:10E210005695479556954795842F0895AA2797FFB9
:10E2200004C0809590958A1F9A1F77FF04C060955F
:10E2300070956A1F7A1F669F9001779FA001679F64
:10E24000300D411D5A1F300D411D5A1F889FF0018E
:10E25000999F2E0F3F1F401D511D899F300D411D5D
:10E260005A1F300D411D5A1FCA01B901112480CF18
:10E270004FB720E430E0F8948091C9008F77809305
:10E28000C9008091C9008F7B8093C9008091C9002B
:10E290008F7D8093C9005A9A52985B9A539A832F24
:10E2A00099278093CD002093CC008091C800826094
:10E2B0008093C80088E18093C9008091CA008F775D
:10E2C0008093CA008091CA008F7B8093CA0080919E
:10E2D000CA008F7D8093CA008091CA008F7E809390
:10E2E000CA008091CA00877F8093CA008091C900CC
:10E2F0008B7F8093C9008091CA0084608093CA009C
:10E300008091CA0082608093CA008091C80087FF14
:10E3100003C08091CE00F9CF8091C90080688093BE
:10E32000C9004FBF08950F931F93CF93DF93482FDA
:10E330004F5F893108F089C080912F07841710F44E
:10E3400040932F07CB0183539B4268E170E00E940A
:10E35000E27AA42FBB27FD01EA0FFB1FE05DF84F17
:10E36000808191819B01281B390BC90137FF03C0B4
:10E37000909581959F4F069794F480912003883C57
:10E3800030F480912003865F8093200308C088ECDE
:10E390008093200380916F008F7D80936F00FD013B
:10E3A000EA0FFB1FE05DF84F808191819C01220FF5
:10E3B000331F280F391F260F371F37FF02C02D5F6D
:10E3C0003F4FE901D595C795D595C795CB010196E6
:10E3D0008C179D0714F4219706C061507040C61732
:10E3E000D7070CF4219680912003843BD8F08D014F
:10E3F0000A0F1B1FF801E05DF84F80819181FE013B
:10E40000E81BF90BCF0163E070E00E94E27ACB01D8
:10E41000880F991F860F971F0C59184FF801918389
:10E42000808307C0AA0FBB1FAC59B84F11961C922E
:10E430001E92E42FFF27EE0FFF1FE05DF84FD18300
:10E44000C083443011F410929301DF91CF911F915A
:10E450000F910895CF93DF9320917408822F99270D
:10E46000807F9070409709F06CC02F3109F046C052
:10E4700080917508809328042091770820932A04BE
:10E480008091780880932904822F992790933107EF
:10E4900080933007222309F054C080910906282F69
:10E4A0003327220F331FF901EC59F84F11821082E4
:10E4B00080910A06A82FBB27AA0FBB1FFD01EC59AC
:10E4C000F84F1182108280910C06E82FFF27EE0F83
:10E4D000FF1FCF018C59984FEC0119821882205DE3
:10E4E000384FE90119821882A05DB84F11961C922D
:10E4F0001E92E05DF84F1182108223C0C22FCF70B0
:10E50000CA30F8F48091750880939E08809176084F
:10E5100080939D08809177088093A0088091780867
:10E5200080939F0860919D0870919E088C2F0E9497
:10E53000937160919F087091A0088C2F8F5F0E944B
:10E540009371DF91CF910895CF93C82F8F3F49F4F6
:10E5500080912B048F3F29F410922D0410922C04EB
:10E5600032C020912D04222339F4CF3111F485E0FB
:10E5700001C084E080932E0480912E0490912C049D
:10E580008217A0F4892F809580932C048F3F19F473
:10E590008EEF80932C0480912C04C81711F40E94F4
:10E5A0002A7210922D0410922C040BC0E22FFF2728
:10E5B000EC58F74FC0832F5F20932D049C0F90934E
:10E5C0002C04C0932B04CF9108959091270493328B
:10E5D00040F4E92FFF27E658F74F80839F5F909321
:10E5E00027040895833218F48D5F809327040895DB
:10E5F00090E2EDE7F8E08FE19193815087FFFCCF47
:10E600000895CF93CFB723E031E0F8948091C9000B
:10E610008F778093C9008091C9008F7B8093C90058
:10E620008091C9008F7D8093C9005A9A52985B9A55
:10E63000539A832F99278093CD002093CC0080910B
:10E64000C80082608093C80088E18093C9008091EF
:10E65000CA008F778093CA008091CA008F7B809315
:10E66000CA008091CA0080628093CA008091CA006B
:10E6700080618093CA008091CA0088608093CA003C
:10E680008091C90084608093C9008091CA00846031
:10E690008093CA008091CA0082608093CA008091F2
:10E6A000C80087FF03C08091CE00F9CF8091C900D8
:10E6B00080688093C9008091C90080648093C900FC
:10E6C0000E94F872CFBFCF910895282F99278F709D
:10E6D0009070892B31F4209580912604822B8093B1
:10E6E000260408958091F101882309F441C08091A6
:10E6F000E80285FF0AC082E980937A0883E280936A
:10E700007B0885E580937C0802C010927A0880918E
:10E71000F2018F3071F4809126040E948F6F88235C
:10E7200041F081E980937A0880937B0881E38093AC
:10E730007C081092F1018091C80085FFFCCF809188
:10E74000C9008F7E8093C9008091C9008E7F80931D
:10E75000C90080917A08882311F48EEF01C08EE7FA
:10E760008093CE00809126048093F20110922604BB
:10E7700008951F920F920FB60F9211248F939F93BB
:10E78000EF93FF939091F101992309F040C080919C
:10E790002F04882361F480917A08882311F483E0A0
:10E7A00003C0813999F481E080932F040FC0833036
:10E7B00099F480917A08882349F090937A0880919F
:10E7C000C9008E7F8093C9008EEF1EC08091C90062
:10E7D00081608093C9000EC0833261F48091C900CA
:10E7E0008E7F8093C9008FEF8093CE0081E080936D
:10E7F000F10114C080912F04E82FFF27E658F74F4E
:10E800008F5F80932F0480818093CE0007C0109289
:10E810002F048091C90080618093C900FF91EF911E
:10E820009F918F910F900FBE0F901F901895EF92B0
:10E83000FF920F931F93CF93DF937C018B01EA012B
:10E84000452B39F0F80181918F01F7010995219746
:10E85000C9F7E6E0CDB7DEB70C945A7BEF92FF9292
:10E860000F931F93CF93DF937C018B01EA01452B1C
:10E8700041F0F8010F5F1F4F8491F701099521972F
:10E88000C1F7E6E0CDB7DEB70C945A7B0F931F9328
:10E89000CF938C01C62F161634F480E2F801099547
:10E8A000C1501C16D4F3CF911F910F9108950F936F
:10E8B0001F93CF938C01C62F161634F480E3F80112
:10E8C0000995C1501C16D4F3CF911F910F91089553
:10E8D000A5E3B0E0EEE6F4E70C94327B2E96EEADC5
:10E8E000FFAD2E9788249924540180912504882314
:10E8F00021F42C961FAE1EAE2C975EE4452E512CB3
:10E900004C0E5D1E6F01B60105C0153239F008943A
:10E91000C11CD11CF60114911123B9F7A601461BA5
:10E92000570B31F02C968EAD9FAD2C970E942E7414
:10E93000112309F46AC20894C11CD11CFF24FDA64E
:10E94000FCA64FEFE42EF9A6F6010894C11CD11CD9
:10E950001491153721F0812F80628837B1F4F0FED1
:10E960000AC0F20124E030E0420E531E8080918004
:10E97000A280B3800AC0F20142E050E0440E551E6E
:10E98000808191814C01AA24BB24103221F489A5F5
:10E990008823D1F61DC0133219F458E0F52AD4CFDC
:10E9A0001A3211F01D3291F41A3259F4F20182E058
:10E9B00090E0480E591EE081ECA7EE232CF6E1957D
:10E9C000ECA790E1F92AAFEDFA22BECF1B3211F489
:10E9D00019A7BACF1E32C1F5F6010894C11CD11C8B
:10E9E00014911A3279F4F20122E030E0420E531E03
:10E9F000408151813FEF4F3F530714F44FEF5FEFDA
:10EA0000E42EA2CF40E050E0812F80538A30A0F462
:10EA1000CA0133E0880F991F3A95E1F7840F951FDB
:10EA2000480F591F410F511D40535040F6010894A3
:10EA3000C11CD11C1491E8CF8FEF4F3F580714F43D
:10EA40004FEF5FEFE42E85CF103329F4F4FC7CCF39
:10EA500090E2F92A79CF812F81538930D8F440E0B0
:10EA600050E0CA0123E0880F991F2A95E1F7840F2F
:10EA7000951F480F591F410F511D40535040F6013B
:10EA80000894C11CD11C1491812F80538A3048F303
:10EA90004CA75FCF183619F4A4E0FA2A55CF1C36DC
:10EAA00019F4B1E0FB2A50CF133661F43E0108940B
:10EAB000611C711CF20122E030E0420E531E808185
:10EAC00089833CC1143421F0143611F0193651F504
:10EAD000143411F431E0F32AF0FE0AC0F20144E0EC
:10EAE00050E0440E551E80809180A280B3800CC0FF
:10EAF000F20182E090E0480E591E808191814C0124
:10EB0000AA2497FCA094BA2CB7FE0AC0B094A09493
:10EB100090948094811C911CA11CB11C8DE289A74A
:10EB20000AE06FC01F3411F01F3631F41F3411F4A6
:10EB300091E0F92A08E064C0103779F4F201A2E00C
:10EB4000B0E04A0E5B1E808191814C01AA24BB2457
:10EB500000E1B0E4FB2A18E753C01337C1F5F20116
:10EB600022E030E0420E531E608071806114710417
:10EB700089F43E010894611C711C88E289838EE649
:10EB8000F301818385E78B838CE68C838D8389E217
:10EB90008E831F82E7FC13C08E2D992787FD9095E9
:10EBA000AC0160E070E0C3010E94FF78009729F09B
:10EBB000382E3618E3140CF0C3C03E2CC1C0F3014C
:10EBC00001900020E9F731973E2E3618B9C015356F
:10EBD00011F0153731F4153511F4F1E0FF2A0AE090
:10EBE0000FC0183519F0183709F0A0C000E1F3FE86
:10EBF00007C081149104A104B10411F020E4F22AA9
:10EC000019A6EDA6E7FC02C03FEDF32289E2682ECB
:10EC1000712C6C0E7D1E81149104A104B10421F4A9
:10EC20004DA5442309F47BC0802F9927AA27BB2731
:10EC30008EA79FA7A8ABB9AB202E332490E08916EE
:10EC400090E0990691E0A90690E0B90648F0C50168
:10EC5000B4012EA53FA548A959A90E94F57A17C06D
:10EC6000AFEF8A169104A104B10449F040F0C40149
:10EC7000B1010E94CE7A9B014427552708C0882DF8
:10EC8000602F0E94C27A282F3327442755272AABAA
:10EC90003BAB4CAB5DAB0A3059F48AA9880F880FA7
:10ECA000880F9AA9990F890F382D381B832F10C010
:10ECB000003139F48AA98295807F482D481B842F22
:10ECC00007C08AA9880F880F880F582D581B852FD9
:10ECD00090E02EA53FA548A959A982169306A4063F
:10ECE000B50608F091E08AA89BA8ACA8BDA88A3018
:10ECF00010F4805D04C0895A183509F48F7DD30162
:10ED00008E933D01992309F099CF083041F4F3FE29
:10ED100006C0803321F080E3FD0182933F01CE01E4
:10ED20000196382E3618F8E23F0E0BC0112309F475
:10ED30006CC03E010894611C711C1983B1E03B2E2C
:10ED400019A6032D2DA4231827FC222489A5882386
:10ED500011F00F5F02C0F6FC0E5F020DEF2CFF24D6
:10ED6000C70180739070892B49F48CA5801B682F94
:10ED70002C968EAD9FAD2C970E94467489A5882352
:10ED800031F041E050E0BE01675D7F4F0AC0E6FE12
:10ED90000EC080E38AA71BA742E050E0BE01665D7B
:10EDA0007F4F2C968EAD9FAD2C970E941774C70194
:10EDB00080739070809749F48CA5801B682F2C96E7
:10EDC0008EAD9FAD2C970E945774622D2C968EAD00
:10EDD0009FAD2C970E945774832D992787FD90959E
:10EDE000AC01B3012C968EAD9FAD2C970E94177489
:10EDF000E4FE89CD2CA5201B2CA7622F2C968EAD6E
:10EE00009FAD2C970E9446747ECDE2E1CB5C0C94C2
:10EE10004E7B2FB740E0F894E0E0F0E081E2809391
:10EE200057009491E2E0F0E0809357003491E4E0E1
:10EE3000F0E08093570084912FBF9E3199F43639CA
:10EE400041F4893011F441E00DC08A3059F442E0B8
:10EE500009C0373939F4863011F443E003C08530F6
:10EE600009F444E0842F992708959FB7F89480917E
:10EE7000C900877F8093C9008091C9008F7E8093ED
:10EE8000C9008091C9008F778093C9008091C90023
:10EE90008F7B8093C9008091C9008F7D8093C900CA
:10EEA00052985A9A53985B9A9FBF08951F93CF9395
:10EEB000DF93182F80912504882309F48DC0809159
:10EEC000F001181709F488C080912404882321F4E4
:10EED0000E9409778093240488EC9CE09F938F9391
:10EEE000CBE3D2E1DF93CF93E0913004F091310492
:10EEF00009950F900F900F900F90812F99278230D6
:10EF0000910501F1833091052CF4009761F0019790
:10EF100069F024C084309105D9F084309105ACF0BB
:10EF20000597C9F01BC088EB9CE002C086EA9CE014
:10EF30009F938F93DF93CF93E0913004F09131044E
:10EF4000099518C08DE89CE0F3CF8AE69CE0F0CFED
:10EF50008CE59CE0EDCF84E59CE0EACF85ED9CE07C
:10EF60009F938F93DF93CF93E0913004F09131041E
:10EF7000099510E00F900F900F900F90809124044E
:10EF8000843011F0823099F40E943577812F8150BE
:10EF9000833018F40E94196B1DC0143019F40E94BC
:10EFA000017318C01530B1F40E94387113C01123D9
:10EFB00089F08BEE9CE09F938F938BE392E19F937C
:10EFC0008F93E0913004F091310409950F900F90E8
:10EFD0000F900F901093F001DF91CF911F91089542
:10EFE0000F931F9381E0809325044091EF01E4E0AB
:10EFF000FCE020E030E05FE4849199272F5F3F4FF1
:10F00000829FB001839F700D929F700D112446273F
:10F010005150319657FFF0CF4093EF01ECEDFBE0FC
:10F0200020E030E057E2849199272F5F3F4F829F85
:10F03000B001839F700D929F700D1124462751508F
:10F04000319657FFF0CF4093EF018091240488233D
:10F0500021F40E940977809324048091EF01833486
:10F0600059F088E190E029E20FB6F894A8958093D2
:10F0700060000FBE2093600088E694E7909331040F
:10F080008093300486E09DE09F938F930BE312E121
:10F090001F930F93E0913004F091310409950F9084
:10F0A0000F900F900F9086E690E09F938F9380E5EE
:10F0B00090E09F938F931F921F92809102016AE0CC
:10F0C0000E94C27A892F99279F938F938091020182
:10F0D0000E94C27A99279F938F938CE29DE09F9321
:10F0E0008F931F930F93E0913004F09131040995B1
:10F0F00084E09CE09F938F931F930F93E0913004E3
:10F10000F091310409958CED9BE09F938F931F93B1
:10F110000F93E0913004F091310409958DB79EB7BB
:10F1200046968DBF80E69DE09F938F931F930F932C
:10F13000E0913004F0913104099583EC80938100D3
:10F1400080916F00806280936F000F900F900F90FE
:10F150000F901F910F91089580912504882361F0ED
:10F160008091F001843011F40E9472738091EF015C
:10F17000833411F01092250408951F920F920FB658
:10F180000F9211242F933F934F935F936F937F932D
:10F190008F939F93AF93BF93EF93FF932091CE00F4
:10F1A0009091F001892F8150833020F4822F0E94AA
:10F1B000746B0BC0943021F4822F0E94657305C0DC
:10F1C000953019F4822F0E94A472FF91EF91BF91A4
:10F1D000AF919F918F917F916F915F914F913F91EF
:10F1E0002F910F900FBE0F901F901895FB01DC011F
:10F1F00002C005900D9241505040D8F70895FC018F
:10F200004150504030F001900616D1F73197CF01B0
:10F210000895882799270895A0E0B0E0E2E1F9E792
:10F220000C943A7B6C017B01EA01590121978FEF25
:10F23000CF3FD80789F086010894C11CD11CC701B3
:10F240000894E11CF11CF5010995F80180832197D0
:10F25000FFEFCF3FDF0779F7EAE0CDB7DEB70C94D9
:10F26000567BCF92DF92EF92FF920F931F937C0118
:10F270006B01FB010995082FC7010196F60109955D
:10F28000182FC8011F910F91FF90EF90DF90CF9042
:10F290000895A0E0B0E0EFE4F9E70C943C7B8C012A
:10F2A0007B01EA01690121978FEFCF3FD80771F009
:10F2B000F70121917F01C8010F5F1F4F622FF601F7
:10F2C00009952197FFEFCF3FDF0791F7E8E0CDB732
:10F2D000DEB70C94587BCF92DF92EF92FF920F93A0
:10F2E0001F936C018B017A01FA010995812F9927EF
:10F2F000682FC6010196F70109951F910F91FF90A4
:10F30000EF90DF90CF9008955058BB27AA270ED0DA
:10F31000E0C0D1D030F0D6D020F031F49F3F11F4CE
:10F320001EF4C6C00EF4E095E7FBBCC0E92FE2D0A6
:10F3300080F3BA17620773078407950718F071F412
:10F340009EF5FAC00EF4E0950B2EBA2FA02D0B01FE
:10F35000B90190010C01CA01A0011124FF27591B1A
:10F3600099F0593F50F4503E68F11A16F040A22F20
:10F37000232F342F4427585FF3CF46953795279591
:10F38000A795F0405395C9F77EF41F16BA0B620B90
:10F39000730B840BBAF09150A1F0FF0FBB1F661FD7
:10F3A000771F881FC2F70EC0BA0F621F731F841F1A
:10F3B00048F4879577956795B795F7959E3F08F040
:10F3C000B3CF9395880F08F09927EE0F97958795FF
:10F3D000089598D088F09F5790F0B92F9927B7518A
:10F3E000A0F0D1F0660F771F881F991F1AF0BA9509
:10F3F000C9F712C0B13081F09FD0B1E008959CC030
:10F40000672F782F8827B85F39F0B93FCCF38695FE
:10F4100077956795B395D9F73EF49095809570955B
:10F4200061957F4F8F4F9F4F0895E89409C097FBD8
:10F430003EF490958095709561957F4F8F4F9F4FCB
:10F440009923A9F0F92F96E9BB279395F69587950F
:10F4500077956795B795F111F8CFFAF4BB0F11F4D2
:10F4600060FF1BC06F5F7F4F8F4F9F4F16C0882379
:10F4700011F096E911C0772321F09EE8872F762FAF
:10F4800005C0662371F096E8862F70E060E02AF0F0
:10F490009A95660F771F881FDAF7880F96958795DC
:10F4A00097F9089597F99F6780E870E060E0089504
:10F4B0009FEF80EC089500240A941616170618068C
:10F4C0000906089500240A94121613061406050668
:10F4D0000895092E0394000C11F4882352F0BB0FF9
:10F4E00040F4BF2B11F460FF04C06F5F7F4F8F4F5C
:10F4F0009F4F089557FD9058440F551F59F05F3F97
:10F5000071F04795880F97FB991F61F09F3F79F045
:10F5100087950895121613061406551FF2CF4695C7
:10F52000F1DF08C0161617061806991FF1CF869549
:10F530007105610508940895E894BB27662777272D
:10F54000CB0197F90895629FD001739FF001829FCC
:10F55000E00DF11D649FE00DF11D929FF00D839F62
:10F56000F00D749FF00D659FF00D9927729FB00DFF
:10F57000E11DF91F639FB00DE11DF91FBD01CF0112
:10F5800011240895991B79E004C0991F961708F07B
:10F59000961B881F7A95C9F780950895AA1BBB1BF7
:10F5A00051E107C0AA1FBB1FA617B70710F0A61B83
:10F5B000B70B881F991F5A95A9F780959095BC01A4
:10F5C000CD01089597FB092E07260AD077FD04D0B8
:10F5D000E5DF06D000201AF4709561957F4F0895FD
:10F5E000F6F7909581959F4F0895A1E21A2EAA1BD8
:10F5F000BB1BFD010DC0AA1FBB1FEE1FFF1FA217E3
:10F60000B307E407F50720F0A21BB30BE40BF50BDF
:10F61000661F771F881F991F1A9469F76095709568
:10F62000809590959B01AC01BD01CF01089597FB9A
:10F63000092E05260ED057FD04D0D7DF0AD0001CB6
:10F6400038F450954095309521953F4F4F4F5F4F7F
:10F650000895F6F790958095709561957F4F8F4F3F
:10F660009F4F08952F923F924F925F926F927F9299
:10F670008F929F92AF92BF92CF92DF92EF92FF92C2
:10F680000F931F93CF93DF93CDB7DEB7CA1BDB0B6E
:10F690000FB6F894DEBF0FBECDBF09942A88398813
:10F6A00048885F846E847D848C849B84AA84B9841A
:10F6B000C884DF80EE80FD800C811B81AA81B98126
:10F6C000CE0FD11D0FB6F894DEBF0FBECDBFED013A
:10F6D0000895EE0FFF1F0590F491E02D0994FFCFE0
:10F6E0005E010A010164FF01FFFF01FC01FC010151
:10F6F000737373FF03007D0000C409C40964001123
:10F7000048656C6C6F20576F726C640000000000DD
:10F7100000000000000000000000000000000000E9
:10F7200000000000000000000000000000000000D9
:10F7300000000000000000000000000000000000C9
:10F7400000000000000000000000000000000000B9
:10F7500053706F727400004E6F726D616C000042E6
:10F760006567696E6E6572000051756164726F0045
:10F7700000640001200B050000ECFF6440415A4684
:10F7800064640A02969696960840403A10FB303818
:10F7900001380190D0030090D00300F4017800FFFD
:10F7A000036400020406070808080706040200FEB6
:10F7B000FCFAF9F8F8F8F9FAFCFE0002040607086A
:10F7C000080B0A0D0B0C0E0B0F10FA200101017033
:04F7D000FF010F0026
:00000001FF
